:020000040800F2
:100000002618002405030008A9020008A902000818
:10001000A9020008A9020008A9020008A902000814
:10002000A9020008A9020008A9020008A902000804
:10003000A9020008A9020008A9020008A9020008F4
:10004000A9020008A9020008A9020008A9020008E4
:10029000A9020008A90200080000000000000000F8
:1002A000FFECC2925D7D05C5EFF305801EF0040FE3
:1002B00002D0EFF309818D466A4602F16802EFF33E
:1002C00011831EF0100F0CBF2DED108A90B02DE998
:1002D000FC4F6946DFF828D000F070FAB0E8FC4F18
:1002E0001EF0100F0CBFB0EC108A40301EF0040F4F
:1002F0000CBF80F3088880F3098883F31188704766
:100300000004002408B51E4B1E48DA1CC11E121A38
:1003100022F00302994288BF0022002100F0A5FCD0
:10032000194B1A48DA1CC11E121A22F00302994214
:1003300088BF0022164900F083FB00F019F900F095
:1003400055FA00F073F9BFF34F8FBFF36F8F4FF083
:10035000E023D3F8902F22F00102C3F8902FD3F8B6
:10036000942F22F00102C3F8942FBFF34F8FBFF3F5
:100370006F8F00F0C3FC00F00CFA00F0CBFC00BF64
:10038000381500240001002400010024000000248E
:1003900088A500086F4A82B0D2F8003423F4802385
:1003A00043F48033C2F800346B4B0193019B002B64
:1003B00003DDD2F800349B0304D5019B002B04DC41
:1003C00002B07047019B013BEFE7624BD3F8182462
:1003D00022F4706222F00F0242F00802C3F81824DF
:1003E000D3F81C2422F4E06242F04002C3F81C243B
:1003F000D3F81C2422F4E06242F48062C3F81C2487
:10040000D3F8182422F0700242F04002C3F81824F6
:10041000D3F8202422F0700242F04002C3F82024D6
:100420004E4AC3F828244E4AC3F830244D4AC3F834
:10043000382402F50032C3F840244B4AC3F82C2478
:10044000D3F8002442F0A852C3F80024D3F80024C3
:100450009001FBD5D3F800241101FBD53D4BD3F817
:1004600000249200FBD5D3F80C2842F00602C3F812
:100470000C28D3F8182842F44042C3F81828D3F8BF
:1004800018289004FBD5334BD3F804289104FBD5EE
:10049000D3F8F4244FF0B04142F00202C3F8F42440
:1004A000D1F82C2442F00102C1F82C24D3F81828EA
:1004B0009204FBD52D4A22211160D3F8102422F09A
:1004C000070242F00302C3F81024224BD3F8102491
:1004D00002F03802182AF9D1D3F8542422F44052F9
:1004E00042F40052C3F85424D3F8582422F4407242
:1004F00042F40072C3F85824D3F8502422F4E042A6
:1005000042F48052C3F85024D3F8502422F4E0225D
:1005100042F48032C3F85024D3F8582422F0E04249
:1005200042F08052C3F85824D3F8542422F44012E5
:1005300042F40012C3F85424D3F8582422F4403271
:10054000C3F85824D3F8502422F04052C3F8502462
:1005500036E700BF0040025848BE210012202000AC
:10056000770203072F0201018808BF000020005214
:1005700010B52A4C00200122D4F8003443F00103C6
:10058000C4F80034264BC3F80821C4F81004254BE6
:10059000D4F80024134043F01003C4F80034224B75
:1005A000C4F82C34D4F8003423F48023C4F8003485
:1005B000C4F8600400F07EF8FFF7ECFED4F8D834FD
:1005C00043F0006343F00103C4F8D834D4F8DC34BA
:1005D000C4F8DC34D4F8D434C4F8D434D4F8E034D7
:1005E00043F0805343F09F03C4F8E034D4F8E83478
:1005F000C4F8E834D4F8EC34C4F8EC34D4F8F0346B
:1006000043F01003C4F8F034D4F8E434C4F8E4340C
:10061000D4F8F434C4F8F43410BD00BF00400258DC
:100620000080005167EFFEEA0000FF017047FFEC19
:1006300030B4EFF3118400238022EFF3108372B6FD
:1006400082F3118883F31088BFF34F8F174B18493B
:10065000D3F800280B8802F4807578B101339BB27F
:100660000B8075B1CBB10023BFF34F8FE4B284F39D
:100670001188C3B1042030BC00F04FB85BB1013B1E
:10068000EDE70B88002BEED0084B42F48072C3F8E4
:1006900000280123E8E7002DE5D022F48072034B07
:1006A000C3F80028DFE730BC704700BF00400258A5
:1006B00000040024EFF3118200238021EFF3108364
:1006C00072B681F3118883F310880749D1F8003896
:1006D00023F48073C1F800380021044B1980D3B291
:1006E00083F31188FFF7A4BF0040025800040024E0
:1006F00030B5EFF3118400238025EFF3108372B639
:1007000085F3118883F31088036823EA0101E3B2BB
:100710000A43026083F3118830BD82B0002245F2A3
:100720006161B0F57A7F0BD8002240F6A2016428FF
:1007300011D800220A2818D8002200BB02B0704746
:100740000192019B8B4202DDA0F57A70E9E7019BE3
:1007500001330193F5E70192019B8B4201DD64387F
:10076000E5E7019B01330193F6E70192019BDC2B46
:1007700001DD0A38DEE7019B01330193F6E70192C0
:10078000019B152B01DD0138D7E7019B0133019354
:10079000F6E7BFF34F8FBFF36F8F4FF0E0230022D8
:1007A000C3F8502FD3F8142D42F40032C3F8142D9F
:1007B000BFF34F8FBFF36F8F7047FFEC70B50A4DDB
:1007C00006460C462B680BB91C462960304600F0E3
:1007D000F6F82968304600F07FFB14B900232C6836
:1007E0002B60204670BD00BF04040024EFF3148387
:1007F00043F0040383F314884FF0E023D3F8342F3D
:1008000022F04042C3F8342FD3F8882D42F470020E
:10081000C3F8882D7047FFEC0F2810B52DDDA0F12F
:1008200010041F2C08DC03F1604303F561430B60E7
:100830000123A340136009E03F2C09DC1D4C303834
:100840001C440C60012303FA00F01060002010BD6E
:100850005F2C04DC184C50381C440C60F2E77F2CF1
:1008600004DC164C70381C440C60EBE7952C1EDC45
:10087000134C90381C440C60E4E7124B04380B60B6
:100880000B2814D8DFE800F006090C131313131318
:100890001313130F4FF48033CCE74FF40033C9E741
:1008A0004FF48023C6E7084B0B600123C2E74FF0EB
:1008B000FF30CCE704E100E008E100E00CE100E0FB
:1008C00010E100E024ED00E010E000E04FF0E02354
:1008D00021494FF0FF3010B55B6803F00F035A1C3D
:1008E00003F1382361339B0041F8040B9942FBD19B
:1008F0004FF0E0231949C3F8081D4FF08031C3F8C9
:10090000181DC3F81C1DC3F8201D5301144A03F120
:10091000604303F5644342F8041B9342FBD1002477
:10092000104B11490B2022461C6000F0ADFA224604
:100930000E49032000F0A8FA4FF0E022D2F81C3D47
:1009400023F07F4343F0E043C2F81C3DF02383F3E0
:10095000118862B610BD00BF80E100E00000000811
:1009600000E400E004040024F1090008C1090008C3
:1009700013B5802301AA69460446FFF74DFF20B94D
:100980000F2CDDE9003102DD196002B010BD1A68DC
:1009900022EA01021A60F8E713B5002301AA6946AA
:1009A0000446FFF739FF20B90F2CDDE9003102DDE5
:1009B000196002B010BD1A680A431A60F9E770475F
:1009C00008B54FF0E023D3F82C2DD3F8283DEFF3F2
:1009D000118300238022EFF3108372B682F3118813
:1009E00083F31088AD21014800F032F9689F0008B8
:1009F000CA6E012A08B508D0022A0AD01AB9D42230
:100A0000086F00F01DF8002008BD0A6F034B1A6044
:100A1000F9E70A6F11604A6FF8E700BF0404002489
:100A200018DF88DFCD06CD767CD30CD3D982D912DE
:100A30002C00050A0F14191E232800BFAFF30080F5
:100A400000B501B400F004F801BC00BDAFF30080B4
:100A500000B5042A60DB00F0030E61F3830E7A4BCD
:100A6000D3E80EF0AFF30080AFF30080AFF3008067
:100A700011F8013B00F8013BA2F1010211F8013B22
:100A800000F8013BA2F1010211F8013B00F8013B23
:100A9000A2F101022DE9F01F282A07DBB1E8F81FB7
:100AA000A0E8F81FA2F12802282AF7DADFF89CE173
:100AB0004FEA920BDEE80BF051F8043B40F8043BA0
:100AC00026E0B1E81800A0E8180021E0B1E83800FD
:100AD000A0E838001CE0B1E87800A0E8780017E052
:100AE000B1E8F800A0E8F80012E0B1E8F801A0E8E9
:100AF000F8010DE0B1E8F803A0E8F80308E0B1E878
:100B0000F807A0E8F80703E0B1E8F80FA0E8F80F4D
:100B1000BDE8F01F02F00302002A08BF00BD11F873
:100B2000013B00F8013B013A08BF00BD11F8013B51
:100B300000F8013B013A08BF00BD11F8013B00F885
:100B4000013B00BDAFF30080AFF30080AFF3008046
:100B500011F8013B00F8013BA2F1010211F8013B41
:100B600000F8013BA2F1010211F8013B00F8013B42
:100B7000A2F10102282A35DB2DE9F01FB1E8F81FA8
:100B800020F8023B4FEA134364F31F434FEA144437
:100B900065F31F444FEA154566F31F454FEA1646B5
:100BA00067F31F464FEA174768F31F474FEA184895
:100BB00069F31F484FEA19496AF31F494FEA1A4A75
:100BC0006BF31F4A4FEA1B4B6CF31F4BA0E8F80F67
:100BD0004FEA1C4C20F802CBA2F12802282ACDDAD9
:100BE000BDE8F01F042A97DB51F8043B20F8023BD4
:100BF0004FEA134320F8023BA2F10402BAE711F8CE
:100C0000013B00F8013BA2F1010211F8013B00F8A1
:100C1000013BA2F1010211F8013B00F8013BA2F1F6
:100C20000102042AFFF678AF51F8043B00F8013BBB
:100C30004FEA132320F8023B4FEA134300F8013B2D
:100C4000A2F10402EDE70000200A0008300A0008C3
:100C500008B501F095FA012000F004F8012008B56C
:100C600000F000F808B500F07BFB002A44D010F03B
:100C7000010F03463AD0013A03F8011B012A39D982
:100C8000F0B541EA01259E07ADB22CD0023A23F817
:100C9000025B032A19D95C0705EB054616BF141F32
:100CA000144643F8046BB446224604EB030E072AAD
:100CB00013D8E2086FF0070707FB02423C40032A03
:100CC000234484BF043A43F8046B012A02D9023A50
:100CD00023F8025B02B11970F0BDAEEB0207083ACF
:100CE000C7E900C6E3E7032AD5D8F0E7012AC7D150
:100CF00019707047002AFBD17047704700F008B8A0
:100D0000002070470021084601F0FEB904F0C4BC81
:100D1000704770473C4C01233C4D8C2204F1700617
:100D20002B7083B500212046FFF79FFF0323182275
:100D3000374923773046374B374FC4E9053306230D
:100D4000E38303F087FD354920463E6003F08DFBC9
:100D5000334B01A96846334E1C6002232B7001F00F
:100D600003FADDE9000103F091F9042333603368ED
:100D7000012B45DD3068800003F0A6F92A4B18608E
:100D8000336804602048A17F00F006FBA3681E487A
:100D9000DB685F6001F04AFB1B4800F0EFFA1A487D
:100DA00000F018FBA36805221A7200221F4B1A607C
:100DB00003232B7000F0C0F806F063FC1C4B0BB152
:100DC00000F030FB1B4B0BB107F07BFA1A4B0BB159
:100DD00000F074FF01F096F901F068FA05F03AF8B6
:100DE000042309482B7000F018FB05232B7000F03A
:100DF00039F806232B7000F0AFF801F015FBFCE783
:100E000033685B00B2E700BF100400249C04002498
:100E10002CA10008150D000808040024D8040024A3
:100E2000D4040024A0040024A4040024A804002462
:100E300025140008C3820008BD1C000813B5002457
:100E4000FFF760FF054B40F67A42642100940448A6
:100E500000F0DBF8204602B010BD00BF7998000812
:100E6000809F000813B50024054B4FF40062FE215B
:100E70000094044800F0E2F8204602B010BD00BF24
:100E80003D0E0008909F0008A52870B505460C4649
:100E90001AD8EFF3118600238021EFF3108372B686
:100EA00081F3118883F310881CB9FFF761FD224696
:100EB000074C084BF6B243F8354003EBC5035A60C4
:100EC00086F31188002070BD6FF01500FBE700BFAE
:100ED000150F0008E0040024A52808B50CD8094A1D
:100EE00052F830305BB102EBC00252689847064BB3
:100EF0001A68064B1A6008BD0022054BF6E71A4631
:100F0000FBE700BFE0040024D8040024D40400243C
:100F1000150F000808B5EFF3118300238022EFF3CB
:100F2000108372B682F3118883F31088362101484A
:100F3000FFF78EFE9B9F0008054B1B682BB1054AEF
:100F4000126812B91A8C01321A840020704700BF4F
:100F5000D804002404040024134B10B51A68C2B14D
:100F6000124B1B68ABB9EFF311848021EFF31083B0
:100F700072B681F3118883F31088B2F92030002B08
:100F800009DC002313840A4B1B6853B9E4B284F3D1
:100F90001188002010BD013B1BB21384002BF5D13A
:100FA000EFE701F09BF9F1E7D804002404040024E2
:100FB000CC0400242DE9FF4105468C2088461646C6
:100FC0001F4603F081F80446E0B10023A0F81E801C
:100FD0002946324603930C9B02930B9B01930A9B79
:100FE00000933B4600F034F8051E06DA204603F075
:100FF0005BF8284604B0BDE8F0812046E56800F0C3
:1010000073F9F6E76FF00B05F3E71FB5069C009246
:101010000A46CDE9013400231946FFF7CBFF04B09F
:1010200010BD1FB5079C0294069CCDE90034134601
:101030000A460221FFF7BEFF04B010BD13B5049CA1
:10104000CDE9003413460022FFF7EBFF02B010BDDC
:101050002DE9F347867F88460546914631461F466F
:10106000DDF828A000F098F9041E3ADB284606F0C7
:10107000030600F0D4F9041E0CDB87B15246394652
:10108000284601F099F9041E05DB284600F076F9A0
:10109000041E13DA57B1284600F0A2F921E03246C7
:1010A0005146284601F0C0F8041EEEDAAB6B002B67
:1010B000F1D03146284601F02BF9ECE70B9B49466D
:1010C0000A4A2846009600F013F8041EE2DB0C9A48
:1010D0004146284600F09CF8041EDBDB284600F061
:1010E00079F9204602B0BDE8F08700BF0D13000873
:1010F0002DE9F74F04460E4601929946EFF311870A
:1011000000238022EFF3108372B682F3118883F3F9
:101110001088DFF8F4A0DFF8F480DAF8005000203F
:10112000D8F800300135364A116888420DDB106866
:10113000C00002F0C9FF324A0546002842D1FFB282
:1011400087F311886FF00B0036E0012D1168B8BFEE
:1011500001250139294053F821B0BBF1000F2ED1F0
:1011600043F82140FFB2E560CAF8005087F31188C8
:10117000019BF6B29DF83020594603202674667410
:10118000C4E90539E38B62F3010304F1440223F05F
:101190006003E38300F082F9204684F81CB001F07C
:1011A00045F9FFF7C9FE1749204603F05EF904230D
:1011B0002377FFF7D1FE584603B0BDE8F08F013525
:1011C0000130B1E711684FF0000C0D4B4900116080
:1011D0001A68D8F8000002EBD272BCEB620F04DB95
:1011E00002F062FFC8F8005097E750F82C000CF1AD
:1011F000010C1A68C168013A0A4045F82200E7E785
:10120000A0040024AC040024A8040024A4040024A6
:10121000344B2DE9F74F002914BF884698460746FE
:101220000024154641461822703003F02FFB40463B
:1012300087F8884003F022FB461C4DBB2C46023445
:10124000384606EB840101F075F806464FEA84093A
:10125000002844D000EB090AA9F10809B346043D6F
:10126000C0F800A0404603F009FB0446B1444146E3
:101270000134504603F0E6FA5444CB451BD100201C
:101280004AF8040CBB68DB685E6003B0BDE8F08F11
:1012900040F2011955F824000028D0D0013603F09F
:1012A000EDFA7B6B06449E4216D201344C45F1D1D7
:1012B0006FF00600E9E74BF8044F55F8041F0846A5
:1012C000019103F0DBFA80460199204608F10108FC
:1012D00003F0B8FA4444D0E76FF05A00D5E76FF056
:1012E0000B00D2E778A1000810B5EFF311840023BA
:1012F0008022EFF3108372B682F3118883F3108893
:1013000001F03CF8E4B284F3118810BD38B5134BFA
:101310001C68E38B03F00303022B02D0204600F08D
:10132000A3FBA368012040F20111DB685A6852F860
:1013300020304BB9E38BA56903F00303022B08D1DE
:101340001146A847FFF78EFC01308842EFD10120FB
:10135000F8E70146284603F0A1F8F8E7D80400248E
:101360000446002208B5E4B2034B2146186800F099
:10137000A3FB204600F07EFFD804002410B51821FE
:10138000044600F0D7FF20B1A368DB6803600020AB
:1013900010BD6FF00B00FBE770B506464FF48E7082
:1013A00002F092FE044690B100F0ABFB051E04DA99
:1013B000204602F079FE284670BD04F12400B46096
:1013C00006F090F92046002503F073F9F3E76FF07B
:1013D0000B05F0E7D0E902321A6001225A72704719
:1013E00038B58468054634B1637A012B04D9013BD2
:1013F00063720023AB6038BD204600F093FB2046AB
:1014000000F030F904F1240006F070F9204603F0F2
:101410006FF9204602F048FEEBE700F090BB00F0C9
:101420008EBBFFEC0023044A044942F83310013319
:10143000A62BFAD1FFF74ABAE0040024150F0008E2
:1014400038B5044618B3C068B0B1EFF31182002379
:101450008025EFF3108372B685F3118883F310882B
:101460000C4B00251B68013B03400B48006840F80B
:101470002350D3B283F31188A36B13B1204600F03D
:1014800047FF2046FFF7ACFF204602F00DFE00208C
:1014900038BD00BFA0040024A4040024F8B51746FA
:1014A000194B06460C461D68FFF746FD0FB16B6CE5
:1014B0003B60D4B1EFF3118300228021EFF310825F
:1014C00072B681F3118882F31088022E11D0032E98
:1014D00014D0012E14D16A6C21680A4300246A6476
:1014E000DBB283F3118800F011F8FFF735FD2046D9
:1014F000F8BD21686A6C22EA0102EFE72268EDE795
:101500006FF01504ECE700BFD8040024174B37B583
:101510001D68FFF711FD6C6C284600F0F5FCE443F4
:101520000440019424B9FFF717FD204603B030BDF5
:1015300001A800F06FF8431C044610D0014601A832
:1015400002F0F5FF2146284600F012F8044630B1BB
:10155000011D284600F09AF8204600F02DF8019B66
:10156000002BE5D1FFF7F8FC0120DFE7D8040024C9
:1015700038B58368EFF3118500228020EFF31082E5
:1015800072B680F3118882F3108800209C693CB108
:1015900022798A4209D103F1180148B102F04AFFC9
:1015A000EDB285F31188204638BD20462468EEE769
:1015B000084602F035FFF3E710B5037B83B9EFF37C
:1015C00011848022EFF3108372B682F3118883F3C3
:1015D00010880E4902F004FFE4B284F3118810BDB4
:1015E000022B0CD1EFF3118400238022EFF3108340
:1015F00072B682F3118883F310880549EAE7012B5C
:10160000EDD1BDE8104002F04FBD00BF180A002424
:10161000100A002438B5054601242146284602F068
:1016200096FF20B90134202CF7D14FF0FF3420462B
:1016300038BD38B5044600F14C05284602F0F0FEEE
:1016400050B904F15405284602F0EAFE38B94FF0CB
:10165000FF32C4E9112038BD00F0B0FCEDE700F026
:10166000ADFCF0E738B5044600F11005284602F05D
:10167000D7FE28B91834204602F0D2FE18B938BD7A
:1016800000F07AFBF2E7FFF797FFF4E72DE9F0416E
:101690000D460978044629B3443002F058FF01286A
:1016A00007467ED1EFF3118600238022EFF31083EB
:1016B00072B682F3118883F31088237FF6B2062B6B
:1016C00012D1297804F1480002F041FF60B12B6883
:1016D0002046E3656B6823660023A36400F04EFE9A
:1016E00086F311880026C0E086F31188A468297863
:1016F000EFF3118200238020EFF3108372B680F3A2
:10170000118883F31088A36913B11879884208D12E
:10171000D2B282F3118833B12A685A606A689A603B
:10172000E0E71B68F0E7564B1B68FBB1554802F039
:1017300077FE20B9544802F073FE0028D2D02B68FF
:1017400043606B688360EFF3118500238022EFF321
:10175000108372B682F3118883F3108804F11801A4
:10176000EDB202F03DFE85F31188BBE7EFF3118681
:1017700000238022EFF3108372B682F3118883F383
:1017800010884048F6B202F04BFE86F3118800281C
:10179000D5D1102002F090FC0028A3D001230373C0
:1017A000CDE7FFF7C9FB2978A06800F0C9FB064622
:1017B00058B343684BB300F0D5FB002858D073688A
:1017C0004360B2688260F3689B0604D429780123E1
:1017D0008B40134383602B68C3606B680361EFF336
:1017E000118600238022EFF3108372B682F31188F2
:1017F00083F3108804F14C01F6B202F0F1FD2349A5
:10180000204600F04FFE86F311880026FFF7A4FB68
:10181000EFF3118800238022EFF3108372B682F376
:10182000118883F31088237F062B08D12B6820466C
:10183000E3656B6823660023A36400F09FFD5FFAF5
:1018400088F888F31188002F15D1237F052B03D149
:101850000421204600F014FA237F072B05D12B78B2
:10186000082B02D1204600F0C8F93046BDE8F081CF
:101870006FF00B06CAE7F8DA6FF01506F5E700BF60
:1018800004040024180A0024100A0024AB180008DD
:1018900010B50C4600F06AF920B12146BDE81040B1
:1018A000FFF7F4BE6FF0020010BD2DE9F04F87B0D6
:1018B000044602F08BFD03684FF0800A04F15409DE
:1018C0000193B4F92230029304F14C030593EFF332
:1018D0001183EFF3108772B68AF3118887F31088AB
:1018E000B4F81E8018F400725FFA83F804920AD0EC
:1018F00088F3118802F06AFD019B0360029B6384F8
:1019000007B0BDE8F08F059802F08AFD0646002872
:10191000EED0E28B494642F40072E28302F060FDB1
:10192000D4F844B0B5684BEA0505656488F31188BE
:10193000736806F10C01049A307B9847EFF3118825
:10194000039BEFF3108372B68AF3118883F3108838
:1019500003934946E38B30465FFA88F823F400731B
:10196000E383636C5D4083EA0B031D4085EA0B054E
:10197000656402F03FFD88F31188FFF7C7FD30462C
:1019800000F01CFBA3E77047054B10B51C68FFF780
:10199000D3FA204600F010F9BDE81040FFF7DCBA9A
:1019A000D804002408B5024B01201B68FFF75AF940
:1019B000D804002408B58068203002F0C8FD002853
:1019C000D4BF0020012008BD0023094A10B512F839
:1019D000334002EBC301844204D14878C04300F095
:1019E000010010BD01330B2BF1D10120F9E700BF3D
:1019F00084A1000838B580684AB10023194A12F85A
:101A0000335002EBC304A94214D16468B4B9EFF3B4
:101A1000118400238022EFF3108372B682F31188C1
:101A200083F310882030E4B202F081FD84F3118842
:101A3000002414E001330B2BE1D1E8E7EFF311852B
:101A400000238022EFF3108372B682F3118883F3B0
:101A500010882030EDB202F05EFD85F3118820463B
:101A600038BD00BF84A100082DE9F043866800243A
:101A7000104D4FF002092036A04685B0304602F0E6
:101A800062FD6B6873B12F7801A90022CDF80C902C
:101A90003846CDE90138012300F084F93946304653
:101AA00002F039FD013408350B2CEAD1002005B0D5
:101AB000BDE8F08384A1000810B5C38B04461B0564
:101AC00015D43AB9806828B1437A012B02D12C3061
:101AD00002F058FD204600F00BF82046FFF780FC8E
:101AE0002046FFF7A6FDE38B43F40063E38310BDBC
:101AF00010B5044600F020F82046BDE8104000F084
:101B0000A6B838B50546382002F0DEFA044630B1F2
:101B10000122002102F0CDFC0020EC6038BD6FF006
:101B20000B00FBE710B5C468204600F078F82046AB
:101B3000BDE8104002F0B8BA243000F06DBA0023BE
:101B40000246012110B50446184606F099FA002312
:101B500022460621012006F093FA002322460621A0
:101B6000022006F08DFA002010BDFFEC0346EFF3D3
:101B7000118100228020EFF3108272B680F3118869
:101B800082F310880A4A106860B1002B0EDB094A04
:101B90001268013A1A4050F8220018B1C2689A42FD
:101BA00018BF0020CBB283F3118870470020F9E7FB
:101BB000A4040024A004002438B50446EFF31185E2
:101BC00000238022EFF3108372B682F3118883F32F
:101BD0001088037F043B032B0BD800F065FA042325
:101BE00007212046638400F04BFAEDB285F311889B
:101BF00038BD072100F0EAFAF7E710B5EFF31184DA
:101C000000238022EFF3108372B682F3118883F3EE
:101C1000108800F0B3FBE4B284F3118810BD30B13A
:101C200003881B0401D401230380002070476FF058
:101C30001500704710B5FFF7F2FF041E05DA644285
:101C400002F0C4FB04604FF0FF34204610BDEFF3F8
:101C5000118200238021EFF3108372B681F3118883
:101C600083F31088037F052B06D1016C0B880133A9
:101C70001BB20B8000230364D3B283F31188704737
:101C800038B5EFF3118400228025EFF3108272B68D
:101C900085F3118882F31088027F052A09D1056C2B
:101CA0002A88013212B22A8000224184026400F0A4
:101CB00065FBE4B284F3118838BDFFECF8B500246D
:101CC000284B294E6020C3E90044284BC3E9004457
:101CD000274BC3E90044274BC6E90044C3E900444D
:101CE00002F0EAF9054648B100F160072C75284674
:101CF0001835314602F074FBAF42F7D1602002F094
:101D0000DBF9044658B100F160050227174E27752C
:101D100020461834314602F063FBAC42F7D1402034
:101D200002F0CAF9044658B100F140050027104EF0
:101D3000277320461034314602F052FBA542F7D1FA
:101D4000402002F0B9F9044658B100F140050227DD
:101D5000084E277320461034314602F041FBAC4256
:101D6000F7D1F8BD300A0024280A0024200A0024F4
:101D7000180A0024100A002410B5EFF31184002380
:101D80008022EFF3108372B682F3118883F31088F8
:101D90000349E4B202F024FB84F3118810BD00BFB4
:101DA000300A00242DE9F04F1746554A1F2885B008
:101DB000D2F800A005460C46DAF8089004D96FF076
:101DC000150005B0BDE8F08FD9B92946484600F0A6
:101DD000B7F80646FFB994B12768012F32D13A46C9
:101DE00029465046FFF706FE07468FBB3EB13046F8
:101DF00009F1100102F0FEFA3046FFF7BDFF0020A6
:101E0000DFE7002BE1D10B68012BDED0FFF7DCFD13
:101E10000028DAD1D3E729465046FFF7CBFD30B191
:101E200000230122C7E900230223BB60D3E72EB1C0
:101E300073683B60B3687B60F368F6E7C7E90066E8
:101E4000BE60C8E7002229465046FFF7D3FDCCE725
:101E5000E6B9EFF3118B4FF0800A0023EFF3108304
:101E600072B68AF3118883F3108826485FFA8BFBD9
:101E700002F0D6FA06468BF31188DFF888B05EB11F
:101E800009F110013046357402F0AAFA77606368F0
:101E9000B360A368F360B2E7502002F00DF9064684
:101EA000C0B1EFF31183EFF3108872B68AF3118893
:101EB00088F3108800F15002304659461436CDE9B7
:101EC000022302F08DFA029A039B9642F4D1DBB210
:101ED00083F31188EFF31183019A0293EFF31082D9
:101EE00072B68AF3118882F310885846019202F084
:101EF00097FA029B0646DBB283F31188BFE700BF67
:101F0000D8040024300A0024002337B582680193E6
:101F1000EFF311858021EFF3108372B681F31188FE
:101F200083F3108894692CB9EDB285F31188019878
:101F300003B030BD217901A802F0EDFA2468F2E780
:101F400038B50D46044640B1FEF7F6FF246914B1DA
:101F5000237CAB4203D1FEF7FFFF204638BD246847
:101F6000F5E7FFEC124B10B51B6843B1114802F0C6
:101F700057FAE0B91048BDE8104002F051BAEFF34B
:101F8000118400238022EFF3108372B682F311884C
:101F900083F310880748E4B202F042FA84F3118810
:101FA00028B9182002F088F808B10123037510BD84
:101FB00004040024280A0024200A002410B5037D0C
:101FC00083B9EFF311848022EFF3108372B682F3AA
:101FD000118883F310880E4902F002FAE4B284F308
:101FE000118810BD022B0CD1EFF311840023802245
:101FF000EFF3108372B682F3118883F310880549DA
:10200000EAE7012BEDD1BDE8104002F04DB800BF6A
:10201000280A0024200A002438B50446EFF311856D
:1020200000238022EFF3108372B682F3118883F3CA
:102030001088F0B14368E3B1104B00201B68DBB19E
:10204000A3420FD123681BB19A68A1680A449A6021
:1020500058B10A4902F0EEF900206060EDB285F354
:10206000118838BD18461B68E9E7044802F0D8F922
:10207000F2E76FF01500F1E71B68FFDE380A002475
:1020800038B50C46074B054653F8311003EBC40333
:102090001B79DB0703D500F015F82C7738BD02F06B
:1020A000D9F9FAE738A10008054B027F10B553F8BB
:1020B0003210044602F0E4F90023237710BD00BF7C
:1020C00038A1000810B50B68027C5BB11C7C9442FF
:1020D00006D25A68C0E900328AB95860086007E041
:1020E0001B68F2E74A68036022B94360C1E9000057
:1020F000012010BD4260106048600020F9E71060C8
:102100005860FAE77047FFEC37B5124D2C682CB1D8
:10211000114802F025FA012003B030BD0F4802F04B
:102120001FFA40F2011369464FF60C70ADF800300B
:102130008DF80240019503F053FE011E04DA494276
:10214000074802F00DFAE6E7064802F009FA2046D1
:10215000E2E700BF400A0024B39F0008D69F0008B2
:1021600001A0000840A00008044B1B680360C3F1F5
:10217000105303F500230B60704700BF649F0008F5
:1021800008B504F0BDFB04F0BBFB04F0B9FB0D4B3C
:10219000186818B90C4B1B681B6873B9002007F04E
:1021A00055FCEFF3118300238022EFF3108372B606
:1021B00082F3118883F31088FEE7BDE8084007F03A
:1021C00045BC00BF04040024D80400242DE9F041DC
:1021D00006460F46114DD5F8008006F0A9F839469D
:1021E00004463046FFF74CFF0D4B1B681BB106F051
:1021F000B3F80443E4B23CB10A4B1A6832B1C8F8F0
:102200006C202A68D26E1A60BDE8F0812B6808F154
:102210006C00D96EBDE8F04100F0A7B8D8040024E6
:10222000CC0400240404002438B5836B0C46054616
:1022300011469BB9204601F03FFFA863A86BB0B1DF
:102240000119E86321F00701091A696300F0CCF86D
:10225000EB8B002043F48053EB8338BD436BA342E8
:10226000ECD000F055F8AB6B002BE7D1E2E74FF074
:10227000FF30F2E7094C08B52368EFF31183002320
:102280008022EFF3108372B682F3118883F31088F3
:1022900006F0BCF92368D86E00F002F8D8040024D8
:1022A0000146012000B500DF5DF804FB08B5084ACF
:1022B000C0230849013B42F8041BFBD1064B0BB17C
:1022C000AFF3008000F038FBBDE8084001F078BCB7
:1022D00000010024EFBEADDE0000000038B50A4C5E
:1022E000256806F039F830B1084B1A6822B1EA6661
:1022F0002268D26E1A6038BD236805F16C00D96E71
:10230000BDE8384000F031B8D804002404040024AB
:1023100010B50446806B20B1E38BDB0401D501F0DE
:10232000C3FEE38B23F48053E3830023C4E90E331D
:10233000636310BD38B5CD1D836B044625F00705DA
:102340007BB1436BAB420ED9C36B2A4600211846C2
:10235000FEF78BFCE26B03462A44E263626B521B7E
:102360006263184638BD0023FBE703460A46022095
:10237000194600B500DF5DF804FBFFEC70B50546BB
:102380000B4C2668FFF790FE284605F0ADFF30B1F4
:10239000084B1A6822B1F2662268D26E1A6070BDCC
:1023A000236806F16C00D96EBDE87040FFF7DDBF11
:1023B000D80400240404002470B5836B06460D463F
:1023C000144623B1C18B01F00301FFF7A1FF2C4498
:1023D000284624F00704611BC6E90E55716300F01E
:1023E00003F8002070BDFFECC21D80B522F007028B
:1023F00082B0134600AF79B9391DB94228BF3946BA
:1024000021F00701091A21F003011144054A8B420A
:1024100004D10837BD4680BD0144F1E743F8042BE1
:10242000F5E700BFEFBEADDE7047FFEC38B5002525
:10243000C168044645668566C56661B9184B18686B
:1024400040F2EE23A0F2EE206363C4E90E00BDE883
:102450003840FFF7C9BF436BD422C06B2946D43B39
:102460001844E066FEF701FCE36B616BE26E0B441F
:1024700013606369E26E23F00103C2F884304FF009
:102480008072E36EC3F888206FF01602E36E9A62E2
:10249000F022E36EC3F8CC50E36E5A6038BD00BF43
:1024A000649F000810B5426E04460B46FAB91B4AF9
:1024B000126882421CD11A4C216811B9BDE8104043
:1024C0001847A1F1D400C2E91931D4222060FEF7E7
:1024D000B7FA236803F1D4021A60124A2368C3F8DA
:1024E000842080225A604FF08072C3F8882010BD8B
:1024F0004166D422C16E8166A1F1D400E066FEF788
:102500009FFAE36E03F1D4021A60064AE36EC3F841
:1025100084208022E36E5A60E36EE4E7D80400244E
:10252000040400242925000838B50D4B1C68F0234D
:10253000A56E83F3118862B6636E20469847EFF369
:10254000118300238022EFF3108372B682F3118887
:1025500083F31088002328466366FFF7A1FE00BFBF
:10256000D804002410B5846E01F4D873A0F850107C
:10257000226822F4D87213432360826E936861F359
:102580000003936010BD10B5EFF311840023802287
:10259000EFF3108372B682F3118883F31088FFF78C
:1025A000E1FFE4B284F3118810BDFFECF0B5C26B1B
:1025B000EFF3118000238021EFF3108372B681F3D3
:1025C000118883F31088936E1D6825F0010105F0D2
:1025D00001041960D66D576E730803EB4703B3FB14
:1025E000F6F3642B33D9013325F400415B0821F065
:1025F0000101956E2960956EEB60204B0B4092F8BF
:10260000561001292DD143F4C06392F85750092D7B
:1026100002D0082D2AD149B343F48053916EC0B241
:102620000B602343966E92F858107568494225F462
:10263000405501F4005129437160956EA96821F459
:102640004071A960926E136080F31188F0BDC3F3EE
:10265000420523F00F0341F400411B041B0C2B43E4
:10266000C7E7022908BF43F48063CEE7B2F85610EB
:10267000B1F5E06F08BF43F08053CFE7FEE9FFEF0D
:10268000C36B9A6E506AB3F8522040EA0242C0B25D
:102690000A600022A3F85220704710B5C06BEFF318
:1026A000118400238022EFF3108372B682F3118825
:1026B00083F31088B0F8503039B143F02001E4B210
:1026C000FFF761FF84F3118810BD23F4907121F0AE
:1026D0000101F4E7C36B9B6ED869C0F340107047EB
:1026E000C36B9B6E9962704710B5C06BEFF311849A
:1026F00000238022EFF3108372B682F3118883F3F4
:102700001088B0F8503041B143EA020189B2E4B216
:10271000FFF739FF84F3118810BD23F08001F5E73E
:10272000C36B9B6ED869C0F3C010704738B50346C1
:1027300010469B685D6940F201139942EC6B05D02D
:10274000B1F5817F1BD06FF0180038BD9AB394F8B3
:10275000563093B15A1E534253415A024FF480737C
:1027600094F858101A4342EA811242F03002826013
:10277000E16D02F09DF80020E7E71A46F0E7D2B1DC
:10278000926802F03003302B15D112F4807304D01C
:1027900012F4007F0CBF0223012384F856308368B3
:1027A000C3F3801384F8583002F09EF8E0652846A1
:1027B000FFF7FCFEDFE76FF01500C6E710B5C46B4E
:1027C00094F86000FEF7D4F8002294F860001146F7
:1027D000BDE81040FEF758BB38B5C56B06492A4620
:1027E00095F86000FEF750FB044618B995F86000B4
:1027F000FEF7D2F8204638BDFD27000810B5144674
:10280000926ED3699BB29806A4F8523013D5B4F8EF
:10281000501089060FD5204604F02BF8B4F852303A
:102820001A0606D5B4F850301B0602D5204603F030
:10283000EAFF002010BD13F00E0FEFD00E2313623D
:10284000ECE7FFEC38B5C46B00210546A36E1960B8
:10285000C36B9A6E1C4B9A4203D110221B48FDF7A2
:1028600047FFE06E01F00EFB206F01F00BFBA16E45
:1028700094F8583028464A685B4222F47D5203F4AB
:10288000005313434B60A26E114B11680B40136051
:10289000A26E94F85510936823F4E06323F00103CB
:1028A00043EA41639360FFF781FEA26E0020136844
:1028B00043F0005343F00D0313600123A4F85000CC
:1028C00084F8543038BD00BF00100140F044025875
:1028D00003BEFF3370B50021C46B054684F8541065
:1028E000EFF3118680220B46EFF3108372B682F36A
:1028F000118883F310882046F6B2FFF733FE86F383
:102900001188EB6B9A6E0A4B9A4204D10A46094829
:102910001021FDF7EDFEA26E136823F00D03136086
:10292000E06E01F097FB206FBDE8704001F092BBB4
:1029300000100140F04402587FB50B49684601F091
:1029400081FF0023094D1C4655F8041B39B15E1C5C
:10295000303368468DF8093003F070FD334601349A
:10296000082CF1D104B070BD7BA00008DCA10008E8
:10297000704738B50A460169044629B14B690361BD
:1029800003B9436100234B61637E207EC3F3C0051E
:1029900020B9E068007C60F3C3036376CB6820460F
:1029A0004A819847637E65F3C303637638BD37B5C4
:1029B0000446C0680A4680B10368B4F85E1000910E
:1029C00021469D6804F11D03A847002803DA237CF3
:1029D00043F00103237403B030BD6FF00400F6E749
:1029E000F0B5047E3CB313466401144FE5592E0440
:1029F00015D4AE03124E48BF45F080652E403343D8
:102A000043EA814301F04F0143F0805343F4004314
:102A1000E351437EC28023F04F0319434176027E87
:102A20000123084900201032D1F81C489340234369
:102A3000C1F81C38F0BD21462346D5E7000B0840FD
:102A400000F8F3FF00000840F0B590F818C0144EED
:102A50004FEA4C17BC59250417D4A303114D42EA81
:102A6000814301F04F0148BF44F0806425402B436F
:102A700043EA8C5343F0805343F40043BB51437EFD
:102A8000C28023F04F0319434176007E0123064A9A
:102A900083400020D2F81C180B43C2F81C38F0BD4C
:102AA0000009084000F833FC00000840437E8A8893
:102AB000DB06C97801F0030101D5FFF7C5BFFFF7B9
:102AC0008FBFFFEC417E027ECB064FEA42124CBF25
:102AD000084B094B890713441A6822F4001248BFB7
:102AE00042F080521A60437E23F0080343760020B0
:102AF000704700BF00090840000B084001F07F0349
:102B0000F0B5EFF3118400218025EFF3108172B648
:102B100085F3118881F310888718FD7C93B1062B0B
:102B20000ED801219940294039B18E074FF0010399
:102B30001AD49C460133072B06D1E4B284F31188E2
:102B4000002010E02946EFE70CFA03F63142F1D0FD
:102B500025EA0605E4B2FD7484F311881C214B4379
:102B600022B160331844F0BD0226F1E703F59273F9
:102B7000F8E710B5C0B1B9B1EFF31182002380249A
:102B8000EFF3108372B684F3118883F310884B7EC1
:102B9000097EC3F30013184401238B40C17C0B430F
:102BA000C374D3B283F3118810BDFFEC024BD3F88A
:102BB0000808C0F30D20704700000840037C61F353
:102BC0004103037400207047EFF31182002380203B
:102BD000EFF3108372B680F3118883F310880848EE
:102BE000D0F8043841B123F00203C0F80438D3B25E
:102BF00083F311880020704743F00203F5E700BF1C
:102C000000000840084601F04FBA10B5182001F046
:102C100053FA044618B118220021FEF726F8204680
:102C200010BDFFEC70B5EFF3118600238022EFF3A7
:102C3000108372B682F3118883F31088037CDA065E
:102C400011D50B4CD4F80838DB070CD5D4F8045850
:102C5000052045F0010325F00105C4F8043801F012
:102C6000E7F8C4F80458F6B286F31188002070BD66
:102C70000000084070B54B7E05460C465B070CD43F
:102C800022695AB9237E1A485B01195841F0006144
:102C90001950637E62F38203637670BDD18819B9DF
:102CA0002046FFF766FEEBE7E388124E5A1E1144FA
:102CB000227EB1FBF3F152014B43905900F060408A
:102CC000034343EAC1430A499351237E5B015A58A7
:102CD00042F004425A50637E43F004036376237E3D
:102CE000002BDAD16B7C062262F307136B74D4E7F6
:102CF000000B0840100B08401023054A1361054BD8
:102D00001169C90601D5013BFAD10320FDF705BDC4
:102D100000000840400D030040F02000054A064B2B
:102D200010611169890601D5013BFAD10320FDF735
:102D3000F4BC00BF00000840400D030038B5036933
:102D400004460D4643B1437EDB0606D5007E800176
:102D5000FFF7E2FF23691BB938BDFFF7CDFFF9E7A5
:102D600029462046FFF705FEF4E710B5EFF311847E
:102D700000238022EFF3108372B682F3118883F36D
:102D800010886FF06D01E4B2FFF7D8FF84F311886B
:102D9000002010BD70B5437E0446DE063CD5037EA0
:102DA0003D495B015B581D0434D5EFF311850023C9
:102DB0008022EFF3108372B682F3118883F31088B8
:102DC000027E5201535823F4004343F09043535082
:102DD000324A037E590102EB431318688007FCD581
:102DE0008B58EDB243F002038B50207E8001FFF739
:102DF00093FF207E2A490122D1F81C3882402046C8
:102E000023EA0203C1F81C386FF06D01FFF796FF4B
:102E100085F31188002070BDEFF311860023802216
:102E2000EFF3108372B682F3118883F310881C4D80
:102E3000D5F8043843F40073C5F80438D5F80438DD
:102E40001B07FBD5227E0A201649F6B252015358C1
:102E500023F4004343F090435350FDF75EFC237E80
:102E6000114A02215B01204699500122D5F804380D
:102E700043F48063C5F80438217ED5F81C3810313E
:102E80008A406FF06D0123EA0203C5F81C38FFF792
:102E900055FF86F31188BDE700090840080908407E
:102EA00000000840000B0840080B0840002882B0D2
:102EB00006DD0023034904330A6898420192FADCD4
:102EC00002B070470010084030B503460B4C1A1D85
:102ED0001B1A994200DC30BD2368C3F3072502F8B2
:102EE000043C02F8035CC3F30745C3F3076302F82D
:102EF000025C02F8013C1346E9E700BF00100840FD
:102F0000F0B5057E1F4F6D01EB5903F0004392B3FE
:102F1000C688541E3444B4FBF6F4467E134306F0D0
:102F2000030643EAC443012E174E08BF43EA447325
:102F3000EB51457E047E05F003056401012DA35984
:102F400008D1124DD5F80858ED0554BF43F0805311
:102F500043F0005323F08043033243F004439210C4
:102F6000A351037E00201B0303F1804303F50123DB
:102F7000824202DCF0BD0124CFE751F8204001304D
:102F80001C60F5E7100908400009084000000840EF
:102F9000F8B50D6907460C465DB90B7E30495B01FB
:102FA0005A5842F000625A50637E65F3820363769A
:102FB000F8BDEB881BB94B7E43F040034B762A8962
:102FC000EB889A4208D3617E480605D4204600214A
:102FD000BDE8F840FFF7CDBC9B1A627E002B22F0C3
:102FE0004002627602DDE6889E4212DD1E46217EA8
:102FF0001C4B4A01D358F21C9BB2B3EBA20F11DA5F
:10300000194A0123D2F834088B400343C2F83438FC
:10301000CEE7ECD12A79D207E8D5627E42F04002B1
:103020006276E3E72B893246296820461944FFF788
:1030300067FF637E43F004036376237E23B97B7CC2
:10304000052262F307137B742B891E44EB88B6B20A
:10305000B3422E81ACD8637E5906A9D4B6E700BF2F
:10306000000908401809084000000840184A38B50F
:103070000346C0688A60EFF3118400228025EFF3D5
:10308000108272B685F3118882F310885A7E12F08E
:10309000080219D11D694A614DB95A7EC3E904116C
:1030A000510708D50020E4B284F3118838BD5A696D
:1030B00051615961F6E71946D30602D5FFF768FF5B
:1030C000F0E7FFF7D7FDEDE76FF00F00EBE700BF8C
:1030D000000089FF054B064AC3F8102BD3F8002BDC
:1030E00042F00442C3F8002B704700BF00000840C4
:1030F0001800086010B504466030FFF701FF042295
:10310000637C62F307136374BDE81040FFF7E2BF0E
:1031100000221146FFF7EEBF344A00202DE9F047A8
:10312000D2F80438324C23F00103C2F80438FFF718
:10313000F3FDE06818B103682146DB689847FE2379
:103140002C4E2D4F00254FF0FF0A4FF01C09E37461
:10315000237509FB05483046C7F800A06FF06D01E4
:10316000C7F800A20135FFF7E9FD98F8793006F1BC
:10317000C4006FF06D0123F04C0320371C3688F833
:103180007930FFF7DBFD98F83D31072D23F04C0334
:1031900088F83D31DDD1154B4FF0FF320021154845
:1031A000C3F818284FF00112C3F81C280B22C3F8EB
:1031B0001428C3F81028D3F8002822F4FE62C3F8BC
:1031C00000284022238A23F4706323F0040323821F
:1031D00002232372FFF738FC402200210748FFF743
:1031E000FFFBBDE8F047FFF775BF00BF00000840D8
:1031F000C80D0024280E002408090840EC0E002405
:1032000038B5124D0446D5F8043843F40073C5F8B8
:103210000438D5F804381B07FBD5227E0A200C4958
:103220005201535843F0804343F400135350FDF7C9
:1032300074FAD5F80438002043F48063C5F80438E4
:10324000637E43F00803637638BD00BF000008408A
:10325000000B0840427E0346D20601D4FFF7D0BFE0
:10326000027E06485201115841F40011115000200D
:103270005A7E42F008025A76704700BF00090840A3
:1032800010B5EFF3118400238022EFF3108372B6A0
:1032900082F3118883F3108829B1FFF713FCE4B29D
:1032A00084F3118810BDFFF7D5FFF8E7F8B5437C2C
:1032B000044603F0F003202B40F0AC8000F592753B
:1032C0006FF046012846FFF739FD6FF0460104F123
:1032D0006000FFF733FD94F83D31A77D23F008032C
:1032E000B4F81760E07D84F83D3194F87930B4F893
:1032F000191023F00803B4F81B2084F87930238ACE
:1033000023F001031B051B0D43F440532382637D0F
:1033100013F0600F05D004F115012046FFF747FBBD
:103320005BE00C2F26D80FF2080C5CF827F000BFEA
:10333000653300081D340008753300087534000833
:103340007533000813350008613500086135000841
:103350006935000885350008173300081733000861
:10336000DB330008207C470704D5022A02D11F0660
:1033700000D526B1237C43F0010323742DE003F034
:103380001F03012B47D0022B0CD0002BF2D10029B8
:10339000F0D1C0F30013C0F34000A17740EA43002E
:1033A000607715E001F07F03062BE3D8C3EBC3037E
:1033B0000A064FF002024FEA83034CBF603303F565
:1033C000927323445B7EC3F3C00363770023A37728
:1033D00004F11D012046FFF78DFE237CDB0716D587
:1033E00094F87830284676495B015A5842F4001226
:1033F0005A5094F8793043F0080384F87930FFF795
:10340000FFFE237C43F001032374FFF763FE0023D8
:10341000A4F85E30F8BD6677A677D9E7207C470729
:10342000A8D5002AA6D103F01F03022B17D1002E26
:103430007FF471AF01F07F0006283FF66CAFC0EB60
:10344000C0000E064FEA80004CBF603000F592705D
:103450002044FFF737FB2046FFF75AFEBDE7002B5D
:103460007FF459AF012E7FF456AF034662F3041385
:103470002374F0E7277C78077FF57CAF002A7FF480
:1034800079AF03F01F03022B12D1002E3DD101F0C2
:103490007F00062839D8C0EBC0000A064FEA80003A
:1034A0004CBF603000F592702044FFF7D3FED2E7A6
:1034B0005BBB012E03D147F010072774CBE7022E28
:1034C00023D1CBB20BBB090AA37C0139042914D840
:1034D000DFE801F0030B0D0F1100012262F303037B
:1034E000A374237C43F02003C2E70222F6E7032201
:1034F000F4E70422F2E70522F0E723F00F03A374B8
:10350000237C43F001032374EBE73B077FF532AFE5
:1035100001E7DF067FF42EAF0A437FF42BAF7F2E47
:103520003FF628AF637C03F00F03022B3FF422AF7A
:10353000244AD2F8003823F4FE6343EA0013C2F8A9
:10354000003858B90246930043EA0223228A22F443
:10355000706222F00402134323827CE70122F2E727
:10356000DE067FF407AFD6E6207C40077FF502AF8A
:10357000DB067FF4FFAE0E437FF4FCAE012A7FF43E
:10358000F9AEC8E6207C47077FF5F4AED8067FF495
:10359000F1AE0A437FF4EEAE04F115012046FFF7C9
:1035A00006FA00287FF419AF228AF6B2064B1340C0
:1035B0001EB143F4027323820FE743F48073FAE7EA
:1035C0000009084000000840F7F0FFFF2DE9F04F28
:1035D00085B0DFF8B092D9F81440D9F8181041F44A
:1035E000403242F4407222400C4022F0E96222F460
:1035F000E02222F47D7222F00102C9F8142000F0CA
:103600009D80270300F19E80660313D5DFF8749236
:10361000D9F81838D9F81C2813409BB20193002B15
:1036200040F03A81D9F81838FF21954A9BB2002B17
:1036300040F02081002C12DA924A0121924DD2F8FA
:103640000438284623F00103C2F80438FDF761FB73
:10365000E86820B103685B690BB1294698472105EA
:103660000AD58949C86818B103681B6903B198472E
:1036700000218548FDF74DFBE20659D5814B1D6AB7
:1036800005F00F09B9F1060F52D805F4F012B2F5A2
:10369000002F00F0A781B2F5402F00F0B181B2F504
:1036A000802F45D1C5F30A15002D41D0DFF8D88110
:1036B0001C2606FB0986D6F83471002F40F07D8168
:1036C00096F83CA1BAF1000F40F07381D6F8307142
:1036D0007B7C03F0F003102B40F06B81402DAB4658
:1036E00007F11D00A8BF4FF0400B1FFA8BF10191AD
:1036F000FFF7EAFBA5EB0B00FFF7D8FB96F83D318F
:10370000022238466AF3820386F83D317B7C62F3FD
:1037100007137B740199A7F85E10FFF7C7FD1C2300
:1037200003FB098898F83D3123F0040388F83D3104
:10373000564B1C4200F07981FFF7EEFC002005B0EB
:10374000BDE8F08FD9F81868D9F81C281640360C57
:103750000ED1D9F81838FF214D4A1B0C002B3FF42D
:1037600053AFDD0701D5106811605B082032F5E723
:10377000DFF820810027A8F59275F00740D5444B6B
:103780004FEA471A5AF80310D9F8142801EA02033D
:10379000D90701931ED501223D4B4AF803206A7CCC
:1037A000002F44D102F0F002602A13D1D5F8342161
:1037B0006ABB95F83D2167F3820285F83D2195F8B3
:1037C0003D2112F0040105D1FFF784FC6A7C61F30E
:1037D00007126A74019B9A0703D502222C4B4AF800
:1037E0000320019B1B070BD56A7C02F0F002202A04
:1037F00002D12548FFF75AFD0822254B4AF803203D
:10380000760807F1010708F11C08B6D1FCE6394635
:103810002048FFF7AEF895F83D211E4967F3820274
:10382000A1F5927085F83D21FFF724FAC7E702F071
:103830000F02022ACED1D8F810104FF01C0B41B95C
:103840000BFB075B9BF83D2161F382028BF83D2166
:10385000C0E70BFB075B40460021FFF78AF89BF8A7
:103860003D214146084822F004028BF83D21FFF734
:1038700001FAAFE7D80700D511605B082032D6E621
:103880000809084000000840C80D0024001080000E
:10389000080B0840EC0E0024704F4FF00008A7F111
:1038A000600A019BDA0773D50121D9F81028D9F8ED
:1038B00034584FEA481B01FA08F32B420293684B35
:1038C00018BF42F080025BF80360164016F0010357
:1038D00003933BD0029B012225EA0305604BC9F804
:1038E00034584BF803209AF81120B8F1000F57D143
:1038F00002F0F002502A10D15849A1F16000FFF700
:1039000047FB9AF87920530707D4FFF7E3FB9AF8AF
:10391000112068F307128AF811209AF8101088060F
:1039200014D5504B21F020019AF81220D3F8040846
:1039300002F00F0E22F00F0200F0700040EA0E10AD
:10394000C3F804088AF810108AF81220320703D549
:103950000822434B4BF80320F30607D5394650465F
:10396000FFF716FB10223E4B4BF8032030060FD515
:10397000039B4BB9029B39463A4A25EA03053A486C
:10398000C2F83458FFF704FB8022354B4BF8032074
:10399000019B08F101081C375B08019381D149E6BE
:1039A00002F00F02022AD1D139462F48FFF7F0FA70
:1039B000CCE72846FFF77AFAB1E63889FE883B68FB
:1039C000361A1844AE42A8BF2E461FFA86F8414662
:1039D000FFF77AFAA81BFFF769FA3B899844A7F822
:1039E0000880A5E6204A527C02F0F002102A7FF4FB
:1039F0009FAED3F8002B42F08062C3F8002B97E60D
:103A00001A480821FFF760FA90F90010A0F1150399
:103A1000C288002906DB2AB15A7C012161F3071212
:103A20005A7485E65A7C0221F8E7A3047FF5D1ADEC
:103A30000C4BD3F800296FF30A0242F04002C3F89E
:103A40000029D3F8042842F48072C3F80428DA6805
:103A500022F4705242F4C052DA60BAE5280E002413
:103A60000809084000000840C80D0024DD0D0024AE
:103A700038B50B4CE060214603681B689847054643
:103A800018B10023E360284638BD7520FCF784FF99
:103A900001212046FFF798F802232372F3E700BFC5
:103AA000C80D002470B50446EFF31185802600236D
:103AB000EFF3108372B686F3118883F31088FFF753
:103AC0002BFBEDB285F311880E4D20462368294665
:103AD0005B689847EFF311840023EFF3108372B60D
:103AE00086F3118883F310887520E4B2FCF740FF59
:103AF00000212846FFF768F80846E96084F311883A
:103B000070BD00BFC80D002470B52B4DE86808B12A
:103B1000FFF7C8FFEFF3118600238022EFF3108335
:103B200072B682F3118883F3108800212248FFF7D0
:103B30004BF875200C462972FCF71AFF75202146B8
:103B40002246FDF7A1F91D4BFF204FF0FF32F6B2E0
:103B5000C3F80809C3F8080BC3F82809C3F8280BF1
:103B6000C3F84809C3F8480BC3F86809C3F8680BE1
:103B7000C3F88809C3F8880BC3F8A809C3F8A80BD1
:103B8000C3F8C809C3F8C80B4FF48060C3F81048E5
:103B9000C3F81448C3F83448C3F81C48C3F81828BD
:103BA000FFF7BAF8FFF7A8F86B7C64F303036B74B4
:103BB00086F3118870BD00BFC80D002400000840C6
:103BC0008B4AF8B5D2F80C3823F0007343F08073B9
:103BD000C2F80C38D2F80C385901FBD5854840277B
:103BE00000F050F9844800F04DF9844800F04AF99B
:103BF000834EFFF789FF834B4FF4F4720021184680
:103C0000FDF733F880490246034604464FF01C0C8A
:103C100042F8601B4260FE22C274027500220CFB57
:103C200002411C335E641C6501F1780591F879103E
:103C300041F010016970D1B2013283F85C1061F07B
:103C40007F01072A83F84810697821F00301697021
:103C5000A3F84A70E3D100234021DAB20133C0F85F
:103C600024611C30072BC0F8144180F8202180F813
:103C70000C21A0F80E11F0D1002264497520FDF747
:103C800003F9002803DABDE8F840FFF73DBF604CB8
:103C90008023604DA360E36843F04003E3600320AA
:103CA000FCF73BFD2369002B01DB013DF7D12369C4
:103CB00043F001032361574B554C2269D20701D5CC
:103CC000013BFAD103200025FCF727FDA36B14204C
:103CD00043F48033A36300F0ABF82368322043F051
:103CE000C0032360E36823F0005343F08043E360A4
:103CF00000F09EF8C4F8005ED4F800384FF48060FD
:103D000023F4C053C4F80038D4F8003843F0030358
:103D1000C4F8003840F20123636203F59203A36202
:103D20004933C4F804314933C4F808314933C4F87D
:103D30000C314933C4F810314933C4F814314933D4
:103D4000C4F81831FEF7E8FFFEF7D6FF4FF0FF3357
:103D5000C4F81058FF21C4F814582F4AC4F8345836
:103D6000C4F818382D4BC4F81C58186820330028A4
:103D7000ACBF00204FF0084043F8200C43F8105C23
:103D800043F8181C9342F0D1254B0022FF2025490F
:103D90001C682033002CACBF00244FF0084443F8CB
:103DA000204C43F8102C43F8180C8B42F0D1184BE0
:103DB00014489A614FF0FF325A6059691A4A21F04B
:103DC0007F4121F47C0121F47C4121F0FF010A4371
:103DD00000215A61154A9A6181229A60FEF7F4FE29
:103DE000FFF79AF97520BDE8F840FCF7D5BD00BF94
:103DF000004002580BAC08000CAC08000AAE0900E9
:103E000048A20008C80D00242CA20008CD350008E7
:103E100000000840400D0300E00908400009084088
:103E2000000B0840E00B08400AFCB0F810380C000A
:103E300082B0002245F261610092009B834201D36F
:103E400002B070470192019B8B4203D9009B013362
:103E50000093F2E7019B01330193F4E703060BD4CF
:103E6000C0F30312064B53F822202AB100F00F00D2
:103E7000012311B18340936170471030FAE700BF0E
:103E800064A200082DE9F04710F080060446C0F354
:103E9000031840F0D9806E4B53F82850002D00F0E5
:103EA000D38000F4402300F00F07B3F5002F00F09B
:103EB000B780B3F5402F00F0B580B3F5802F40F008
:103EC000B380C0F30021FFF7C9FF0121EFF3118296
:103ED00000238020EFF3108372B680F3118883F300
:103EE0001088022940F0A28014F4704FC4F3033EFE
:103EF00014D023074FF00F094BBFA7F108033B462F
:103F0000242020209B0050F805C009FA03F90EFA7E
:103F100003F32CEA090C43EA0C0343514FEA470C24
:103F20000323D5F80090032903FA0CF329EA0309C7
:103F30006FEA030001FA0CF343EA09032B6078D01F
:103F400004F44033B3F5803F75D0A3F50039D9F1BF
:103F5000000343EB09035B00D5F80C9003FA0CF364
:103F600000EA090943EA0903EB60BEF1000F13D12F
:103F700023074FF00F0A4BBFA7F108033B464FF052
:103F8000240E4FF0200E9B005EF805900AFA03F312
:103F900029EA03034EF8053001F1FF3EBEF1010F9F
:103FA0000DD804F44066B6F5006F46D0B6F5406F04
:103FB00045D0A6F58069D9F1000646EB0906AB6845
:103FC00006FA0CF6BEF1010F00EA030046EA00060D
:103FD0004FF00100AE6000FA07F06B6831D8A6051B
:103FE0002FD5034301296B6014D0E30512D504F0EB
:103FF0000C04BF000F2104F1B04407F00C07D4F803
:104000000834B94008FA07F823EA010348EA030331
:10401000C4F80834D2B282F311880020BDE8F087DA
:10402000022153E7032151E731464FE74FF0000EDD
:1040300074E7002390E701238EE70226BFE70326FB
:10404000BDE723EA0003CDE76FF01500E6E700BF08
:1040500064A20008C0B2FFF715BFFFEC02060346DA
:1040600010D4C0F30311084A52F8210058B10122BC
:1040700003F00F03016902FA03F30B4214BF104669
:10408000002070470020704764A200080A460146DD
:10409000034808B500F052F8024B186008BD00BF95
:1040A00086A00008B00F0024024B0146186800F0FB
:1040B000C7B800BFB00F0024024B0146186800F0DB
:1040C0001BB900BFB00F0024024B0146186800F076
:1040D00070B900BFB00F0024F8B50D46044616466F
:1040E00000F05AF805F11F006168AB19082520F0AF
:1040F0000F00012623F00F03A0F11007DA1B114473
:10410000103AC4E9011740F8105CA1684E60A0F1B4
:10411000080140F8082CA3F108024D60E26043F862
:10412000085C50F8083C2046E2683343536000F0D6
:104130005FF82046BDE8F84000F052B801F10F03E7
:1041400070B5A2F5A27423F00F034FF4A2720C44D1
:10415000184600211D46E41A03F5A276FCF785FDFA
:10416000034600F1200200F5A071A2F110009A614F
:1041700010321033D8618A42F7D1284600F007F890
:10418000284622463146FFF7A7FF284670BD012288
:10419000002100F099B9FFEC104B37B51C680546BB
:1041A0004CB101A900F0AAF901980028D4BF002061
:1041B000012003B030BD04F04DFA00280CDB284686
:1041C00004F06CF9002801DB0120F2E700F0FEF8B2
:1041D0000368002BF3DCF7E72046EAE70404002439
:1041E000024B1B680BB904F0A5B970470404002406
:1041F00038B5054608680C4600F015F8421C05EB7A
:10420000021205EB0015AB6923B1196811B12068E2
:10421000814205D39460C4E9023203B1DC6038BD49
:104220001A469B68F0E7B0F5800F07D2030900201B
:10423000012B00D8704701305B08F9E71220704766
:1042400070B505460C46A9B1FFF7A6FF98B9EFF384
:10425000118300228021EFF3108272B681F311885E
:1042600082F31088D5F84021DBB22260C5F84041C6
:1042700083F3118870BD54F8043CA4F1080123F0C5
:10428000010344F8043C54F8083CCA185068C607B7
:1042900013D4CB58D2E902061344B06008B1D668F3
:1042A000C660126854F8080C104444F8080C5A68A8
:1042B00002F0010202435A601A4654F8043CCB1A39
:1042C0005868C00710D4D3E90210816009B1D868DA
:1042D000C86054F8081C186808441860516801F058
:1042E00001010143516019462846FFF781FF284626
:1042F000BDE87040FFF774BFF8B506460F46EFF310
:10430000118300228021EFF3108272B681F31188AD
:1043100082F310880022D0F84041DBB2C0F840217F
:1043200083F31188002C39D1002F35D007F1170500
:1043300025F00F05AF422FD83046FFF72DFFB5F51A
:10434000800F32D22846FFF76EFF06EB001084691B
:10435000FCB12368AB42A36829D3E26893600BB138
:10436000E268DA602368581B0F280CD923446119CE
:1043700060514D6025605A6802F0010202433046E8
:104380005A60FFF735FF6368083443F0010344F8CF
:10439000043C3046FFF724FF2046F8BD256821463F
:1043A00030462C46FFF74CFFBCE71220CDE71C46F9
:1043B000CEE738B50D46FFF79FFF044618B12A46F1
:1043C0000021FCF752FC204638BDFFEC08B500F098
:1043D0008DFA08B1143008BD0048FCE7B40F002482
:1043E000002303600B6813B90860486070474B688E
:1043F0001860FAE70B6802468BB180B1834208D19E
:104400001A680A604A689A4209D100234B607047D3
:104410002BB118461B689342FAD100F00BB87047D5
:104420000346006828B102681A6002B95A60002386
:10443000036070470A680346006852B148B14A6891
:1044400082424FF0000206BF4B60114601681960BE
:1044500002607047002303604B6843600A6812B92A
:104460000860486070471860FBE7002343600B68F2
:10447000036013B9C1E900007047586008607047D5
:10448000D0E9003232B90B6033B94A600023C0E989
:10449000003370471360F7E75A60F7E70D4616469A
:1044A000044608B500F02EFA31462846A047FCF72E
:1044B000D9FB30B1B2F5004F03D212B20280002016
:1044C00070476FF01500704708B530B1B2F5004F76
:1044D00003D212B20280002008BDFFF777FF162337
:1044E00003604FF0FF30F7E728B121B103880020C7
:1044F0001BB20B6070476FF01500704710B5FFF7E7
:10450000F3FF041E05DA6442FFF760FF04604FF01A
:10451000FF34204610BD1F299FBF012203688A4037
:1045200013439ABF036000206FF0150070471F29E6
:104530009FBF012203688A4093439ABF0360002013
:104540006FF01500704703460020186070471F2960
:104550009DBF0068C84000F001006FF01500704773
:104560000FB413B504AB53F8044B019303F020FFD1
:10457000019A2146503000F07AF802B0BDE81040B0
:1045800004B0704770B5044638B300F0D5F8012187
:10459000201D002600F023F8012104F1500000F056
:1045A0001EF8012104F19C0000F019F8D4F8E8503D
:1045B00025B9204600F0C8F8304670BDB5F8443043
:1045C0009B0703D430462D680646F1E701212846B3
:1045D00000F005F80028F5DAF5E70646ECE7F8B54F
:1045E000436805460F46002B3EDBB0F844309B077E
:1045F0003AD500F0BCF86C69FCB1EE69B44207D161
:10460000284600F0D4F8EC696B69E41A2046F8BD3E
:104610002B6A9C4226D1361B32462146686803F03D
:1046200000FC00280DDA95F8463043F0020385F8C7
:104630004630FFF7CBFE04686442284600F0B7F826
:10464000E4E70444361A0FB1002EE5DC6B6926441A
:10465000EB61B442D4D0EB695A1CEA6114F8012B27
:104660001A70F6E70024E8E76FF00804CEE770B5AB
:1046700086B0044616460D46014601A800F0C8F86B
:10468000204600F074F82946324601A800F05CF993
:104690000546204600F08BF8284606B070BD08B5E8
:1046A000FDF7C8FA002803DABDE80840FFF78EBE20
:1046B00008BD38B50122044600212C30FFF704FF65
:1046C0004FF0FF35002304F130006563C4E9453342
:1046D00000F03CF804F17C00C4F8805000F036F89B
:1046E00004F1C800C4F8CC50BDE8384000F02EB842
:1046F00038B504462C30FDF79DFA0023C4F8183174
:10470000D4F814516DB904F13800FFF7C8FF04F173
:104710008400FFF7C4FF04F1D000BDE83840FFF784
:10472000BEBF284650F8083BC4F81431FFF7B7FF66
:104730002846FFF7B9FCE3E710B50446204603F02E
:10474000ADFE0028FADB10BD03F0F4BE08B5002171
:104750004FF0FF330122083001814360FFF7B4FEC0
:10476000002803DABDE80840FFF730BE08BD70B589
:10477000044603F0ABFF0546E368984203D1238A61
:104780000133238270BD04F10806304603F086FE33
:10479000031E07DAFFF71AFE0368042BF5D08C2BF3
:1047A000F3D05B42002BEDD10123E560E9E710B5C2
:1047B000044603F08BFF238A012B0ED1002304F162
:1047C000080023824FF0FF33E36003F0B3FE0028BC
:1047D00005DABDE81040FFF7F9BD013B238210BDAB
:1047E00001210069FFF7FBBE38B504460D4621697B
:1047F000284600F0B3FD013003D0E3680133E360E5
:1048000038BDFFF7E3FD0368042BF0D0F8E7FFECB9
:10481000094B03604B6963B1B1F84430074A13F4A4
:10482000807F074B08BF134683600023C0E9033134
:104830007047024BF8E700BFE947000899530008AA
:10484000E1470008421E11F8013B02F8013F002B2E
:10485000F9D170470B4610B562B913F8012B002A45
:10486000FBD104E013F8014B00F8014B14B9581ABE
:10487000013810BD013AF5D10270EEE703461A4641
:10488000013311780029FAD1101A704710B502448B
:1048900004460139904205D011F8013F00F8013B70
:1048A000002BF7D1121A0021FCF7DFF9204610BDCA
:1048B00030B50C4B0025D3E900428A4208D0A14212
:1048C00006D0013508331F2DF5D10C464FF4805228
:1048D0008368C46123F4805323F00F031343836080
:1048E000002030BD84A20008C06970471FB50020B9
:1048F00001A903F077FD0028ACBF0298002005B0A5
:104900005DF804FB2DE9F0410A4D2B6843B90A4CD0
:104910000A4E0B4FDFF82C80B44203D101232B60E9
:10492000BDE8F08154F8043BBB42F5D34345F3D2D4
:104930009847F1E7B80F002480A5000880A500087B
:104940000000000880A5000807B5009200220B4671
:10495000114600F003F803B05DF804FB2DE9F04FB9
:104960008FB004460025DDF860B01978002900F00A
:104970000084252907D0013302932368204601359E
:10498000D9469847E9E393F801A09A1CBAF1250F9C
:104990000292F2D000273E46B846B8F13F0F48D801
:1049A000BAF12B0F3AD010D8BAF1200F38D0BAF1A3
:1049B000230F3BD0BAF12A0F58D118F4807F5BF84F
:1049C000043B4AD023EAE37707E0BAF12D0F2AD05F
:1049D000BAF1300F30D148F00108029B13F801AB57
:1049E0000293BAF1000FD8D1AAF14503022B00F2CD
:1049F00097800AF1200A48F400585FFA8AFA18F4FE
:104A0000807F08BF0627BAF1650FF9B240F09E809B
:104A1000013148F48048C9B200229FE048F0020802
:104A200048F00408D9E748F00808D6E748F010082D
:104A3000D3E7B8F5007F24D2AAF13003DBB2092B0B
:104A4000B8D818F4807F4FF00A020ABF48F08008F7
:104A500002FB073702FB0636BFE7002BA7BF48F073
:104A600080081E465E4248F08808B6E7BAF12E0F6D
:104A700040F0768318F4807F40F07B8348F48078A0
:104A8000ABE7BAF17A0F0FD0BAF1740F0CD0BAF1CC
:104A90006A0F06D128F480681FFA88F848F4206865
:104AA0009BE7BAF16C0F0BD118F4007F18BF48F4E4
:104AB000006828F480681FFA88F848F400788CE7CA
:104AC000BAF1680F0BD118F4806F18BF48F4006872
:104AD00028F400781FFA88F848F480687DE7BAF176
:104AE000700F81D128F420681FFA88F848F4007804
:104AF0000AF0DF03532B40F0C481D946A24B59F88A
:104B000004ABBAF1000F08BF9A4618F4807F5046F4
:104B100014BF39464FF0FF3100F040FC07460FE06C
:104B2000AAF16503022B7FF66AAFBAF1630FDFD1FA
:104B3000D94601270DF1200A59F8043B8DF82030A1
:104B400018F0080F40F08F81B04686E1BAF1660F89
:104B50007FF462AF0A4648F400480F210BF1070BBF
:104B60000F2908A82BF0070928BF0F21B9EC020B69
:104B700000F032FB9DF82430DDF820B003F009028C
:104B8000012A38D018F0020F38D1C8F3800A4FEA52
:104B90004A1A13F00C0F3ED0BAF1000F0CBF0323DA
:104BA0000423B3420CDA18F0080FA6EB030608D171
:104BB00037462368202120469847013FF9D13544E4
:104BC0000026BAF1000F04D0236851462046013573
:104BD00098479DF8243008F400586C4F13F0080FE4
:104BE0006B4B08BF1F463B469A461AF8011B41B95A
:104BF000EF1BFD18A9E04FF02D0ACAE74FF02B0A72
:104C0000C7E7B8F1000F01D02039C9B223682046A8
:104C100098475346E8E7C3B2B8F5804F01931AD2DC
:104C20001A4608A905330B44019919B113F8011D5F
:104C3000302929D01BF1040F2BDB934529DABBF176
:104C4000000F48F4004802DB019B9B4524DA0BF17E
:104C50000107019BDF1B0FFA88F3002B0393B6BFFC
:104C60002BEAEB7305230133BAF1000F00D00133B7
:104C7000A7B17A1C1344B342B4BFF31A002318F04F
:104C8000090F1FD11E4614E001990139C9B20191E3
:104C9000CAE7019B5F1EDEE70027DCE718F0100F74
:104CA00018BF0133E7E7202120460493013E9047D7
:104CB000049B2268002EF6D11D44BAF1000F05D1E5
:104CC000B24648E01E46BAF1000F04D023685146B0
:104CD00020460135984718F0080FF1D0039B002BB0
:104CE00058DA2BEAEB7A7B42ABEB0A020493019B86
:104CF0000AF1FF3A04999A4236BF08AB3027D3181D
:104D000002F1010238BF5F796B1C8A450393236867
:104D100026DA18F0100F06D0BAF1FF3F03D12E218A
:104D200020469847039DD3450AD19DF82530352B61
:104D300028D805D19DF8243013F0100F08BF312773
:104D400001352368394620469847374602E2013E3E
:104D50003021204698472368002EF8D15544BDE7FE
:104D60003946204605929847BAF1FF3F059A07D188
:104D7000AB1C2E2120460592039323689847059A81
:104D8000039DB4E73127DBE77CA300088FA0000870
:104D90008BA000089DF82510204631291EBF9DF8E4
:104DA000243023F010038DF8243023689847002F17
:104DB00023683BDD2E21204698470122023592468A
:104DC000019920462368013551450AF1010A88BF3F
:104DD00038325FFA8AFA92BF30216A4412F8131C03
:104DE000984757455246EBDA18F4005F236820468F
:104DF0000CBF652145219847BBF1000F04DB1FD193
:104E00009DF82430DB061BD5CBF1000B2D21236848
:104E1000204698473021BBF1090F13DC2368204658
:104E20009847043523680BF130018CE718F0100F18
:104E300001D10135D8E72E21204602359847D3E726
:104E40002B21E4E70131ABF10A0BC9B2E3E708F12A
:104E5000FF3823682021204698474745F7D335443B
:104E60004646A5EB08050AEB070806E0236820463E
:104E70001AF8011B984706B1013EC245F6D13D44E0
:104E800063E7BAF1640F08F4206302D0BAF1690F46
:104E90007BD1B3F5206F63D10BF1070B2BF0070B20
:104EA000D946DBF8041059F8080B28F4805B002978
:104EB0002BF0100B06DA40424BF4805B61EB4101B2
:104EC0001FFA8BFB1BF4807F04D01FB950EA01034B
:104ED00000F0CA800DF1200A0A23524600F04EF974
:104EE000A0EB0A005FFA80F81BF4807FCDF8048005
:104EF00000F0BC802BF0010A47451FFA8AFA40F304
:104F0000B88044F21002FBB20BEA0202102A03D16D
:104F10002BF0110B1FFA8BFA1AF0100F00F0B38070
:104F200008F138026A4412F8192C302A40F0A380A4
:104F30002AF4C04A2AF0100A1FFA8AFA1AF0080F57
:104F400040F0B2801AF0010F06D09E4240F3C680B6
:104F5000F31A03EB0807F3B25B1B5FFA83FB9EE0D7
:104F6000D94618F4007F59F8040B4FEAE0719CD140
:104F700018F4806F99D018F4006F0BBF40F3C03164
:104F800040F3C01100B240B28FE7B3F5206F1DD1DE
:104F90000BF1070B2BF0070BD946DBF8041059F87F
:104FA000080B28F0060BBAF1580F1FFA8BFB47D0FD
:104FB000AAF16F03DAB2092A4AD8092B48D8DFE8E8
:104FC00003F05127474747471847473818F40071FF
:104FD0000BF10409DBF8000001D00021E1E718F42F
:104FE0008063FAD018F4006301D180B2F5E7C0B253
:104FF000D7E728F016080A231FFA88FB1BF4807FE6
:1050000003D017B950EA01022ED00DF1200A64E74F
:10501000029B1B78562B0AD1029B013302934368F3
:105020001A68079201682046FFF78EFC95E04BF066
:10503000100B1BF0100F01D04BF4804B1023DDE759
:1050400018F0100F01D04BF4C04B4FF40473D5E7A8
:10505000236820462521023598472368514620467B
:1050600098477AE00823C9E7B8463DE74346DA4661
:1050700052E7434650E71AF4804F01D1013300E074
:105080000233DBB25AE741F206021AEA020F3FF49A
:1050900055AFF3E7236820212046013598470BEBF5
:1050A0000503DBB29E42F5DC9E42CCBFF61A002619
:1050B0001AF0100F14D023683021204698471AF4B4
:1050C000804F33D01AF4005F05F1020523680CBF4E
:1050D0007821582120469847BA4619E047463BE7D1
:1050E00041F206031AEA030FF6D01AF0020F05F197
:1050F0000105236814BF2B2120211AF4805F18BFFB
:105100002D21E7E70AF1FF3A23683021204698472E
:10511000C245F7DCA7EB08034745B8BF00231D4491
:10512000B8F1000F04D1019B1D440EE60135D3E711
:1051300008F1FF330EAA204652FA83F25FFA83F891
:10514000236812F8181C9847EAE7013F23682021DA
:1051500020469847002FF8D13544CB46029B04E403
:10516000BAF17A0F3FF4A5ACBAF1740F7FF48FACAB
:105170009FE428460FB0BDE8F08F00BF2DE9F8434B
:1051800013F400791C4606460F4618BF23F400743A
:10519000154618BF4FF001094FEAE478304639460A
:1051A0002246434604F08AF8092AB4463B4606469E
:1051B0000F4609DC3032A44505F8012B73EB0803D8
:1051C000ECD22846BDE8F883B9F1000F01D03732A0
:1051D000F1E75732EFE7FFEC2DE9F74F10EE904A79
:1051E00007460E4614F000441CBFB1EE400B0124EC
:1051F000B5EE400BF1EE10FA11D121EAE172053063
:10520000302144F00204FBF730FD0025BB190022D9
:1052100030465A713C713D6003B0BDE8F08FB4EE8A
:10522000400BF1EE10FA02D744F00804EDE79FEDD1
:10523000407BB4EE470BF1EE10FA02DD44F00404BB
:10524000E3E79FED3D6BB4EEC60BF1EE10FA14D41C
:105250003D4908230F25012031ED027B20EE077B1D
:10526000B4EEC67BF1EE10FA04DB00FA03FCB0EEFC
:10527000470B6544013BEFD216E09FED316B33499C
:1052800008230F25012031ED027B20EE077BB4EED1
:10529000C67BF1EE10FA05D500FA03FCB0EE470B21
:1052A000A5EB0C05013BEED232B125EAE5730133E3
:1052B0001A449642A8BF1646254B03EBC60393ED4E
:1052C000007B30EE070B9FED1E7BB4EEC70BF1EEBB
:1052D00010FA04DBB2EE047B013580EE070B07F118
:1052E000040BDFF87090DFF870A051EC100B03F0A6
:1052F000FFFF6FF0030388460090DB1B0193019BC7
:105300005B449E4282DD4A4653460098414603F084
:10531000D5FF3030514600920BF8010F98464846B1
:105320000A22002303F0CAFF81468A46E7E700BF4E
:10533000FFFFFFFFFFFFEF7F00003426F56B0C43FC
:105340000080E03779C3414350A4000898A40008C6
:1053500088A300080080C6A47E8D030037B50A46E6
:105360008DF8070004460D460DF10700012100F0FD
:1053700021F800280BDD0A2C0BD195F846305B078D
:1053800007D501212846FFF72AF9002801DA4FF056
:10539000FF34204603B030BD002070470246014470
:1053A00010B58A42134603D01C780132002CF8D184
:1053B000181A10BD2DE9F04106460F46154642B9B0
:1053C000FFF704F84FF0FF34092303602046BDE8DF
:1053D000F081B2F844309B070CD4FEF7F7FF0923A5
:1053E00003604FF0FF3495F8463043F0020385F830
:1053F0004630EBE753693BB90A460146686802F05C
:1054000010FD041EE2DAECE71046FFF7B0F928467B
:1054100000F045F8002807DA4FF0FF342846FFF780
:10542000C6F9002CD2DADEE7D5E90640241A202C92
:1054300001D11F2F23D8BC42314628BF3C4622460B
:10544000A7EB0408FBF7FCFAEB69AA692344344490
:105450009342EB610CD2B8F11F0F13D9424621469B
:10546000686802F0DEFC0028D6DB0444A41BD5E704
:1054700000212846FFF7B3F80028ECDACCE73446E1
:10548000B846EBE7B8F1000FF0D021464246E86994
:10549000F419FBF7D5FAEB694344EB61E6E710B585
:1054A000044630B9FEF792FF092303604FF0FF3046
:1054B00010BD4369E3B1FFF75AF9206A626990426F
:1054C00013D0E36994F847101B1A2046C4E9072259
:1054D0000022591A84F84720012200F00BF8002816
:1054E00003DA2046FFF763F9E0E72046FFF75FF9AC
:1054F0000020DDE700F000B870B504460D46164602
:10550000FFF7CDFF002802DA4FF0FF3070BD2046D4
:1055100000F010F80028F7DB0023324629466068C7
:1055200084F8473002F05FFB01304FF0FF3018BFC6
:105530000020EBE7426932B1B0F844309B0702D556
:105540000121FFF74CB800207047022901D100F07B
:1055500061BB012901D100F0C1BB704708B500F063
:1055600083FBBDE8084000F0FFBBFFEC38B50F4DF2
:1055700004462B7813F0FD0F09D1C20707D500F0C0
:105580007FFB002803DB0A4B02221A7004E02B7811
:10559000012B02D94FF0FF3038BDA307FAD500F038
:1055A000EFFB0028F6DB024B0122EEE7D2140024C9
:1055B000D114002410B5084C606004F019F8FFF70E
:1055C000D5FF002804DB054A13680133136010BDC2
:1055D0006368002BF1D1FAE7C0140024BC14002446
:1055E00008B5FFF7E7FFA0F120035842584108BD76
:1055F00073B5044601AE00256420FFF7DBFF0028E9
:1056000007DB013506F8010B042DF5D1019B0020C5
:10561000236002B070BDFFEC70B5094E04460D4624
:105620003378022B01D100F051FB3378012B05D1E7
:1056300029462046BDE8704000F0B8BB70BD00BFF1
:10564000D214002410B5114C236801331DD06268B8
:105650000F4B9A4219D90F4B9B6803F1006303F576
:1056600000339A4211D204F023F803F0EFFFFFF762
:1056700075FF03F0F9FF03F0BDFF204604F032F898
:105680002046BDE8104004F0F1B810BD000002084B
:10569000FFFF0108AC00002410B500230B4C54F8A8
:1056A000232022B154F82320013A44F82320013367
:1056B000042BF4D1064B1B7833B9A36823B902201D
:1056C00004F0B6F83223A36010BD00BFC01400245C
:1056D000D0140024024BD860DA68002AFCD170474D
:1056E000C01400242DE9F04FAF4B8FB000250646C3
:1056F000DFF8C0821D700395DFF8C8A2D8F8084013
:1057000003F090FF0EB1CAF80060DFF8BC924FF0D2
:10571000FF37CAF8085089F80050012004F078F8E3
:1057200026B1DAF80030002B00F067820020FFF786
:1057300041FF0490049B002BF2DB012004F058F899
:10574000049B213B1F2BE8D801A252F823F000BF95
:10575000595800086F580008D15700081B57000817
:105760001B5700081B570008F95800081B57000872
:1057700097590008515A00087F5A0008BF5A00087C
:105780003F5B0008E15A00080F5B00089D5B0008C2
:105790002F5800081B5700081B5700081B5700080C
:1057A0001B5700081B5700081B5700081B57000811
:1057B0001B5700081B5700081B5700081B57000801
:1057C0001B5700081B5700081B570008D758000834
:1057D00000250220FFF704FF002800F00382039B4E
:1057E00003F00303032B40F0FD8101234FF0000B76
:1057F000022089F8003003F0FBFF03F064FF5846F5
:1058000003F075FF0446002867D1022089F80000E4
:1058100003F0FEFFD8F80830A34265D8039B0024AC
:1058200043F0040389F800400393CAF80840039B3F
:105830005D4A03F00303032B137808BF002613B956
:105840005A4B1B78137041F21203022106A8ADF8DF
:105850001830FFF7E1FE60E70220FFF7C1FE0028E5
:1058600000F0C081039B43F001030393DFE74FF493
:105870007A70FFF79FFE051EC0F2B4810220FFF789
:10588000AFFE002800F0AE81681E042800F2AA8155
:10589000DFE800F0030B0E11140004214448FFF769
:1058A000BBFE039B43F00203DFE704214148F6E718
:1058B00004214148F3E704214048F0E71C2528462D
:1058C000043503F030FF0421069006A8FFF7A4FE7C
:1058D0002C2DF4D1E5E701257BE7584629460BF14D
:1058E000010B03F00AFF8AE7204603F01CFF01309A
:1058F00040F0518104348DE73220FFF75BFE051E36
:10590000C0F2708115F0030240F06C812B19D8F8B9
:1059100008108B4200F26681B5F5807F00F262814B
:10592000DFF89CB05946AA4214D1C820FFF758FEB0
:10593000002800F0578124B9214B4FF0FF321F6837
:105940001A6025F003052544AC4215D1039B43F0B2
:1059500008038AE74FF47A70CDE90021FFF72AFEA9
:10596000049004980028C0F23D8104980199009A9F
:1059700001F8010B0132D6E7DBF80010204603F0F6
:10598000CCFE204603F0CFFE5BF8042B904240F0A3
:1059900002810434D8E70220FFF722FE002800F03D
:1059A00021810025AB4643E0D2140024D114002409
:1059B00098A40008AC000024B0000024B400002427
:1059C000BC130024C0140024D01400240DB9791C89
:1059D0003CD1284603F0A7FE894B06905B68BBB913
:1059E000DFF81CC21A46082142F30000013920F0FA
:1059F000925020F4EF2020F49B6020F0070080EA12
:105A00005202F1D101334CF8042BB3F5807FE9D178
:105A100006A9002211F8013B0132794883EA0B0301
:105A2000042ADBB250F8233083EA1B2BF2D1043571
:105A3000D8F80830AB42C9D8042106A8CDF818B070
:105A4000FFF7EAFD039B43F010030EE73846C3E778
:105A5000002305A80593FFF7CBFD002840F0C28086
:105A60000220FFF7BDFD002800F0BC80059803F080
:105A700064FE0421069006A8FFF7CEFDD7E60023BA
:105A800005A80593FFF7B4FD002840F0AB80022085
:105A9000FFF7A6FD002800F0A5800598820740F0DA
:105AA000A180082800F29E8003F09AFE042106904F
:105AB00006A8FFF7B1FD039B43F04003D5E60220A3
:105AC000FFF78EFD002800F08D8003F039FE0421E1
:105AD000069006A8FFF7A0FD039B43F08003C4E6F1
:105AE0000220FFF77DFD00287CD006A9142003F0DA
:105AF0002DFE05460421059005A8FFF78DFD2946DA
:105B000006A8FFF789FD039B43F48073ADE60220EE
:105B1000FFF766FD002865D020223A49172506A820
:105B2000FEF7B4FE042105A80595FFF775FD29468B
:105B300006A8FFF771FD039B43F4007395E664200C
:105B4000FFF738FD00284DDBC5B21E2D4AD80220D4
:105B5000FFF746FD002845D04FF4D07003F0E3FD79
:105B600083464FF4D27003F0DEFD274B9B4539D1BD
:105B7000264B984236D1DFF898B04FF4D07045EA02
:105B80000B0B594603F0C9FD4FF4D07003F0CBFD69
:105B900058453FF44CAE41F2121356E64FF47A707A
:105BA000FFF71EFDF0B17B1C0DD141F2120306A8D8
:105BB0000221ADF81830FFF72FFD64200FB0BDE8CB
:105BC000F04FFFF787BD039B03F01B031B2B09D18D
:105BD0003946002003F0A1FD002003F0A4FD874218
:105BE000E3D0D8E741F21233022106A8ADF818300D
:105BF000FFF712FD002303938FE50FB0BDE8F08F90
:105C0000BC0F002493A00008FFECC2925D7D05C587
:105C100000ECC29238B50F4B0F4C002808BF184655
:105C200003F0C2F90D49206003F0CCF90C4B00B130
:105C300018604FF0FF320B4D432118682A6002F0C4
:105C400081F8002805DB28602068BDE83840FEF7B1
:105C50002BBA38BD3FA00008D4140024ABA0000824
:105C6000D81400247400002410B5044C206801F0FE
:105C70003FFE4FF0FF33236010BD00BF74000024CF
:105C800013B50F4C2368002B0FDA0E4B4321186815
:105C900002F058F8002803DA4FF0FF3002B010BDD0
:105CA000094B20601868FEF7FFF901220DF107018A
:105CB000206802F081F80128EED19DF80700EDE799
:105CC00074000024D8140024D4140024024B0A4683
:105CD0000146186802F0A5B8740000241E4B70B588
:105CE000002808BF184688B003F05EF91B49064635
:105CF00003F068F9054638B31849002003F062F94B
:105D000030B303F00FF804464321284602F01AF896
:105D1000031E13DB124D69462B6003F08BF9029BC7
:105D20002146684623F4B87343F030030293FEF72C
:105D3000BFFD6A460021286803F081F9304608B0AB
:105D4000BDE87040FEF7B0B94FF4E134054DDBE734
:105D50004FF4E134D8E700BF3FA00008ABA0000833
:105D600078000024ADA0000810B5044C206801F0B4
:105D7000BFFD4FF0FF33236010BD00BF780000244B
:105D8000094B07B5186800280BDB01220DF107014C
:105D900002F012F8012804D19DF8070003B05DF865
:105DA00004FB4FF0FF30F9E778000024F8B5044613
:105DB00046184FF47A75094FB44208D1F8BD012254
:105DC0002146386802F02DF8012804D0013D002D4D
:105DD000F5D10134F0E74FF47A75FAE77800002442
:105DE00003464FF604720846934210B513D04FF69F
:105DF0000C72934212D04FF60172934224D1FAF7FB
:105E00007FFF0028044613DA6442FEF7DFFA0460DD
:105E10004FF0FF340CE003F019FEF2E70B78012B92
:105E200015D14B78012B05D0022B08D07BB900246B
:105E3000204610BD4968807801F07EFAE1E74B68A2
:105E4000186801F0F1FAF2E76FF01804DCE76FF080
:105E50001504D9E708B500F05FFDBDE8084000F083
:105E600013B8002070471046704708B54AB14B6818
:105E70008A6803F0050313438B6013B1086902F0CD
:105E80001BFB002008BDFFEC00234FF4DB7202492E
:105E9000024802F05DB900BF9CA40008B8A0000849
:105EA00070B504460D46A36B20469B6A98470028B0
:105EB000F9D0A36B294620461B6ABDE870401847FD
:105EC0002DE9F74F458C0446B0F9263088462DB2AF
:105ED0004FF0800901920135AB42D8BF0025A28C5A
:105EE00012B2AA420AD0638C2DB2A26A00201BB261
:105EF00002F80380658403B0BDE8F08F019B002B9E
:105F000030D0EFF3118AEFF3108772B689F311885E
:105F100087F31088A28C12B2AA421ED1E27802F056
:105F2000FF0BE2B90121A26B20466170526A9047D3
:105F300004F11A0002F078FAA26B06465946526A3A
:105F4000204690475FFA8AFA8AF31188E27862B9AC
:105F5000002EC4DA6FF00300CDE70026F2E76FF001
:105F60007F06EFE76FF00A00C5E76FF07F00C2E73A
:105F70002DE9F74F836880460E4601925C6904F173
:105F80002C0A504602F050FA051E12DB00254FF095
:105F9000800B019B9D4204D2E37873B10DB96FF081
:105FA0007F05A36B204601219B699847504602F06C
:105FB00083FA284603B0BDE8F08F238EE28D19B234
:105FC00012B28A421ED0626B0133525C1BB2B4F92A
:105FD00032109942D8BF00232386E36813F4E07F90
:105FE00005D00A2A07D113F0400F18BF0D22013542
:105FF00006F8012BCDE70D2AF9D113F4807F18BFE5
:106000000A22F4E7002DCCDCD8F80830002B49D068
:10601000D8F8001011F0400147D1EFF31189EFF3E8
:10602000108772B68BF3118887F31088A26B204615
:106030005FFA89F992699047E18D228E09B212B216
:10604000914227D1A26B0121204692699047E18DB0
:10605000228E09B212B2914202D089F3118898E7D8
:10606000E278A2B9012204F11C00A27002F0DCF96E
:1060700089F31188002802DBE378002B89D0002DFA
:106080008FD1E378002B8AD16FF0030589E76FF099
:106090007F00EDE789F31188A36B012120469B69FE
:1060A000984776E76FF050057BE76FF00A0578E7D1
:1060B0002DE9F04183685E6906F11805284602F073
:1060C000B3F9041E23DBF378002B36D13378013388
:1060D00013F0FF0734D0012F2DD1EFF311880023E7
:1060E0008022EFF3108372B682F3118883F3108855
:1060F00033795FFA88F86BB9B36B30461B68984701
:10610000041E07DA88F31188284602F0D5F92046E4
:10611000BDE8F081B36B30469B689847041EB36BB3
:1061200003DA5B6830469847ECE79B69012130460B
:10613000984788F311883770E6E76FF07F04E3E74C
:106140006FF01704E0E7F7B50E4600F13C0700F1E9
:106150004C0557F8044F8CB16368A26843F01803EC
:1061600033401343A3604BB101A92069FEF7BCF98A
:10617000019B002B02DC206902F09EF9AF42E8D1BE
:1061800003B0F0BD2DE9F84383680E4615465C69FF
:1061900004F11E08404602F047F9071E47DB002DB8
:1061A0004FD004F13C02002352F8045F002D34D19B
:1061B000103304F1200944F8236004EB83034846BC
:1061C000736102F063F9638CB4F926201BB20133CA
:1061D0009A42D8BF0023A28C12B29A422AD14846D2
:1061E00004F12C0902F068F9484602F04FF9E28DFB
:1061F000238E484612B21BB29A421EBF736803F048
:1062000001031D4302F058F9E378BBB145F01805CE
:1062100029462046FFF797FF06E00133042BC3D140
:1062200000236FF00F077361404602F045F93846CE
:10623000BDE8F883756805F00405D0E7002DF3D0BC
:10624000E6E77369002BEFD01D607561ECE7FFECAA
:106250002DE9F047836880460F4616465D69464B38
:106260001B6823B1EB78ABB16FF07F0425E002F03F
:10627000A7F80028F6D105F1200A504602F0D4F81C
:10628000041E1ADBEB7803F0FF018BB3504602F0DB
:1062900013F9E9E7EFF3118400238022EFF3108371
:1062A00072B682F3118883F3108807EB0608B845AD
:1062B00006D1E4B284F3118834462046BDE8F08765
:1062C0002B6917F8011BD80703D50D2905D11A072B
:1062D00005D42846FFF7E4FDE9E70A29F9D113F0D0
:1062E000240F03D00D212846FFF7DAFD0A21F0E73D
:1062F000D8F80030B146284683F04008AB6BC8F3AD
:1063000080185B6A9847B9F1000F01D1344623E049
:106310002B6917F8011BD80703D50D290AD11A07D5
:106320000AD442462846FFF7CBFD041E10DB09F1D4
:10633000FF39E8E70A29F4D113F0240F01D10A212B
:10634000EFE742460D212846FFF7BAFD041EF6DAB4
:10635000B14501D2A6EB09046A8CAB8C12B21BB218
:106360009A4204D0AB6B012128465B6A984750469D
:1063700002F0A2F8A1E700BF040400242DE9F047D1
:1063800000F1200804460E46404602F04DF8051E76
:106390001DDBEFF3118700238022EFF3108372B629
:1063A00082F3118883F31088E37803F0FF0553B379
:1063B000638C6FF07F05A384FFB287F311881E4FB3
:1063C000002DD7F800902CDA404602F075F82846E8
:1063D000BDE8F087A36B0121204684F801A05B6A29
:1063E0009847484602F020F8A36B054600215B6AF7
:1063F00020469847002DDFDB628CA38C12B21BB2C3
:106400009A42E7D1D8E74FF0010A04F11A09F3E7FD
:106410004FF47A7002F0E4F83B68A3EB0903B3424F
:1064200006D2A36B2046DB6A98470028F0D0CBE762
:106430006FF07305CBE700BFE01400244FF0FF338B
:106440002DE9F0418B6005460B790C462BB14B6969
:1064500043F001034B6105230B610122002104F18C
:10646000200004F11A07FEF724F80122002104F1AC
:106470002C00FEF71EF80122002104F11800FEF79F
:1064800018F80022384604F11C061146FEF711F8F0
:10649000002230461146FEF70CF80122002104F1DB
:1064A0001E00FEF706F80021384602F0E7FB002147
:1064B000304602F0E3FB234628464FF4DB720249E4
:1064C000BDE8F04101F044BEBCA4000810B504468C
:1064D0000121FFF738FEA3783BB1002304F11C0033
:1064E000A370BDE8104001F0E7BF10BD10B5044631
:1064F0000421FFF728FE63783BB1002304F11A0062
:106500006370BDE8104001F0D7BF10BD70B583685F
:106510000E4615465C69A36B1B69F3B9B6F58D7F12
:106520000DDAB6F58A7FC0F2B680A6F58A73052B20
:1065300000F2B180DFE803F07995AFAFA1ABB6F51B
:10654000427F36D040F209339E424ED040F20733AC
:106550009E420AD06FF0180093E0984710F1190F8F
:10656000DCD0002800F099808BE0EFF3118100234C
:106570008022EFF3108372B682F3118883F31088C0
:10658000228EE38D12B21BB29A420ADCE38D228E78
:106590001BB212B29B1ACAB282F311882B60002080
:1065A0006FE0228EE08D12B2B4F9323000B2121ACE
:1065B000F0E7EFF3118100238022EFF3108372B62E
:1065C00082F3118883F31088A28C638C12B21BB201
:1065D0009A4203DC638CA28C1BB2DAE7A28C608C3B
:1065E00012B2B4F9263000B2E1E7EFF311810023D3
:1065F0008022EFF3108372B682F3118883F3108840
:10660000628CA38C12B21BB29A4206DAA38C628C03
:106610001BB212B29B1A013BBDE7628CA08C12B276
:10662000B4F9263000B2121AF4E7EFF31186002312
:106630008022EFF3108372B682F3118883F31088FF
:1066400035F0020301D1E38D2386013D012D04D8ED
:10665000638C2046A384FFF749FFF6B286F31188C6
:106660009DE742F210712046FFF788FE002896D081
:1066700010F1190F3FF46EAF03E0002D02DA6FF056
:10668000150070BDA368002BF9DAA56087E74FF00D
:10669000FF33A36083E76FF0180040F201139E42BE
:1066A0000BD0B6F5817FECD1002DE8D02B68E360EC
:1066B0006B682361EB68636171E7002DDFD0E368ED
:1066C0002B6023696B606369EB6068E770B5044613
:1066D0000D46EFF3118600238022EFF3108372B68C
:1066E00082F3118883F3108881F00103C37089B9A4
:1066F0001821FFF728FD637823B104F11A006570B3
:1067000001F0DAFEA3782BB1002304F11C00A37082
:1067100001F0D2FEF6B286F3118870BD10B50446C2
:1067200000211A3001F013FF002104F11C0001F0D8
:106730000EFF012104F1200001F009FF012104F105
:106740002C0001F004FF04F11E000121BDE81040FF
:1067500001F0FDBE70B5836805465C6904F118065A
:10676000304601F093FE2378012B06D9013B2370BC
:10677000304601F0A1FE002070BD0021A36B204631
:1067800021709B6998472B685B0604D44FF47A61AB
:106790002046FFF7F3FDEFF3118500238022EFF38E
:1067A000108372B682F3118883F31088A36B20469E
:1067B000DB68984723791BB9A36B20465B68984731
:1067C000EDB285F311882046FFF780FE2046FFF7E3
:1067D000A5FFCDE710B54369044613F0010003D0CF
:1067E0000A44914201D1002010BDA368002B04DDB2
:1067F0000B78032B03D01A2B03D00131F1E70A20C9
:10680000F2E70720F0E770B5002504462E46628CBB
:10681000A38C12B21BB29A4211D1628CA38C12B219
:106820001BB29A4204D1A36B002120465B6A9847B1
:10683000ADB2EDB12046BDE87040FFF757BEA36B87
:1068400020469B6A98470028E7D0A38C2046A16A7F
:106850001BB2A26BC95C126A9047A38CB4F92620C4
:1068600001331BB29A42A38400DCA6840135CEE733
:1068700070BD2DE9F341C58D0026B0F932300446D4
:106880002DB237460135AB42D8BF0025A36B204659
:10689000DB69984770B916B12046FFF717FE37B18C
:1068A0003946A06801F07AFE2046FFF737FF02B0B4
:1068B000BDE8F081B4F8308001A9A36B20460FFA3F
:1068C00088F85B69984701228DF803000DF10301F8
:1068D0002046FFF77FFFA8450746D7D0E38D013656
:1068E0009DF803101BB2626BB6B2D1542BB20135C6
:1068F000E385B4F93230AB42D8BF0025C6E7FFECE0
:1069000008B5044B186818B103689B6803B1984731
:10691000002008BD7C000024002070477047C36B36
:1069200093F85430002B0CBF6FF07F0000207047AD
:10693000704700207047C36B93F85500032894BF3D
:1069400000200120704770B5036805460E469B681D
:106950009847044650B1C6803046FDF7ADFB206035
:1069600028B92B6821462846DB6898470024204632
:1069700070BD806890F8543013B10121FFF7A6BEB6
:10698000704700218068FFF7A1BE10B5836840F210
:10699000093081425B6900F0A98011DC40F20730C8
:1069A000814264D0B1F5427F00F0848040F2011052
:1069B000814228D0B1F5817F50D06FF018000DE0F2
:1069C00040F6025081420AD040F60350814213D073
:1069D00040F601508142F0D15A66002010BD002AD5
:1069E00000F0A580D3F85A101160B3F85E109180C2
:1069F00093F860309371F0E7002A00F0988093F8E4
:106A000058301360E9E7002A00F09180D9681160DE
:106A1000196951605969D16093F85F10E1B101F1D2
:106A2000FF3EDEF1000141EB0E0148024FF48071A0
:106A300093F85E400843A4F1020CDCF1000444EB3F
:106A40000C0440EA841040F0300090601046D3F807
:106A50005A10FDF72DFFC0E70846E9E7002A66D087
:106A60001168D96051681961D2685A61B5E7EFF3CE
:106A7000118000218024EFF3108172B684F3118815
:106A800081F310881C8ED98D24B209B28C4205DCAA
:106A9000D98D1B8E09B21BB2CB1A07E0198EDC8D83
:106AA00009B2B3F9323024B2091B5B1AC1B281F3C7
:106AB0001188A6E7EFF3118000218024EFF3108105
:106AC00072B684F3118881F310889C8C598C24B29F
:106AD00009B28C4203DC598C9B8C09B2DBE7998CA0
:106AE0005C8C09B2B3F9263024B2DDE7EFF31180F4
:106AF00000218024EFF3108172B684F3118881F3B2
:106B000010885C8C998C24B209B28C4206DA998C7C
:106B10005B8C09B21BB2CB1A013BC7E7598C9C8C2A
:106B200009B2B3F9263024B2091B5B1AF4E76FF0FF
:106B3000150053E770B50D46044658B151B10868C9
:106B400008B1FDF7B1FA236829462046DB68BDE8A5
:106B50007040184770BD10B590F85430044693B19A
:106B6000002180F85410FFF7B1FDA06E03685B6848
:106B70009847E06E03685B689847206F0368BDE83C
:106B800010405B68184710BD70B50C468568EFF380
:106B9000118600238022EFF3108372B682F31188EE
:106BA00083F3108800212846FFF790FD2846FFF761
:106BB000D2FF0023F6B26B84AB8486F3118823687E
:106BC0005B6923B120460121BDE87040184770BDC4
:106BD0002DE9F04184680D46002C49D02046FFF78E
:106BE000BAFF3220FDF724F9A16E29B12B6828469F
:106BF0005B6898470023A366616F21B16868FFF75F
:106C000099FF00236367264604F130074FF0000820
:106C1000D6F8E41021B1206FFFF78CFFC6F8E480AE
:106C20000C36BE42F4D1216F29B12B6828465B682F
:106C3000984700232367EFF3118600238022EFF3A8
:106C4000108372B682F3118883F3108804F18808E8
:106C5000D4F8887077B9F6B286F31188E16E21B165
:106C60002B6828465B689847E76600236384A38403
:106C7000BDE8F0814046FDF7D3FB41680029E7D02D
:106C8000E06EFFF757FF94F85530013B84F855301C
:106C9000DEE7FFEC2DE9F84F84680D46804621655C
:106CA0004B6840219C606868FFF74DFE60670028D4
:106CB00079D03E4B0122C36028462B6894F8AC1073
:106CC0001E68032341F08001B047A06630B96FF021
:106CD000120429464046FFF77BFF61E084600122F1
:106CE0002B68284694F8B0101E68022341F08001FA
:106CF000B047E0660028EAD0846000222B6828466E
:106D000094F8B4101E680223B04720670028DED034
:106D100004F1E00604F5887A4FF0000B8460B14678
:106D20004021206FFFF70FFE706000283BD0A6F8CF
:106D300008B006610C3656F8082C1D4B5645D3603A
:106D4000EED104F1C0064FF0800A6021E06EFFF73B
:106D5000FAFD706038B30661164A7368DA60EFF3C3
:106D6000118BEFF3108772B68AF3118887F31088BE
:106D700004F188013046FDF733FB94F855205FFAA3
:106D80008BF3013284F8552083F3118808364E4581
:106D9000DBD12B685B6913B1012128469847002499
:106DA0002046BDE8F88F6FF00B0492E71D690008DC
:106DB00083710008ED72000837B504461546084691
:106DC0001A466946002300F08BFB23682A46694671
:106DD0001B682046984703B030BDFFEC2DE9F04119
:106DE00090F8543004460E468B4242D0FFF7B3FE73
:106DF000002E3ED0012E44D1002204F19807A06E4F
:106E00003B461146FFF7D8FF051E36DBA36E002276
:106E100002219C603B46E06EFFF7CEFF051E2CDB97
:106E2000E36E324631469C603B46206FFFF7C4FF5D
:106E3000051E22DB236F264604F13007DFF8488069
:106E40009C60D6F8E410C1F80C80206F03681B69C1
:106E50009847054688B994F856300C360133BE423F
:106E600084F85630EDD10121204684F85410FFF704
:106E70002DFC00252846BDE8F0812046FFF76BFE7B
:106E8000F8E76FF01505F5E7837100082DE9F84381
:106E90000F46117884689E4611F060095388656F2B
:106EA00092F803809078B2F804C0D6887CD15278EA
:106EB000063A052A00F2CF80DFE802F003CD423A1D
:106EC000644BB8F1020F26D0B8F1030F2CD0B8F103
:106ED000010F40F0C0802C6800F0FEFA00F11002B3
:106EE000234650F8041B904243F8041BF9D1028852
:106EF00012201A8086424FF001032946A8BF064699
:106F00002B71EE80786803681B699847002809DABE
:106F100000236B8106E004F19801286800F015FB5E
:106F20000028E7DABDE8F883296800F099FAF7E766
:106F3000002940F09080D9B22046FFF74FFFEFE7DD
:106F4000802940F088802B6894F854201A70012022
:106F5000D0E701297FD194F85420012A7BD1D4F8BD
:106F60009C20944502D00132944574D1002B72D1FB
:106F70002046FFF7F0FD94F854102046FFF72EFF4F
:106F80000020B7E7812966D194F85420002A62D105
:106F9000D4F89C20944502D00132944558D1002B5E
:106FA00056D12A681370D2E7B9F1200F53D1527825
:106FB000203A032A4FD8DFE802F014023140A12919
:106FC00049D1D4F89C309C4545D1D4F85A200720AB
:106FD0002B681A60B4F85E209A8094F860209A7149
:106FE00088E7212937D1072E35D1D4F89C309C452C
:106FF00031D1BEF1000F0BD0DEF80030C4F85A30AA
:10700000BEF80430A4F85E309EF8063084F8603094
:10701000636E002BB4D000209847B1E721291AD124
:10702000D4F89C20944516D103F0030384F858301B
:10703000636E002BA4D00120EEE721290BD1D4F8F8
:107040009C309C4507D1636E002B99D00220E3E76A
:107050006FF0200066E76FF05E0063E700230B81AE
:10706000006F4968C388CB8003681B691847FFEC31
:107070002DE9F0470446EFF3118800238022EFF357
:10708000108372B682F3118883F3108800F17809B7
:107090004846FAF7C1FF94F85930002B44D004F168
:1070A000900AD4F890502DB95FFA88F888F31188C7
:1070B000BDE8F0876A6800212B8910681789184499
:1070C000B4F93220FF1AE38D0133BFB29BB2934271
:1070D000A8BF0023228E8EB212B293420DD116B1F8
:1070E0002046FFF7F3F9B7421BD85046FDF798F951
:1070F00029462046FFF7B2FFD3E7B742EFD9E68D26
:1071000010F801C00131626B36B202F806C01AB243
:107110000133E2859BB2B4F932209342A8BF002329
:10712000D8E72B891E442E81D4F89030002BBBD099
:107130002346034AC821484601F0D6FAB4E700BF07
:107140007F71000810B5C06BEFF31184002380221B
:10715000EFF3108372B682F3118883F3108859B16C
:1071600090F8593013B9012380F85930FFF780FFA8
:10717000E4B284F3118810BD80F85910F8E7FFF7E6
:1071800077BF38B584680869EFF311850023802242
:10719000EFF3108372B682F3118883F31088B1F98C
:1071A0000A3013F16E0F0CD08BB9038104F19001FA
:1071B000FDF716F92046FFF75BFFEDB285F3118866
:1071C00038BD94F85630013B84F85630F5E7014657
:1071D0002046FFF743FFF0E72DE9F74F8346EFF333
:1071E00011834FF0800A01930022EFF3108272B6F0
:1071F0008AF3118882F31088D0F86C80B8F80620E2
:10720000602A38BF60220092DBF888707FB37D6807
:107210002868EFF31189EFF3108472B68AF31188AE
:1072200084F310880021BBF822C08EB2BBF8242062
:107230000FFA8CFC12B2944502D0009BB3421DD8C9
:10724000BBF82210BBF8242009B212B2914205D13A
:10725000DBF8382000215846526A904716B158464C
:10726000FFF744F95FFA89F989F31188EEB99DF8BF
:10727000043083F3118803B0BDE8F08FBBF82460BD
:10728000DBF8282036B2925D4254BBF82420BBF9CB
:107290002660013212B29642ABF8242003DC4FF094
:1072A0000003ABF824300131BDE70BF18800FDF796
:1072B000B7F89BF8552029464046013A8BF85520EF
:1072C0000122EE802F612A71D8F8002012699047C0
:1072D000002899D0CBE741B1C06B428C838C12B2AD
:1072E0001BB29A4201D0FFF777BF704770B50D46C9
:1072F00084680869EFF3118600238022EFF310837E
:1073000072B682F3118883F3108804F18801F6B213
:10731000FDF766F894F85530013384F8553086F35C
:107320001188B5F90A3023B92046BDE87040FFF74F
:1073300053BF70BD7047FFEC2DE9F04F8FB0242292
:1073400080460F4605A80021F9F78FFC04234FF073
:10735000020A4FF0010B0693032343F25420CDF8A9
:1073600010A0CDE9083BCDE90AA3FCF7A5FE044631
:1073700038B96FF00B0507B13C6028460FB0BDE887
:10738000F08F43F2482904AE002104F198054A46E3
:10739000F9F76BFC84F857800FCE0FC50FCE0FC5E1
:1073A00096E80300C2231D4A85E8030084F85B3099
:1073B0000823102184F85CB084F860304FF4167311
:1073C00084F803B06846638604F58873636342F605
:1073D000E063E38404F55A73A362114BC4E90E34ED
:1073E00004F5405383F84CA2C3F848220D4AC3F871
:1073F0005042434601F059FC21466846FFF71EF80B
:10740000051E04DA20460024FCF74EFEB3E74C4488
:107410002046FCF72DFB0546ADE700BF0CA5000894
:10742000DCA40008C2A0000830B585B085680B4A0E
:10743000102195F857300446684601F036FC68463E
:1074400000F0A7FE2046FCF72DFB05F17800FAF7C7
:10745000E3FD2846FCF728FE05B030BDC2A00008B9
:1074600070B50C4604282BD8DFE800F01503211D69
:107470001F00154D2846FDF701FA0023A21C1946EE
:10748000834202F1020214DB4000032302306370E6
:10749000C0B2207006E0032304204B70092308705B
:1074A0008B70C87070BD094DE4E7094DE2E7094DE6
:1074B000E0E7EE5C013302F8011C02F8026CDFE742
:1074C0006FF01500EEE700BFD0A0000802A1000891
:1074D000E6A00008D6A000080048704724A50008D0
:1074E000012813D002281FD068BB07230B70052387
:1074F0004B705369487163F07F038B700323CB702B
:1075000040230B710A238B710720704707230B70F0
:1075100005234B70D36988718B700223CB70402395
:107520000B7100234B71EFE707230B7005234B70A2
:107530009369C87063F07F038B7040230B71002345
:107540004B710123DFE7002070472DE9F0410D4624
:107550000446002800F087800021042624274FF0ED
:1075600003080846FFF7F1FF8023012102224FF0B4
:10757000090EA070E3710012FA23A671E0704FF0BB
:10758000100CA672052084F800E06270227161710F
:10759000237284F809E06B6884F815C04FF0060C7C
:1075A000E3720023A074E67584F81AC04FF0070C4C
:1075B000E07684F81E8023736173A273E2732174F2
:1075C0006374E7742375A1752776627627776177F0
:1075D0006F6884F820C00F4484F82100E7776F6952
:1075E00084F823804FF00A0867F07F0784F825307D
:1075F00084F8268084F82270402784F827E084F8F5
:10760000247084F828606E6884F82A300E4484F868
:107610002B2084F82C8084F8296084F82D3084F89D
:107620002E3084F82F3084F830C084F83100EE69B1
:1076300084F8332084F8326084F8347084F835306C
:1076400084F8361084F837C084F83800A86960F0F0
:107650007F0084F8390084F83A2084F83B7084F87D
:107660003C3084F83D103E20BDE8F08110B5144652
:107670000846114601F0A6F9204610BD0846FBF762
:1076800077B900F042B9F8B5837804460E468B42CC
:1076900023D2CB00FF2B22D88900406801F09EF94D
:1076A000074668B1A5788020FCF70EFD47F8250055
:1076B00070B9013DA378AB4205DD3846FCF7F4FC18
:1076C0006FF01600F8BD57F82500FCF7EDFCF0E769
:1076D0000135AE42E7D86760A6700020F2E76FF090
:1076E0001700EFE701220021FCF7E3BEF8B50446DE
:1076F0008578013D07D26068FCF7D6FC2046BDE8DE
:10770000F840FAF78CBAAF0070266368D859304455
:10771000103E00F023FA16F1100FF6D16368D85925
:10772000FCF7C2FCE5E72DE9F74FDDF830A089460C
:107730001E460192074600F0CFFD054600F0A6FE6A
:10774000041E3FDBBAF1000F5146AA78B8BF0AF118
:107750000701C9108A42884609DC01312846FFF733
:1077600092FF041E03DA284600F0A6FE2AE0DAF1B2
:1077700000020AF00704686802F0070258BF54428A
:1077800050F828104FEA880A01EB04118A68FAB908
:10779000C1F8009028466A68019B52F80A2002EB63
:1077A000041253606A6852F80A2002EB04129760D0
:1077B0006A6852F80A2002EB041204EBC804D6608F
:1077C00000F07AFE204603B0BDE8F08FD846D7E738
:1077D00001341031082CD9D108F1010BAA7800240A
:1077E0005A45F3DC08F102012846FFF74CFF041E5E
:1077F000B9DB6B680AF1040A019A4FEACB0453F82B
:107800000A30C3F800906B6853F80A305A606B680E
:1078100053F80A309F606B6853F80A30DE60A2E7C5
:10782000F8B5002305460F460B6000F055FD0646EF
:10783000F0B1002D1FDB8378B5EBC30F1BDA00F02E
:1078400025FE041E12DB7368EA1005F007053046BA
:1078500053F8223003EB05153D60AB68002B04BFE5
:1078600000256FF008043D6000F026FE2046F8BDBC
:107870006FF00A04FAE76FF00804F7E7F0B585B097
:10788000044600F029FD054600F000FE002814DB48
:10789000002C0DDBAB78B4EBC30F09DAE2106B6898
:1078A00004F0070453F8223003EB04139A6832B94A
:1078B000284600F001FE6FF0080005B0F0BD1A4642
:1078C0006E4603F110071068083252F8041C344663
:1078D000BA4203C42646F6D1102200211846F9F711
:1078E000C4F9284600F0E8FD684600F037F9E4E7FF
:1078F00010B5FFF7C3FF041E05DA6442FCF766FD0E
:1079000004604FF0FF34204610BD00F05BB8FFEC80
:1079100038B50F4C00F0DAFE05466368984204D192
:10792000238900200133238138BD204600F0B6FDB5
:10793000002807DAFCF74AFD00680428F5D08C28F7
:10794000F3D040420028EFD1012365602381EBE7AB
:107950008400002408B500F0B9FE0A480389012B11
:107960000CD1002303814FF0FF33436000F0E2FDB0
:10797000002805DABDE80840FCF728BD013B03817B
:1079800008BD00BF8400002410B503460446184615
:1079900013F8012B2AB9001B1C30FCF795FB18B912
:1079A00010BD2F2AF3D1F6E700F11803013C14F8BB
:1079B000012F12B900221A70F2E72F2AFAD003F829
:1079C000012BF4E708B50348FFF7DEFF024B186010
:1079D00008BD00BF3FA00008DC14002400232DE9EF
:1079E000F04116461360027888B0002A45D08DF821
:1079F0001C30CDE9010301A8CDE90333CDE90533FE
:107A000000F04AF8002835DA019FDDE903543846D2
:107A100000F036F8037880463846D3B1FFF7B4FF5C
:107A200048B96FF00B04069808B1FCF73DFB2046FF
:107A300008B0BDE8F0813DB16B68C0E90043686003
:107A4000474604460025E2E7A368C0E90043A0607A
:107A5000F6E7FFF799FF0028E3D035B16B68C0E97E
:107A60000043686000243060DDE7A368C0E900439C
:107A7000A060F7E76FF01004D5E76FF01504D6E7C4
:107A80000278034601300AB12F2AF9D11846013392
:107A900002782F2AFAD07047F8B5036804461A789E
:107AA0002F2A08D02A4A14302A4901F0F1F86369D4
:107AB000002B46D02360284B196823681A782F2A98
:107AC00042D100252E4641B90A466FF001002261DD
:107AD000C4E90031C4E90265F8BD53B301F11700F0
:107AE0005F1E10F801CF17F8012FBCF1000F06D16F
:107AF00082B12F2A0ED04A680E461146E3E722B122
:107B00002F2A02D09445F6D3EBD900216FF0010063
:107B10000A46DCE71846FFF7B3FF0346007858B182
:107B2000CA8902F00F02032A08D08A680D46002194
:107B3000E2E71A461946C8E71A46C8E71A4600207F
:107B4000C5E76FF00B00C7E76FF01500C4E700BF93
:107B50003FA00008EBA00008DC14002470B5866884
:107B600005467EB134691CB164680CB1A047044677
:107B7000304600F03FFB0023C5E90033C5E902337E
:107B8000204670BD3446FBE770B5866804460B4658
:107B900015463EB136692EB136691EB1B047002890
:107BA0000DDA70BD012D05D0022D0AD025B16FF080
:107BB0001500F6E762681344002BF8DB6360606829
:107BC000EFE76FF05700ECE737B50C4601A9154613
:107BD000FFF726FE002804DB2A4621460198FFF71E
:107BE000D3FF03B030BD10B5FFF7EEFF041E05DA7A
:107BF0006442FCF7EBFB04604FF0FF34204610BDFD
:107C0000C389024613F00F0014D013696BB1CA0781
:107C100001D59A6862B111F002000BD0DB68002B2D
:107C20000CBF6FF00C00002070476FF0050070472C
:107C30006FF00C0070472DE9F047054688B092467A
:107C4000984600295BD012F0060F4FF0000601A8FD
:107C5000019114BF109B4FF4DB79069618BFD3F83F
:107C600000908DF81C60CDE90266CDE9046600F055
:107C7000AEFA041E19DB029F51463846FFF7C0FFDB
:107C8000041E0DDB1AF4006FC5E900A6C5E90276F3
:107C900010D00599284600F0B7F90028044611DAFB
:107CA00000233846AB6000F0A5FA069868B1FCF7EF
:107CB000FBF90AE0FB8903F00F03032B10D13B69AA
:107CC0001C6834B90698A0B90024204608B0BDE865
:107CD000F08729EA0803524605992846A047DCE7C1
:107CE000012B09D13B691B68002BEBD02846984734
:107CF000D3E7FCF7D9F9E7E76FF00504D0E76FF0B9
:107D00001504E2E770B5044686B00D46164600F04D
:107D100071FF214603462A4602A80096FFF78BFF13
:107D2000041E0CDB002304980093059BDDE902127E
:107D3000FFF7F9FC041E02DA02A8FFF70FFF204646
:107D400006B070BD0EB417B505AA52F8041B019217
:107D5000FFF7D8FF041E05DA6442FCF737FB046026
:107D60004FF0FF34204603B0BDE8104003B0704729
:107D700010B403688468DB0707D55CB123694BB195
:107D80009B683BB15DF8044B18476FF00C005DF841
:107D9000044B70476FF00800F9E737B50C4601A9AE
:107DA0001546FFF73DFD002804DB2A4621460198D1
:107DB000FFF7DEFF03B030BD10B5FFF7EEFF041E86
:107DC00005DA6442FCF702FB04604FF0FF34204602
:107DD00010BD10B40468A40708D583685BB11B69A3
:107DE0004BB1DB683BB15DF8044B18476FF00C00FA
:107DF0005DF8044B70476FF00800F9E737B515469A
:107E00000C4659B101A9FFF70BFD002804DB2A46F7
:107E100021460198FFF7DDFF03B030BD6FF015007C
:107E2000FAE710B5FFF7EAFF041E05DA6442FCF733
:107E3000CDFA04604FF0FF34204610BDB1F5417F0C
:107E400008B5C36805D159681046FCF7FBFC002053
:107E500008BD6FF01800FBE770B5C56806460C4614
:107E60002868002954D0212A52D9C38903F00F036E
:107E7000032B0BD103690A4629465B6B9847002800
:107E800042DB736822200133736040E0A968002957
:107E90003CD021221831601CFCF7DCFC002323704D
:107EA000AB681A696AB1DB8903F00F03013B062B4B
:107EB00007D8DFE803F01D041B1F21231900062348
:107EC0002370AB689A680AB91B690BB90423237045
:107ED000FFF71EFDAC686368AB608BB9FFF73AFD36
:107EE000204600F087F9CCE70923E9E70423E7E718
:107EF0000223E5E70323E3E70523E1E70723DFE7C1
:107F00009A8901329A81E9E7831C00D1002070BD73
:107F10006FF01500FBE770B5C468D4E90056EB8933
:107F200003F00F03032B10D12B691B6B43B9002403
:107F3000284600F05FF93046FCF7B6F8204670BDE1
:107F40002146284698470446F2E7A06808B100F0A9
:107F500051F92046FCF7A8F8E9E72DE9F043064679
:107F60008BB089461746002A48D1D0F80C80446867
:107F7000D8F80050EB8903F00F03032B20D1A14266
:107F80000CDA2B699B6B2BB96FF0850420460BB084
:107F9000BDE8F0833C46414628469847A14503DCAE
:107FA000002CF3DB7460F1E72B6901AA41462846F7
:107FB0005B6B9847002801DB0134EFE70446EFE7ED
:107FC000A142BABFAD681446D8F80850FFF7A0FC2C
:107FD0000DB1A1450FD1D8F80870C8F8085015B1F7
:107FE000AB890133AB81FFF7B5FC002FD8D0384601
:107FF00000F000F9D4E701346D68E9E7012A0CBF0D
:1080000044686FF01504C1E7F7B5856806460F466A
:10801000EB8903F00F03032B19D12B6923B3DC6A1F
:1080200014B35B6B03B301AA2846A047041E0BDB05
:10803000019B1D60019D384600F0B6FF68600D4849
:10804000C6E9020500F0B3F8204603B0F0BD0C20ED
:10805000FCF73AF8034650B1019000240560A86887
:10806000986000F0A4F8E5E76FF05704ECE76FF0D4
:108070000B04E9E790000024C3685968FFF7C4BF08
:108080002DE9F347061E884614461F465DDB12B9EC
:1080900000F0A2F90446022E19DC4C23A4687343B5
:1080A00030331C4404F1240304F14402666063612C
:1080B0002362A4F84480C4E906230C2384F84630E4
:1080C000002F40D10025284602B0BDE8F08701A965
:1080D0003046FFF7A5FB051E08DB019B9868A0B1A1
:1080E0004146FFF78DFD30B16FF00C05002FEAD04F
:1080F00000233B60E7E74C20D4F80890FBF7E4FF4F
:10810000044628B96FF00B05F0E76FF00105EDE7C5
:1081100009F12C0A504600F087F9051E03DA2046C3
:10812000FBF7C2FFE2E7D9F818314BB11C605046AB
:10813000C9F8184100F0C0F92046FCF707FBB1E789
:10814000C9F81441F3E73C60BCE76FF00805CDE7E0
:108150002DE9F34107460E4690461D46FFF7D8FB32
:10816000041E12DB01AA41463846FFF737FC041E05
:1081700009DB019B0024DA8922F00F0242F00102A0
:10818000C3E90465DA81FFF7E5FB204602B0BDE8EC
:10819000F08138B50546FFF7BBFB041E05DB28461A
:1081A00000F06BF80446FFF7D5FB204638BD38B524
:1081B000044650B1FFF7ACFB051E04DBA389013375
:1081C000A381FFF7C7FB284638BD0546FBE738B556
:1081D0000546FFF79DFB041E0ADB2846FFF75CFC03
:1081E000041EA1BF6A68938901339381FFF7B2FB34
:1081F000204638BD10B50446C8B1FFF789FB0028FA
:10820000FBDBB4F90C304BB9E389DB060BD5FFF788
:10821000A1FB2046BDE8104000F044B8013B1BB272
:10822000002BA381F0DDBDE81040FFF793BB10BD2C
:1082300010B5044688B0D0B100240123019001A8F4
:1082400006948DF81C30CDE90244CDE90444FFF7D3
:1082500023FCA04207DBDDE90242636852B15360B0
:108260000023C4E90033069808B1FBF71DFF204640
:1082700008B010BD049A9360F2E710B5FFF7D8FF7D
:1082800068B1B0F90C4034B1C28942F01002C28129
:108290006FF00F0010BD00F005F82046FAE76FF010
:1082A0000100F7E710B5044650B14068FFF7FAFF48
:1082B000A068FFF7F7FF2046BDE81040FBF7F4BECB
:1082C00010BD00F069BBFFEC024A13680133136074
:1082D000704700BFE0140024024B1B68986800B18F
:1082E00024307047D80400240F4B10B51B68044697
:1082F000B3F92020002A0ADD1A7C037C9A4206D2B8
:108300000A49F9F7DFFE0123002023770AE0064936
:108310002046F9F7D7FE02230028F5D00322227762
:108320002268137710BD00BFD8040024CC040024B9
:1083300038B5436804465BB90368032201251A7700
:1083400020460449FCF79CF800232846237738BDD3
:108350000025F5E7D8040024F0B5134D0020134C98
:1083600002262A68236813B923606360F0BD1F6882
:10837000BAB193F810C0117C8C450CD95168C3E98F
:10838000002151B953600120167703222B601A7720
:108390001A463B46E7E71268EAE70B6053600222A1
:1083A000F5E75368FFDE00BFD8040024CC040024A6
:1083B000024B1B6898682C30704700BFD80400241B
:1083C000044B1B6823B11868B0FA80F0400970476D
:1083D00001207047D8040024014B1868704700BF83
:1083E000D804002438B50F4B0C461D6870B1F9F75E
:1083F000BDFBA0B1EB8B03F00303022B07D0AA68EF
:1084000083689A4203D06FF00C0007E02846436B64
:108410002360836B6360C36B0020A36038BD6FF083
:108420000100FBE7D8040024174A38B51468EFF3BD
:10843000118500228021EFF3108272B681F311883A
:1084400082F31088E0B1028812B2002A028802F199
:10845000FF3212B2028006DD002323640020EDB259
:1084600085F3118838BD00232064052120466384EC
:10847000F9F7ACFEB4F922000028EFD04042EEE755
:108480006FF01500EBE700BFD804002410B50446D8
:108490002046FFF7C9FF031DFAD010BD10B5FFF746
:1084A000C3FF041E06DA6442FBF790FF04604FF03E
:1084B000FF3010BD0020FCE738B5002834D0EFF3C2
:1084C000118500238022EFF3108372B682F31188A6
:1084D00083F31088038847F6FF721BB2934205D1DD
:1084E000EDB285F311886FF08A0038BD038801333F
:1084F0001BB2038003881BB2002B0EDC0C4B1C68E4
:108500005CB1236C83420DD104F12400F9F784FDA2
:10851000002320462364F9F731FFEDB285F311887B
:108520000020E2E72468EBE76FF01500DDE700BF0D
:10853000C404002410B5FFF7BFFF041E05DA64422F
:10854000FBF744FF04604FF0FF34204610BD70B5C8
:1085500005460C46F8F7F0FCEFF311860023802265
:10856000EFF3108372B682F3118883F310882B889F
:108570001A0409D42B881B040ED5F6B286F3118891
:10858000F8F7EAFC002070BD002CF3DD013C284622
:10859000FFF792FF24B2EAE72C80EEE737B5041E1E
:1085A0000D4616DB1F2917D8F8F7C6FC0023042256
:1085B000204669468DF800508DF801308DF8022074
:1085C0000193F9F765F90446F8F7C6FC204603B0B5
:1085D00030BD6FF05704F9E76FF01504F6E7FFECD4
:1085E00007B568B1084A0021B0FBF2F302FB1300A3
:1085F00000934FF47A7358430190684600F0EEF808
:1086000003B05DF804FB00BF40420F0038B50F4CCB
:1086100025682846FFF78CFE0D4B1B680BB1FFF752
:108620009BFE246828460421238C013323840223E3
:108630002377F9F725FD0121E86800F019F80323F5
:108640002377238C013B238438BD00BFD80400244A
:10865000CC040024054B186830B1037F032B01D1F3
:10866000C06870476FF00200704700BFD804002454
:1086700070B50E46EFF3118500238022EFF31083CF
:1086800072B682F3118883F31088F9F76FFA044603
:10869000EDB2A0B1027F0C4B53F83210FBF7F0FEA5
:1086A00085F31188002120463246F9F705FAE18B5F
:1086B000204601F00301BDE87040F8F7C1BE85F324
:1086C00011886FF0020070BD38A10008054B1868D2
:1086D00030B1037F032B01D1C06870476FF00200F7
:1086E000704700BFD80400242DE9F0410C4616461F
:1086F0009846054600284ED0002A4CD000294ADB77
:10870000EFF3118700238022EFF3108372B682F318
:10871000118883F3108843680BB1F9F77DFC1F497A
:1087200001346E600E68C5F80C801EB92846FBF750
:1087300057FE24E030463246002391685B1801D58D
:10874000116831B9A3420CDC116829B9E41A134944
:10875000ECE710460A46F0E78868034410460A46EC
:10876000F0E791689642A3EB0103A4EB0304A1EBAD
:10877000040191600AD10949284600F040FAAC6032
:10878000FFB287F311880020BDE8F081034A294633
:1087900000F03BFAF3E76FF01500F5E7380A002424
:1087A00038B50D4C236843B19A680025013A9A60A8
:1087B000236813B19B68002B00DD38BD2046FBF712
:1087C0002FFE23681BB19A6881680A449A60436847
:1087D0004560C0689847EBE7380A00242DE9F74365
:1087E0000F46054600283BD042681F4B9A4237D8B7
:1087F000EFF3118600238022EFF3108372B682F329
:10880000118883F31088DFF864906846F6B2D9F8CF
:108810000080FBF798FE2A460021684600F038F8F1
:1088200010F10B0F044606D186F311880024204670
:1088300003B0BDE8F08387B101A9284600F002FA31
:10884000D9F8003001983946A3EB080290428ABF5C
:10885000C01A0020404400F0E7F986F31188E6E7EB
:108860006FF01504E3E700BFFFC99A3BE014002452
:10887000027F062A0AD140F2FF22A0F85C2074226F
:1088800080F85E2000220266F9F778BD7047FFECA1
:10889000394B2DE9F74306460D4691461C68EFF328
:1088A000118800238022EFF3108372B682F31188BF
:1088B00083F3108807682046F9F726FB38405FFAF3
:1088C00088F70190A0B101A8F8F7A4FE0146204660
:1088D000F8F74EFE1DB143682B6083686B60067924
:1088E000F8F76AFE87F31188304603B0BDE8F083DD
:1088F0003368A364B9F1000F32D0D9F8040004F151
:1089000024081E4A0023C117D9F800E08018DFF8B8
:1089100078C01B4A41F10001EEFB0C0100F0CEFCD7
:1089200023460146174A4046FFF7DEFE2046062151
:10893000F9F74CFC4046F9F76FFB94F85C10002304
:108940001F29A36411D83046FBF701FE80B194F8CB
:108950005C60002DC6D0E36D2B60236E6B60C1E7B9
:1089600006212046F9F732FCE7E76FF00A06F0E748
:108970006FF00306EDE700BFD80400243F420F006C
:1089800040420F007188000800CA9A3B08B500F009
:1089900027FC002008BDFFEC10B5084B4FF0E02489
:1089A0000022074963610F20A261F8F76DFA0723DF
:1089B0000F202361BDE81040F7F7EEBFFF5207001C
:1089C0008D89000838B504464518207808B1AC42B6
:1089D00000D138BD0134F9F7CBFFF6E7024B0A4668
:1089E0000146186800F002B8B00F00242DE9F84FD6
:1089F000074692460D4621B91146BDE8F84FFBF7F0
:108A00007BBC32B9FBF71CFC4FF0000B5846BDE8AD
:108A1000F88F02F1170323F00F0B5A45F4D8A1F198
:108A20000804FBF7B9FB55F8088CC3450AD804D2F3
:108A30005A462146384600F0ABF83846AB46FBF7BD
:108A4000CFFBE3E755F8041C04EB080921F0010112
:108A5000D9F80430611ADA0748684CBF002654F888
:108A60000860C30706EB080354BFD1F800C04FF0FD
:108A7000000C63445B4576D3B445ABEB080308D2E6
:108A80009C4555D2A3EB0C03BCF1000F53D1AB4670
:108A900026E09E42FBD29B1BB246D1E902208260B7
:108AA0000AB1C868D0609C45A4EB030446D90A68A3
:108AB0003846D21A43440A6023600A6842F0010231
:108AC0006260D9F8042002F001021A43C9F80420B8
:108AD000FBF78EFB04F1080BBAF1000F1BD05346D5
:108AE00009EB0600D9E90212916011B1D9F80C2006
:108AF000CA6022689E421A4422602ED9F61AA11832
:108B0000A65023684B60436803F00103334343607E
:108B10003846FBF76DFB3846FBF762FB5D453FF4DB
:108B200075AFA8F1080229465846F7F789FF6DE7A7
:108B30004FF0000AB1E79A466346AEE722686368E1
:108B4000424443F0010322606360D9F8043003F02B
:108B500001031343C9F80430BCE7436803F0010381
:108B600013434360D7E73846FBF73AFB5146384694
:108B7000FBF7C2FB834600283FF448AF2946A8F123
:108B80000802F7F75DFF29463846FBF759FB3DE73A
:108B9000F0B40C680B4606460D196968C90719D46C
:108BA0001859D5E902172844B96009B1ED68CD60BC
:108BB0001D6899181C59AD1A25449D504A601A60C9
:108BC00044689B5804F001041C4344603046F0BCE8
:108BD000FBF70EBB02F110018C4209D39918A41ABD
:108BE0009C504A601A609B5843F001036B60EEE7AB
:108BF000F0BC704708B500F037FA406B08BD0B6851
:108C0000036003B948600860704703460846114690
:108C1000126812B14A689A4201D1FBF7E1BB1A68A7
:108C2000026018607047FFEC4FF47A7290FBF2F329
:108C300002FB13000B60024B584348600020704752
:108C400040420F0038B543680C460568084AD917FA
:108C5000E5FB02311846074B074AC0184FF00003E6
:108C600041F1000100F0DAFA2060002038BD00BFB9
:108C700000CA9A3B3F420F0040420F00084631B104
:108C8000481E01288CBF6FF015006FF085007047FB
:108C90000EB403B503AA52F8041B019200F01DF8AC
:108CA00002B05DF804EB03B070470CB40A4600B59F
:108CB00089B071B1014602A800F020F90BAA0A9907
:108CC00002A80192FBF740FE09B05DF804EB02B088
:108CD000704702A800F02AF9F0E7F0B58DB014460D
:108CE0000D46074602A8019200F020F922462946C7
:108CF00002A8FBF729FE059E01363046FBF7DCF99A
:108D0000044660B10146324606A800F0F7F8019A21
:108D1000294606A8FBF718FE3C600DB0F0BD4FF0E9
:108D2000FF30FAE70A22002100F000B873B50C46C4
:108D30001646019090B301A800F02AF9019B1D7816
:108D40002D2D01D02B2D12D1013301933246214616
:108D5000019800F025F82D2D0FD1B0F1004F08D962
:108D6000FBF734FB222303604FF0004003E00025B3
:108D7000ECE7F9D0404254B910E0002805DAFBF7DF
:108D800025FB222303606FF000403CB135B123681E
:108D900013F8012CAA4201D1013B236002B070BD3F
:108DA0002DE9F04385B00E46154604460190002893
:108DB0004FD001A800F0ECF8019B1F782D2F01D0B7
:108DC0002B2F19D101330193284601A900F045F852
:108DD000051E13DAFBF7FAFA00241623036076B3B4
:108DE0003FB1019B13F8012CBA4204BF03F1FF33DA
:108DF0000193019B336022E00027E5E74FF0FF3845
:108E00000024B8FBF5F805FB08F96FEA0909019B96
:108E100003AA2946187800F095F858B1444503D8BC
:108E2000039B10D199450EDAFBF7D0FA4FF0FF34CF
:108E3000222303602D2FD2D16442002ED1D12046AF
:108E400005B0BDE8F08304FB0534019B01330193B9
:108E5000DDE70029CDD10C46F1E770B502460D469D
:108E60000C68A8B92378302B24D16378661C03F0F2
:108E7000DF03582B04D11021A07800F063F820B94B
:108E80003446082210462C6070BD02341022F9E7E7
:108E9000102809D12378302BF4D1637803F0DF0355
:108EA000582BEFD10234EDE7831E182BEAD94FF08F
:108EB000FF30E9E70A22E5E738B5C36805464469AB
:108EC000E41A944228BF1446002C0ADD00692246A9
:108ED0001844F7F7B5FDEB682A6900212344EB60DD
:108EE000D154204638BD07B501228DF807100DF189
:108EF0000701FFF7E1FF03B05DF804FB064B013A01
:108F00000360064B42614360054B83600023C0E968
:108F100003310B70704700BFE78E0008B98E000860
:108F200099530008C3680133C3607047034B036063
:108F3000034B83600023C360704700BF258F000888
:108F4000995300080A290ADC2F281EDD2F3181429F
:108F50001BDBA0F13003012002B11360704724290C
:108F600013DCA0F13003092BF3D9602805DD56315D
:108F700081420ADBA0F15703EDE7402805DD3631D9
:108F8000814202DBA0F13703E5E700231846E3E75F
:108F900070B5044605682E460135307800F069F852
:108FA0000028F8D1266070BD38B50546FBF766FC91
:108FB0000130FBF781F8044610B12946FBF742FC6B
:108FC000204638BD014A00F003B800BFE414002475
:108FD0002DE9F041884616460446C0B12546297859
:108FE0002C460135D1B1404600F01AF80028F6D1E0
:108FF00029782F46013539B1404600F011F8002894
:10900000F6D000233B702F462EB1376003E012B13B
:109010001468002CE2D12046BDE8F0810C46FAE746
:1090200003461A78184601338A4202D0002AF8D142
:10903000104670470A4640F2011100F08FB870B533
:10904000044616460D4639B100F022F8022D03D130
:109050000021204600F017F8324620464FF4817177
:10906000BDE8704000F07AB808B5FBF73FFC006837
:1090700008BD202805D0093804288CBF0020012015
:109080007047012070470A464FF48A7100F066B8B5
:10909000002240F2151100F061B8F0B5876885B084
:1090A00004460D461668002F55D03B69C3B940F2FF
:1090B0000D339D420DDCB5F5417F0EDBA5F5417505
:1090C000092D0AD8DFE805F02A0909090909091656
:1090D000222640F20F539D422CD06FF0180007E07B
:1090E0005B69002BE3D03246984710F1190FDED0B0
:1090F00005B0F0BD236836B1326822B143F04003B9
:1091000000202360F4E723F04003F9E7236843F4E9
:109110008063F5E7236823F48063F1E7FB8903F0BC
:109120000F03032BD9D03146384605B0BDE8F040D7
:1091300000F032B83B69002BCFD05B69002BCCD05C
:1091400001AA40F20C51204698470028D0DBBDF917
:109150000C303380CCE76FF00800C9E70EB477B568
:1091600007AD01A955F8046B0095FEF759FB041EE5
:1091700006DB2A4631460198FFF78FFF041E05DA09
:109180006442FBF723F904604FF0FF34204603B03C
:10919000BDE8704003B0704738B504460D46C9B10C
:1091A00010B90870002038BD0068FFF7F5FF0028EF
:1091B000F9DB04F11801284600F020F8A36823B970
:1091C000E38903F00F03032BECD10449284600F098
:1091D00015F8E7E76FF01500E5E700BFF1A000081C
:1091E00008B5054B0BB1FFF76FF8FFF7D9FABDE8EB
:1091F0000840F7F78BBD00BFC982000838B50546A7
:109200000C46FBF73BFB611E2B1811F8012F12B91E
:1092100028461A7038BD03F8012BF6E77BB972B9FE
:109220000029BEBF00204FF0004106E008BF002823
:109230001CBF6FF000414FF0FF3000F0D7B9ADF127
:10924000080C6DE904CE002909DB002B1ADB00F0C5
:109250006FF8DDF804E0DDE9022304B07047404216
:1092600061EB4101002B1BDB00F062F8DDF804E04C
:10927000DDE9022304B0404261EB4101524263EB5D
:1092800043037047524263EB430300F051F8DDF8AB
:1092900004E0DDE9022304B0404261EB4101704784
:1092A000524263EB430300F043F8DDF804E0DDE9EC
:1092B000022304B0524263EB4303704753B94AB9E7
:1092C000002908BF00281CBF4FF0FF314FF0FF30CE
:1092D00000F08CB9ADF1080C6DE904CE00F028F86F
:1092E000DDF804E0DDE9022304B07047FFECC29230
:1092F0009FED0B6B41EC170B9FED0B5B27EE066BA5
:10930000BCEEC66BB8EE464BA4EE457BFCEEC77BCD
:1093100016EE101A17EE900A704700BFAFF30080E8
:10932000000000000000F03D000000000000F041DF
:109330002DE9F047089D0E4604460F46002B4AD102
:1093400094468C45B2FA82F260D942B1C2F1200350
:10935000974020FA03F30CFA02FC1F4394404FEAB3
:109360001C4E1FFA8CF6B7FBFEF1230C0EFB117797
:1093700043EA074301FB06F098420AD91CEB0303BA
:1093800001F1FF3780F01581984240F212810239D5
:1093900063441B1AA4B2B3FBFEF00EFB103344EA85
:1093A000034400FB06F6A6420AD91CEB040400F1B4
:1093B000FF3380F00081A64240F2FD806444023811
:1093C00040EA0140A41B00211DB1D4400023C5E99F
:1093D0000043BDE8F0878B4205D90DB1C5E9000116
:1093E00000210846F5E7B3FA83F1002946D1B342DC
:1093F00002D3824200F2F580841A66EB0302012058
:109400001746002DE5D0C5E90047E2E7002A40F005
:109410009380A1EB0C034FEA1C471FFA8CFE01213D
:10942000B3FBF7F607FB1630230C43EA00430EFBB1
:1094300006F0984208D91CEB030306F1FF3802D26C
:10944000984200F2D08046461B1AA4B2B3FBF7F054
:1094500007FB103344EA03440EFB00FEA64508D97F
:109460001CEB040400F1FF3302D2A64500F2B680E3
:109470001846A4EB0E0440EA0640A5E7C1F1200718
:109480008B4022FA07FC4CEA030C06FA01FE20FA94
:1094900007F426FA07F344EA0E0400FA01F84FEA4B
:1094A0001C404FEA1449B3FBF0FE1FFA8CF600FB98
:1094B0001E3349EA03430EFB06F9994502FA01F20D
:1094C0000BD91CEB03030EF1FF3A80F08580994520
:1094D00040F28280AEF1020E6344A3EB0909A4B20C
:1094E000B9FBF0F300FB139944EA094403FB06F6C9
:1094F000A64208D91CEB040403F1FF3068D2A6424F
:1095000066D9023B644443EA0E40A41BA0FB02E67A
:10951000B4427346B14652D34FD05DB1B8EB0302AB
:1095200064EB090404FA07F722FA01F31F43CC4065
:10953000C5E9007400214CE7C2F1200120FA01F3D3
:109540000CFA02FC26FA01F1964033434FEA1C471D
:109550001FFA8CFEB1FBF7F007FB1016190C41EA5D
:10956000064100FB0EF68E4204FA02F408D91CEB09
:10957000010100F1FF382DD28E422BD9023861440F
:10958000891B9BB2B1FBF7F607FB161143EA0143B7
:1095900006FB0EF1994208D91CEB030306F1FF38D4
:1095A00014D2994212D9023E63445B1A46EA004142
:1095B00036E73946EDE6184602E7F045ADD2BEEB98
:1095C000020366EB0C060138B146A6E74646ECE717
:1095D000034698E74046D3E7D6467EE76444023820
:1095E00047E708460DE7023E63442DE7704700BF9A
:1095F0000720704710B54220094CFAF743FC4FF0A2
:1096000000634320C4F88034FAF73CFC4420FAF7A6
:1096100039FC0023C4F88034C4F8D83410BD00BF2E
:109620000040025808B5042000F0BAF9064B4FF488
:109630007A70DB68584300F0A7F900F0D7F9BDE86D
:10964000084000F0BDB900BFAC00002408B500F030
:10965000D5F900F0BDF9002000F0A2F90020BDE826
:10966000084000F091B9FFEC0F4BD3F8002442F012
:109670000102C3F80024D3F800245207FBD50022CE
:10968000C3F81024D3F8002422F0A85222F41022A8
:10969000C3F80024054AC3F82C24D3F8002422F48C
:1096A0008022C3F800247047004002580000FF01E8
:1096B00008B54FF0006000F038FA4FF00160BDE8E7
:1096C000084000F032BA08B500F0C2FB4FF000606D
:1096D00000F018FA4FF00160BDE8084000F012BA3F
:1096E00000F0D2BA4FF0E023C3F8080D70470F28FE
:1096F0008CBF0020012040047047431E0E2B10B584
:10970000044609D821B12046BDE8104000F04ABA0D
:1097100000F032FA0028F6D110BD00F1006000F52B
:10972000003000F0B1BB830705D100F1006000F507
:10973000003000F0EBBB0020704700207047FFECCA
:10974000014B1868704700BF0010005C224BF0B559
:109750001A68224BC2F30B06120C1F885D68BE42CA
:109760001C7A2BD09F89BE4205D101240C2505FB14
:1097700004335D681C7A41F203039A4220D042F21E
:1097800001039A421ED042F203039A421CD041F2D6
:1097900001039A4208BF5A24421E013D0B460A4467
:1097A000934217D215F8016F581C7EB92C258242BE
:1097B0001D7001D9981C5C70401AF0BD0024D5E7DB
:1097C0005924E9E75824E7E75624E5E7034600F87B
:1097D000016CE5E71846EFE70010005CBC000024D0
:1097E00000F1FF5000F58F10D0F800087047FFEC33
:1097F000012802D0022804D0704700210248FAF75D
:109800002DBB00210148FAE7430904004409040084
:109810000128014602D0022803D070470248FAF717
:109820001DBB01210148FAE7430904004409040073
:10983000012808B502D002280BD008BD0948FAF764
:109840000DFC80F001010748C9B2BDE80840FAF7F5
:1098500005BB0548FAF702FC80F001010248C9B2D5
:10986000F3E700BF4309040044090400D0E90032D3
:1098700083F308881047FEE74FF0E0224FF40030F2
:1098800070B5D2F8883D344D43F47003C2F8883D7A
:10989000324B334AD3F8803803F57F1303F57E53F8
:1098A0009B029360FAF7EEFA2E48FAF7EBFA2E488D
:1098B000FAF7E8FA0120F6F7FDFE00202C6DF6F726
:1098C000F9FE2A4B9C4242D100240120F6F7F2FE19
:1098D000264620462C65F6F7EDFE254800F016FBDF
:1098E0000546244800F012FB234B98420ED125F088
:1098F000FF02224B9A4209D1EDB21E2D06D84FF439
:109900007A7300265D43AC4238BF2C464220FAF7FA
:10991000A5FB054660B95EB1FBF794FE0120F6F7A2
:10992000C9FE0D4B114A2C4628461A65F6F7C2FEB1
:1099300001211348FBF709FE02211248FBF705FE3F
:1099400020460024FBF7CEFEFBF77CFEF8E741F251
:1099500088340126C1E700BF0040005800E0F11F35
:10996000AC000024430904004409040007B007B018
:10997000A0010208A40102085D7D05C500ECC292A9
:10998000F3A0000804A10008044B1B6858434FF0E3
:10999000E02320F07F405861704700BFD4000024CE
:1099A000021E054B054814BF0121082102F00402E4
:1099B00019600421F6F79CBED400002410E000E0FA
:1099C000012200210148F6F793BE00BF10E000E03D
:1099D00000220121044808B5F6F78AFE4FF0E02383
:1099E00000229A6108BD00BF10E000E002220021C1
:1099F0000148F6F77DBE00BF10E000E00022022122
:109A00000148F6F775BE00BF10E000E0042838B545
:109A100005460C4613D80120F6F70AFE032D094B24
:109A20004FF000000CBF24F0FF01002153F8253057
:109A3000054A0B431365F6F7FBFD002038BD4FF0D8
:109A4000FF30FBE76CA500080040005801280446E1
:109A500008B502D10021FFF7D9FF2046F7F74DF9ED
:109A600000F0E2F9436803F110010A68D207FCD460
:109A7000DA68D20705D5034A5A6002F18832436892
:109A80005A6070472301674502460A48836893423B
:109A900003D803F5801393420AD80748816891429E
:109AA00005D801F58011914298BF00207047002031
:109AB000704700BFEC000024D800002410B40C460E
:109AC000406811461A4620445DF8044BF6F710BE74
:109AD000012300220C21FFF7F1BFFFEC38B505464A
:109AE000BFF34F8F064C6B68186910F0070006D063
:109AF0000120F6F712FE013CF5D16FF00F0038BDE2
:109B0000404B4C0038B5FFF7BFFF054650B1FEF79C
:109B1000BDFC041E04DB2846FFF7A4FFFEF7CCFCC7
:109B2000204638BD6FF01204FAE738B5FFF7ACFFF6
:109B3000054658B1FEF7AAFC041E05DB2846FFF7D0
:109B4000C7FF2846FEF7B8FC204638BD6FF0120468
:109B5000FAE7B0F5803F10B504460AD200F5800060
:109B60004001FFF791FF03698068E41A00EB44109D
:109B700010BD4FF0FF30FBE7B0F5803F08B50DD2C8
:109B8000FFF7E7FF002300F1200201780130FF29F1
:109B900018BF01338242F8D1184608BD6FF00D009E
:109BA000FBE7FFECF8B50F2800F5806604464FEAA6
:109BB000464661D83046FFF767FF0546FEF766FC6C
:109BC000002852DB2846FFF789FF0746002850D1BE
:109BD0002846FFF747FF04233A460C21FFF76EFFA4
:109BE000EB684FF470620C21E31A28461B0203F461
:109BF000E063FFF763FF80233A460C212846FFF716
:109C00005DFF2846FFF76AFF044678BB034604223F
:109C10000C212846FFF752FF23464FF470620C21B7
:109C20002846FFF74BFF2846FFF752FF2846FEF76E
:109C300043FC24BB3046FFF727FF00B306F5FF3097
:109C400000F2FF10FFF720FFC8B10423043E0D4AC5
:109C5000F1580433013118BF01349342F8D1002C7C
:109C60000CBF4FF400306FF00400F8BD6FF0040437
:109C7000D9E76FF00404D9E76FF00D00F5E76FF056
:109C80000400F2E7040002002DE9F84F06460F46F3
:109C90001546FFF7F9FE0446002800F0C2808368ED
:109CA000B34200F2BE80AA1903F580139A4200F273
:109CB000B880FEF7EBFB002865DB2046FFF70EFFC0
:109CC0008046002840F0AA8020462037FFF7CAFED1
:109CD000302325F01F0B0C211A46B946FFF7EEFE84
:109CE000B3444246B04602230C212046FFF7E6FE6D
:109CF000D84532D0BFF34F8FBFF36F8F59F8203C58
:109D0000C8F8003059F81C3CC8F8043059F8183C21
:109D1000C8F8083059F8143CC8F80C3059F8103C11
:109D2000C8F8103059F80C3CC8F8143059F8083C01
:109D3000C8F8183059F8043CC8F81C30BFF34F8FEE
:109D4000BFF36F8F2046FFF7C9FE08BB636809F1B8
:109D500020091B6913F0C06F17D0002302220C21C9
:109D60002046FFF7ABFE4FF0FF33002214212046C0
:109D7000FFF7A4FE2046FFF7ABFE002D41D12046A1
:109D8000FEF79AFB2846BDE8F88F08F12008AFE7F8
:109D90006FF00405EEE74FF0FF3300221421204658
:109DA000FFF78CFE326857F8203C9A4233D1726834
:109DB00057F81C3C9A422ED1B26857F8183C9A4288
:109DC00029D1F26857F8143C9A4224D1326957F8E5
:109DD000103C9A421FD1726957F80C3C9A421AD132
:109DE000B26957F8083C9A4215D1F26957F8043C19
:109DF0009A4210D1636820371B6913F0C06F0AD1F3
:109E000020365E45C7D14FF0FF3300221421204693
:109E1000FFF754FEB3E76FF00405F4E76FF00405B5
:109E2000ADE76FF00D00AEE74FF0E021054BD1F844
:109E30000C2D02F4E0621343C1F80C3DBFF34F8FC9
:109E4000FEE700BF0400FA052822FF21F6F70DBF48
:109E500010B5054C2046FFF7F7FF04F12800FFF787
:109E6000F3FF024B636010BDE814002400000208F9
:109E700000F10801202208B54068FFF731FC2028D6
:109E800008BF002008BDFFEC1E4A20F01F0310B5DC
:109E900054689C420ED0D46AA3420DD101235B4288
:109EA00003F028031344C0F382044BB934B10024F7
:109EB000204610BD0023F2E70023F4E7124BD062E6
:109EC000A01C934243F820101AD1CCB91A68072A73
:109ED00016D19A6A01320BD003F128042046FFF70D
:109EE000C7FF28B120464FF0FF34FFF7ADFFDFE793
:109EF0000448FFF7BDFF04460248FFF7A5FFD7E778
:109F00001C60D4E7E81400241015002438B5144B65
:109F100020F01F020568596891421AD0D96A8A4216
:109F200015D10122C0F382000A24514204FB02022F
:109F300011F0280102F1020253F8225007D007283D
:109F400005D15C182046FFF793FF20B1ED4328466A
:109F500038BD0022E6E72046FFF776FFF7E700BFAF
:109F6000E81400242618002461726D76372D6D2FB9
:109F700061726D5F686172646661756C742E6300F6
:109F8000626F6F746C6F616465725F6D61696E00A2
:109F90004170704272696E675570006972712F6905
:109FA00072715F756E6578706563746564697372EC
:109FB0002E6300736572636F6E3A3A204552524FBA
:109FC000523A20416C726561647920636F6E6E65F0
:109FD000637465640A00736572636F6E3A2052653C
:109FE000676973746572696E67204344432F414308
:109FF0004D2073657269616C206472697665720ABE
:10A0000000736572636F6E3A204552524F523A2088
:10A010004661696C656420746F2063726561746564
:10A0200020746865204344432F41434D207365727B
:10A0300069616C206465766963653A2025640A006D
:10A04000736572636F6E3A205375636365737366ED
:10A05000756C6C79207265676973746572656420CC
:10A06000746865204344432F41434D2073657269F2
:10A07000616C206472697665720A002F6465762FC0
:10A08000747479537800556D656D00696E66006E65
:10A09000616E00505834424C76312E31372E306785
:10A0A00032353534356262383739002C002F64651B
:10A0B000762F7474795330002F6465762F6E756C2B
:10A0C0006C002F6465762F74747941434D256400CC
:10A0D0004D6174656B004D6174656B204837343396
:10A0E0002D736C696D0042756C6B0025732F2573A1
:10A0F000002F002F6465762F74747953302C353718
:10A10000363030002F6465762F74747941434D30BA
:10A110000053544D33323F3F3F3F3F3F3F00535486
:10A120004D333248375B347C355D780049646C656B
:10A13000205461736B00FFEC000000000000000081
:10A14000CC04002401000000D80400240500000015
:10A15000D804002405000000AC0400240000000026
:10A16000C404002401000000BC040024000000001E
:10A17000B4040024000000003C6E6F6E616D653E0B
:10A1800000FFECC201000000A51900080200000059
:10A19000A519000803000000A51900080601000029
:10A1A000891900080700000089190008080100004B
:10A1B000871900080A000000A5190008090100001D
:10A1C000A51900080B000000A51900080C000000EC
:10A1D000A51900080D000000A519000800000024C2
:10A1E000000000000000000000000000000000006F
:10A1F00000000000000000000000000045280008EA
:10A20000D5280008D9270008BD2700082D270008F9
:10A21000812600089B260008D5260008E1260008B4
:10A22000E92600082127000821270008FD2A000848
:10A23000732B0008AD2B0008252C0008BD2B00084F
:10A24000C92B000800000000AD2A0008952D000869
:10A250000B2C0008052C00086D3000086B2D000841
:10A260008132000800000258000402580008025819
:10A27000000C02580010025800000000000000000E
:10A28000001C025800000000000000003200000026
:10A29000010000004B000000020000006E00000002
:10A2A000030000008600000004000000960000008B
:10A2B00005000000C8000000060000002C0100009E
:10A2C000070000005802000008000000B004000071
:10A2D00009000000080700000A00000060090000F3
:10A2E0000B000000C01200000C00000080250000E0
:10A2F0000D000000004B00000E0000000096000062
:10A300000F00000000E100000110000000C2010089
:10A310000210000000840300031000000008070082
:10A320000410000020A107000510000000CA08006A
:10A330000610000000100E000710000040420F0041
:10A3400008100000009411000910000060E31600DE
:10A350000A10000080841E000B100000A0252600BB
:10A360000C100000C0C62D000D100000E067350085
:10A370000E10000000093D000F100000286E756CE3
:10A380006C2900FFECC2925D0080E03779C3314355
:10A3900000003426F56BFC420000901EC4BCC6428F
:10A3A000000040E59C309242000000A2941A5D42F9
:10A3B000000000E876482742000000205FA0F2413C
:10A3C0000000000065CDBD410000000084D787413A
:10A3D00000000000D01253410000000080841E41A4
:10A3E00000000000006AE840000000000088B34060
:10A3F0000000000000407F400000000000004940D5
:10A4000000000000000014409A9999999999B93F69
:10A410007B14AE47E17A843F2D431CEBE2361A3FB2
:10A420003A8C30E28E79453EBC89D897B2D29C3CBA
:10A4300033A7A8D523F649393DA7F444FD0FA5322B
:10A440009D978CCF08BA5B25436FAC642806C80A79
:10A4500000000000000024400000000000005940FF
:10A46000000000000088C3400000000084D797412E
:10A470000080E03779C34143176E05B5B5B8934600
:10A48000F5F93FE9034F384D321D30F94877825ACC
:10A490003CBF737FDD4F1575050000000000000014
:10A4A00000000000635E0008675E00080000000016
:10A4B000000000006B5E000800000000B1600008B2
:10A4C00055670008715F0008516200080000000035
:10A4D0000D65000885610008000000001F69000884
:10A4E0003169000833690008357300088B6900087A
:10A4F000000000004571000800000000000000009E
:10A50000D77200080000000037690008956C000849
:10A51000D16B00088D6E0008896B00088369000804
:10A5200073690008120100020200004062314B0012
:10A53000010101020301FFEC7D7600087D76000831
:10A54000000000006D76000800000000798000081F
:10A55000177F0008597E0008000000005B7F00089C
:10A560003D7E000800000000000000000000000028
:10A5700007B007B0020007B0000008B0263A09B0E3
:10A58000B0EDFF7F010000000000000000000000AF
:10A5900000000000000000000000000000000000BB
:10A5A00000000000000000000000000000002C017E
:10A5B000440A00240000000000005802700B002430
:10A5C000FCA10008000000240000000000000000C2
:10A5D0000000000000000000000000000003000870
:10A5E0000000000000C2010035000000000E270737
:10A5F00000100140097C09000A7C0900FFFFFFFFF1
:10A60000FFFFFFFF8000002438A5000801000000C4
:10A61000FFFFFFFF0000000000000000000000003E
:10A6200000000000010000004CA500080000000030
:10A6300000000000D95900000000000000000000E8
:10A64000E00100000000000011A100083F00000030
:10A65000500400001EA100083F000000010000009F
:10A660000100000000210052000010080800000056
:10A6700000800000010000000020005200000008DF
:08A680000000000000000000D2
:0400000508000000EF
:020000040802F0
:100000007AC5002405030208A9020208A902020811
:10001000A9020208A9020208A9020208A90202080C
:10002000A9020208A9020208A9020208A9020208FC
:10003000A9020208A9020208A9020208A9020208EC
:10004000A9020208A9020208A9020208A9020208DC
:10029000A9020208A90202080000000000000000F4
:1002A000FFECC2925D7D05C5EFF305801EF0040FE3
:1002B00002D0EFF309818D466A4602F16802EFF33E
:1002C00011831EF0100F0CBF2DED108A90B02DE998
:1002D000FC4F6946DFF828D000F068FFB0E8FC4F1B
:1002E0001EF0100F0CBFB0EC108A40301EF0040F4F
:1002F0000CBF80F3088880F3098883F31188704766
:100300000012002408B501F005F81E4B1E48DA1C47
:10031000C11E121A22F00302994288BF0022002156
:1003200001F0A1FC194B1A48DA1CC11E121A22F066
:100330000302994288BF0022164901F029FB00F010
:1003400021F900F04BFF00F08DF9BFF34F8FBFF3A1
:100350006F8F4FF0E023D3F8902F22F00102C3F803
:10036000902F0522C3F8942FBFF34F8FBFF36F8FE9
:1003700031F162FE00F05EFE00F070FE00F026FD3E
:1003800002F0D8FC8CC20024000F0024D80E0024F8
:1003900000000024640A1C08734A82B0D2F80034BA
:1003A00023F4802343F48033C2F800346F4B01936D
:1003B000019B002B03DDD2F800349B0304D5019B85
:1003C000002B04DC02B07047019B013BEFE7664B5A
:1003D000D3F8182422F4706222F00F0242F00802CF
:1003E000C3F81824D3F81C2422F4E06242F040023F
:1003F000C3F81C24D3F81C2422F4E06242F4806287
:10040000C3F81C24D3F8182422F0700242F04002F2
:10041000C3F81824D3F8202422F0700242F04002DE
:10042000C3F82024D3F8102422F47C5242F4006252
:10043000C3F810244E4AC3F828244E4AC3F8302487
:100440004D4AC3F8382402F50032C3F840244B4A21
:10045000C3F82C24D3F8002442F0A852C3F8002497
:10046000D3F800249001FBD5D3F800241101FBD56B
:100470003D4BD3F800249200FBD5D3F80C2842F072
:100480000602C3F80C28D3F8182842F44042C3F8F7
:100490001828D3F818289004FBD5334BD3F8042838
:1004A0009104FBD5D3F8F4244FF0B04142F002029E
:1004B000C3F8F424D1F82C2442F00102C1F82C2412
:1004C000D3F818289204FBD52D4A22211160D3F8C5
:1004D000102422F0070242F00302C3F81024224B3A
:1004E000D3F8102402F03802182AF9D1D3F8542492
:1004F00022F4405242F40052C3F85424D3F8582452
:1005000022F4407242F40072C3F85824D3F8502405
:1005100022F4E04242F48052C3F85024D3F850242D
:1005200022F4E02242F48032C3F85024D3F8582455
:1005300022F0E04242F08052C3F85824D3F8542409
:1005400022F4401242F40012C3F85424D3F8582481
:1005500022F44032C3F85824D3F8502422F04052F9
:10056000C3F850242EE700BF00400258F82F910036
:1005700012202000770203072F0201018808BF0024
:100580000020005210B52F4C00200122D4F8003476
:1005900043F00103C4F800342B4BC3F80821C4F81E
:1005A00010042A4BD4F80024134043F01003C4F87D
:1005B0000034274BC4F82C34D4F8003423F48023BF
:1005C000C4F80034C4F8600400F096FCFFF7E4FEC1
:1005D000D4F8D83443F0006343F02303C4F8D8348C
:1005E000D4F8DC34C4F8DC34D4F8D43443F48033A5
:1005F000C4F8D434D4F8E03443F0895343F09F0373
:10060000C4F8E034D4F8E83443F4C10343F480433D
:10061000C4F8E834D4F8EC34C4F8EC34D4F8F0344A
:1006200043F4405343F03003C4F8F034D4F8E434D6
:10063000C4F8E434D4F8F43443F00203C4F8F434D6
:1006400010BD00BF004002580080005167EFFEEA75
:100650000000FF01024BDA691206FCD59862704770
:100660000010014010220021144808B500F08EFC53
:10067000134800F079FE134800F076FE124B5A68DA
:1006800022F4FE4222F070021204120C5A601A6820
:1006900022F04F4222F47F0222F47F4222F0FC0239
:1006A0001A600A4A99680A409A6040F62302DA60A2
:1006B0001A6842F00D021A6008BD00BFF0440258EB
:1006C000097C09000A7C0900001001400000F1FFCC
:1006D00010B5D0F88C4001F4D873A0F874102268DB
:1006E00022F4D87213432360D0F88C20936861F30E
:1006F0000003936010BD10B5EFF311840023802236
:10070000EFF3108372B682F3118883F31088FFF73A
:10071000DFFFE4B284F3118810BD10B5EFF311844C
:1007200000238022EFF3108372B682F3118883F3E3
:10073000108849B1D0F88C201368926803F4D873FC
:1007400002F0010213430B800021E4B2FFF7C0FF67
:1007500084F3118810BDFFECF0B5036EEFF3118048
:1007600000228021EFF3108272B681F3118882F3A8
:100770001088D3F88C20156825F0010105F00104DC
:100780001160D3F88060D3F88870720802EB4702DA
:10079000B2FBF6F2642A41D9013225F40041520835
:1007A00021F00101D3F88C502960D3F88C50EA6015
:1007B000264A0A4093F87A10012939D142F4C062DE
:1007C00093F87B50092D02D0082D36D1A9B342F4FD
:1007D0008052D3F88C100A60D3F88C6093F87C10A8
:1007E0007568494225F4405501F400512943716070
:1007F000D3F88C5093F87E60A96821F4407126B13B
:10080000D3F89C600EB141F40071A9602243D3F883
:100810008C30C0B21A6080F31188F0BDC2F342057B
:1008200022F00F0241F400411204120C2A43B9E7EE
:10083000022908BF42F48062C2E7B3F87A10B1F52A
:10084000E06F08BF42F08052C3E700BFFEE9FFEF50
:10085000036ED3F88C20506AB3F8762040EA024247
:10086000C0B20A600022A3F87620704710B5006E6F
:10087000EFF3118400238022EFF3108372B682F32A
:10088000118883F31088B0F8743039B143F0200137
:10089000E4B2FFF730FF84F3118810BD23F49071A8
:1008A00021F00101F4E7036ED3F88C30D869C0F36E
:1008B00040107047036ED3F88C309962704710B5C2
:1008C000006EEFF3118400238022EFF3108372B6E1
:1008D00082F3118883F31088B0F8743041B143EA91
:1008E000020189B2E4B2FFF706FF84F3118810BD5C
:1008F00023F08001F5E7036ED3F88C30D869C0F39C
:10090000C010704708B5036E114693F87D2022B1E0
:10091000D3F8980008B100F013FD002008BDF8B529
:100920000346B1F5887F10469B685D692C6E00F028
:10093000288110DCB1F5817F00F0CC8040F20F13EC
:10094000994200F0FC8040F20113994200F09F8030
:100950006FF018007FE040F23313994253D040F219
:100960003513994278D0B1F5987FF1D1EFF3118624
:1009700000238022EFF3108372B682F3118883F391
:100980001088D4F88C3010F0010F1F6827F0010296
:100990001A60D4F88C30D4F890209D682AD000F0EA
:1009A000060180F0080045F00805A1F1020CA1F154
:1009B000040EC0F3C000DCF1000343EB0C03DEF1D6
:1009C00000014FEA034341EB0E0143EA402322F4C6
:1009D000403043EA414320F40070184300F0C4FC67
:1009E000D4F88C309D60D4F88C301F60F6B286F35A
:1009F00011882FE022F4403025F0080520F4007023
:100A000000F0B2FCECE7EFF3118200238021EFF35A
:100A1000108372B681F3118883F31088D4F88C3078
:100A2000C607196821F001051D60D4F88C506B6869
:100A30004CBF43F4803323F4803380074CBF43F42E
:100A4000003323F400336B60D2B2D4F88C301960D9
:100A500082F311880020F8BDEFF31182002380217A
:100A6000EFF3108372B681F3118883F31088D4F802
:100A70008C300128196821F001051D60D4F88C50D4
:100A80006B680CBF43F4004323F40043DBE7002A08
:100A900000F0918094F87A20D2B1511E4A424A4126
:100AA00051024FF4807294F87C3094F87E509B0190
:100AB00043EA45730B43134394F87D2043EAC27322
:100AC00043F030038360D4F8801001F03BF9C1E7B4
:100AD0001146E8E7002A6ED0936803F03002302A0E
:100AE00069D19A0003D5D4F89C20002A63D0002B4A
:100AF00003DAD4F89820002A5DD013F480721CD059
:100B000013F4007F0CBF0223012384F87A3083683A
:100B1000C3F3801384F87C308368C3F3407384F894
:100B20007E308368DB0F84F87D3001F027F9C4F84C
:100B300080002846FFF710FE8CE71346E5E7EFF349
:100B4000118600238022EFF3108372B682F311889E
:100B500083F31088B4F87430284600216FEA4343C9
:100B60006FEA5343A4F87430FFF7A9FED4F890005D
:100B700020F4402020F4807040F4802000F0F4FB4A
:100B800034E7EFF3118600238022EFF3108372B66F
:100B900082F3118883F31088D4F8900000F0E4FB0E
:100BA000B4F8743001212846C3F30E03A4F874305E
:100BB000FFF785FE1AE76FF015004CE710B5046EDD
:100BC00094F8840000F02EFD002294F88400114671
:100BD000BDE8104002F066B938B5056E06492A46F0
:100BE00095F8840002F05EF9044618B995F884007F
:100BF00000F02CFD204638BDFD0B020810B5144650
:100C0000D2F88C20D3699BB29806A4F8763013D51D
:100C1000B4F8741089060FD5204601F0EFFDB4F842
:100C200076301A0606D5B4F874301B0602D5204675
:100C300001F0AEFD002010BD13F00E0FEFD00E231B
:100C40001362ECE7036E0A461E49D3F88C308B42E0
:100C500020D00CD8A1F540518B421FD001F5806106
:100C60008B421FD0A1F500618B421FD070471649FF
:100C70008B421FD001F580618B421ED0A1F5184137
:100C80008B421DD111484FF000410AB10A460021A4
:100C900000F07CB90D484FF08041F6E70B484FF467
:100CA0008021F2E709484FF40021EEE707484FF4AE
:100CB0000031EAE706481021E7E705482021E4E78C
:100CC000704700BF0078004000100140E84402581F
:100CD000F044025870B50026046E054631462046A1
:100CE00084F87860FFF719FD31462846FFF7AAFF20
:100CF000D4F88C20136823F00D031360D4F890000F
:100D000000F01AFCD4F8940000F016FCD4F89C0013
:100D100008B100F011FCD4F8980018B1BDE870409B
:100D200000F00ABC70BDFFEC38B5046E0022012152
:100D30000546D4F88C301A60FFF784FFD4F8900091
:100D400000F012FBD4F8940000F00EFBD4F89C00E5
:100D500008B100F009FBD4F8980028B120F4402035
:100D600040F4802000F000FBD4F88C10284694F862
:100D70007C304A685B4222F47D5203F400531343F3
:100D80004B60D4F88C20104B11680B401360D4F8E2
:100D90008C2094F87910936823F4E06323F0010326
:100DA00043EA41639360FFF7D7FCD4F88C2000201E
:100DB000136843F0005343F00D0313600123A4F8BC
:100DC000740084F8783038BD03BEFF3338B5084D61
:100DD000002455F8040B10B10021FFF79EFC0134EC
:100DE000082CF6D10348BDE83840FFF79DBF00BF8F
:100DF000E0771708C00300247FB50D490D4801F0C6
:100E000001FB0D4968460D4D00F075FF00231C469F
:100E100055F8041B39B15E1C303368468DF8093033
:100E200001F0F0FA33460134082CF1D104B070BD62
:100E3000C00300244432160851321608E077170820
:100E400013B504460DF106010948FFF766FC0A2CAC
:100E500002D10D20FFF7FEFBE0B2FFF7FBFBBDF870
:100E600006100348FFF747FC204602B010BD00BF44
:100E7000C003002430B4EFF3118400238022EFF389
:100E8000108372B682F3118883F31088BFF34F8FFB
:100E9000174B1849D3F800280B8802F4807578B1F5
:100EA00001339BB20B8075B1CBB10023BFF34F8FE1
:100EB000E4B284F31188C3B1042030BC00F07CB8E4
:100EC0005BB1013BEDE70B88002BEED0084B42F401
:100ED0008072C3F800280123E8E7002DE5D022F452
:100EE0008072034BC3F80028DFE730BC704700BFB7
:100EF000004002586C4B0024EFF311820023802144
:100F0000EFF3108372B681F3118883F310880749D9
:100F1000D1F8003823F48073C1F800380021044B65
:100F20001980D3B283F31188FFF7A4BF00400258A1
:100F30006C4B002470B50446EFF31185002380222A
:100F4000EFF3108372B682F3118883F310880E4A90
:100F5000D2F8083860B143F001034FF47A740A4EB6
:100F6000C2F80838013C06D2EDB285F3118870BD95
:100F700023F00103F3E7D6F80838DB07F4D40120A7
:100F800000F01AF8EEE700BF0040025830B5EFF36A
:100F9000118400238025EFF3108372B685F3118846
:100FA00083F31088036823EA0101E3B20A43026075
:100FB00083F3118830BDFFEC82B000221C49B0F5EC
:100FC0007A7F0BD8002242F22A51642811D80022DD
:100FD0000A2818D8002208BB02B070470192019B72
:100FE0008B4202DDA0F57A70E9E7019B01330193A2
:100FF000F5E70192019B8B4201DD6438E5E7019B37
:1010000001330193F6E70192019BB3F56E7F01DB9B
:101010000A38DDE7019B01330193F5E70192019B5B
:101020005E2B01DD0138D6E7019B01330193F6E722
:10103000AD730100BFF34F8FBFF36F8F4FF0E0230D
:101040000022C3F8502FD3F8142D42F40032C3F815
:10105000142DBFF34F8FBFF36F8F70474FF0E02217
:10106000F0B5D2F8803D03F00704C3F34E31C3F36B
:10107000C9030434B3FA83F505F01F05BFF34F8F9E
:10108000184601FA04F700FA05F6013846EA0706A1
:10109000C2F8606FF7D20139F2D2BFF34F8FD2F8A6
:1010A000143D43F48033C2F8143DBFF34F8FBFF3B8
:1010B0006F8FF0BD4FF0E02210B5D2F8843D43F0C1
:1010C0000104C2F8844DD2F8804DC2F8843D01235A
:1010D00004F007040434A340BFF34F8F5C1E0442A6
:1010E00004D05C422040C2F8700F18444FF0E02456
:1010F000C2188A420AD9884203D24FF0E023C3F8CB
:10110000700FBFF34F8FBFF36F8F10BDC4F85C0F2C
:101110001046EDE7F0B54FF0E026D6F8803D03F03D
:101120000700C3F34E32C3F3C9030430B3FA83F4A8
:1011300004F01F04BFF34F8F194602FA00F701FABB
:1011400004F5013945EA0705C6F86C5FF7D2013AA4
:10115000F2D2BFF34F8FBFF36F8FF0BDF0B44FF0FB
:10116000E0260F1A0124D6F8802D02F00705C2F3FD
:101170004E33C2F3C90204350133AB40AC4002FB2D
:1011800003339F4202D3F0BCFFF7C4BF6342184051
:10119000BFF34F8FC6F8680F20448142FAD8BFF3DF
:1011A0004F8FBFF36F8FF0BC7047FFEC70B50A4DE7
:1011B00006460C462B680BB91C462960304600F0E9
:1011C000B5FA2968304601F095FE14B900232C6861
:1011D0002B60204670BD00BF704B0024EFF31483DA
:1011E00043F0040383F314884FF0E023D3F8342F43
:1011F00022F04042C3F8342FD3F8882D42F4700215
:10120000C3F8882D7047FFEC024B1878421C1A7007
:10121000704700BF6E4B0024202810B50CD9062360
:101220000121202B0AD001FA03F25C1C824201D377
:10123000D8B210BD2346F4E70520FAE71846F8E7D0
:10124000072A1CD901231F2A03FA02F3A2F1030281
:1012500003F1FF3300EA030094BFDB106FF060433B
:10126000014420EA0300194421EA030120FA02F3B1
:10127000D140044A505C044AD35C184370470020B4
:10128000704700BF3D7817083478170840B100292F
:10129000C2F1000214BF0320012002F00402104337
:1012A0004FF0E023C3F8940D70472DE9F0478046D6
:1012B0004FF0FF3A1446FFF7A7FF08EB010628F0AE
:1012C0001F0705468946F01BFFF7A6FF0AFA00FA3A
:1012D0000AEA070A4FF0E027A6EB0A00FFF79CFF97
:1012E000C7F8985D45EA0A0506460246494645F0B4
:1012F00010054046013EC7F89C5DFFF7A1FF0002C4
:1013000044EA460480B2044344F00104C7F8A04D07
:10131000BDE8F0874FF0E0230022D3F8900D11468E
:10132000C0F30720904202DCC3F8941D7047C3F855
:10133000982D0132C3F8A01DC3F89C1DF2E7FFEC05
:1013400003060BD4C0F30312064B53F822202AB134
:1013500000F00F00012311B18340936170471030FA
:10136000FAE700BF487817082DE9F04710F080062B
:101370000446C0F3031840F0D9806E4B53F8285050
:10138000002D00F0D38000F4402300F00F07B3F5E8
:10139000002F00F0B780B3F5402F00F0B580B3F513
:1013A000802F40F0B380C0F30021FFF7C9FF012177
:1013B000EFF3118200238020EFF3108372B680F3E5
:1013C000118883F31088022940F0A28014F4704F32
:1013D000C4F3033E14D023074FF00F094BBFA7F10E
:1013E00008033B46242020209B0050F805C009FA42
:1013F00003F90EFA03F32CEA090C43EA0C034351F8
:101400004FEA470C0323D5F80090032903FA0CF3A5
:1014100029EA03096FEA030001FA0CF343EA09031E
:101420002B6078D004F44033B3F5803F75D0A3F53A
:101430000039D9F1000343EB09035B00D5F80C90A8
:1014400003FA0CF300EA090943EA0903EB60BEF171
:10145000000F13D123074FF00F0A4BBFA7F108036A
:101460003B464FF0240E4FF0200E9B005EF8059097
:101470000AFA03F329EA03034EF8053001F1FF3EAF
:10148000BEF1010F0DD804F44066B6F5006F46D0EA
:10149000B6F5406F45D0A6F58069D9F1000646EB58
:1014A0000906AB6806FA0CF6BEF1010F00EA03006C
:1014B00046EA00064FF00100AE6000FA07F06B68E4
:1014C00031D8A6052FD5034301296B6014D0E3055D
:1014D00012D504F00C04BF000F2104F1B04407F052
:1014E0000C07D4F80834B94008FA07F823EA0103D6
:1014F00048EA0303C4F80834D2B282F3118800200A
:10150000BDE8F087022153E7032151E731464FE759
:101510004FF0000E74E7002390E701238EE70226C8
:10152000BFE70326BDE723EA0003CDE76FF0150010
:10153000E6E700BF48781708C0B2FFF715BFFFEC19
:101540000206034610D4C0F30311084A52F82100E2
:1015500058B1012203F00F03016902FA03F30B42B1
:1015600014BF1046002070470020704748781708C5
:101570000F2810B52DDDA0F110041F2C08DC03F19D
:10158000604303F561430B600123A340136009E04E
:101590003F2C09DC1D4C30381C440C60012303FA3D
:1015A00000F01060002010BD5F2C04DC184C503897
:1015B0001C440C60F2E77F2C04DC164C70381C4491
:1015C0000C60EBE7952C1EDC134C90381C440C602F
:1015D000E4E7124B04380B600B2814D8DFE800F066
:1015E00006090C13131313131313130F4FF4803343
:1015F000CCE74FF40033C9E74FF48023C6E7084B2C
:101600000B600123C2E74FF0FF30CCE704E100E0BC
:1016100008E100E00CE100E010E100E024ED00E072
:1016200010E000E013B5802301AA69460446FFF7E5
:101630009FFF20B90F2CDDE9003102DD196002B0F7
:1016400010BD1A6822EA01021A60F8E713B50023F8
:1016500001AA69460446FFF78BFF20B90F2CDDE98C
:10166000003102DD196002B010BD1A680A431A6029
:10167000F9E7FFEC4FF0E02325494FF0FF3010B5BC
:101680005B6803F00F035A1C03F1382361339B009E
:1016900041F8040B9942FBD14FF0E0231D49C3F8F8
:1016A000081D4FF08031C3F8181DC3F81C1DC3F886
:1016B000201D5301184A03F1604303F5644342F8C7
:1016C000041B9342FBD10024144B15490B202246E6
:1016D0001C6001F0E7FB22461249032001F0E2FB07
:1016E0004FF0E02210490420D2F81C3D23F07F4344
:1016F00043F0E043C2F81C3D224601F0D3FB042036
:10170000FFF7A4FFF02383F3118862B610BD00BF7A
:1017100080E100E00000020800E400E0704B0024DB
:101720003519020831170208351802087047FFEC16
:101730002DE9FF414FF0E02305460E461746D3F84A
:101740002C4DD3F8288D63000FD5304A0020304946
:1017500000F0EAFA5FFA88F33BB13A463146284690
:1017600004B0BDE8F04100F065B8284A00202949DE
:1017700000F0DAFA2B46254A00202749009600F0AF
:10178000D3FAEFF31183EFF31082EFF30581EFF358
:101790001480D2B2DBB200921C4ACDE901101F497D
:1017A000002000F0C1FA4FF0E0230020D3F8302DE4
:1017B000D3F8381DD3F83C3DCDE90042CDE9021302
:1017C000124A4346164900F0AFFA00200F4A154965
:1017D00000F0AAFA14F0020013D00C4A00201249BB
:1017E00000F0A2FAEFF3118300238022EFF31083BD
:1017F00072B682F3118883F31088AD210B4800F094
:10180000CFF9002CEEDA014A0949E9E768781708B0
:101810005C3216087832160892321608A932160879
:10182000E4321608213316083933160871331608C6
:101830005F331608F0B54FF0E02585B006460F4639
:10184000304A00203049D5F8284D00F06DFA334673
:101850002C4A2E490020009700F066FAD5F8283D62
:10186000D5F8342D00202A490092264A00F05CFA6F
:10187000EFF31183EFF31082EFF30581EFF31480A0
:10188000D2B2DBB200921F4ACDE9011021490020FB
:1018900000F04AFA1B4A2049002000F045FAE5070B
:1018A00004D5184A00201D4900F03EFAA00704D5CF
:1018B000144A00201A4900F037FA210704D5114ACA
:1018C0000020184900F030FAE20604D50D4A002045
:1018D000154900F029FAA30604D50A4A0020134945
:1018E00000F022FAEFF3118300238022EFF310833C
:1018F00072B682F3118883F3108865210C4800F0DA
:101900004FF900BF7678170889331608B0331608E8
:10191000CA331608A9321608E73316080C3416081D
:101920002F3416084B3416086F34160891341608F5
:10193000C4341608CA6E012A08B508D0022A0AD093
:101940001AB9D422086F00F023F8002008BD0A6FEE
:10195000034B1A60F9E70A6F11604A6FF8E700BF9E
:10196000704B0024FFECC2925D7D05C5FFECC29276
:1019700018DF88DFCD06CD767CD30CD3D982D9127F
:101980002C00050A0F14191E232800BFAFF3008096
:1019900000B501B400F004F801BC00BDAFF3008055
:1019A00000B5042A60DB00F0030E61F3830E7A4B6E
:1019B000D3E80EF0AFF30080AFF30080AFF3008008
:1019C00011F8013B00F8013BA2F1010211F8013BC3
:1019D00000F8013BA2F1010211F8013B00F8013BC4
:1019E000A2F101022DE9F01F282A07DBB1E8F81F58
:1019F000A0E8F81FA2F12802282AF7DADFF89CE114
:101A00004FEA920BDEE80BF051F8043B40F8043B40
:101A100026E0B1E81800A0E8180021E0B1E838009D
:101A2000A0E838001CE0B1E87800A0E8780017E0F2
:101A3000B1E8F800A0E8F80012E0B1E8F801A0E889
:101A4000F8010DE0B1E8F803A0E8F80308E0B1E818
:101A5000F807A0E8F80703E0B1E8F80FA0E8F80FEE
:101A6000BDE8F01F02F00302002A08BF00BD11F814
:101A7000013B00F8013B013A08BF00BD11F8013BF2
:101A800000F8013B013A08BF00BD11F8013B00F826
:101A9000013B00BDAFF30080AFF30080AFF30080E7
:101AA00011F8013B00F8013BA2F1010211F8013BE2
:101AB00000F8013BA2F1010211F8013B00F8013BE3
:101AC000A2F10102282A35DB2DE9F01FB1E8F81F49
:101AD00020F8023B4FEA134364F31F434FEA1444D8
:101AE00065F31F444FEA154566F31F454FEA164656
:101AF00067F31F464FEA174768F31F474FEA184836
:101B000069F31F484FEA19496AF31F494FEA1A4A15
:101B10006BF31F4A4FEA1B4B6CF31F4BA0E8F80F07
:101B20004FEA1C4C20F802CBA2F12802282ACDDA79
:101B3000BDE8F01F042A97DB51F8043B20F8023B74
:101B40004FEA134320F8023BA2F10402BAE711F86E
:101B5000013B00F8013BA2F1010211F8013B00F842
:101B6000013BA2F1010211F8013B00F8013BA2F197
:101B70000102042AFFF678AF51F8043B00F8013B5C
:101B80004FEA132320F8023B4FEA134300F8013BCE
:101B9000A2F10402EDE700007019020880190208A2
:101BA00008B508F0D3FA012000F004F8002008B5C9
:101BB00000F002F9044608B500F032F8204602F0C1
:101BC0002FFA2DE9F0410E468046174600F0D8F86E
:101BD000054616B300F0D4F801F01AFB002809DB23
:101BE000EB6B002B0FDD4FF0FF3400F0C9F801F074
:101BF0006BFB05E000F0D6F80468002CF0DD6442D1
:101C00002046BDE8F0810C2404FB03540133C4E9F1
:101C10001086A7640024EB63E7E74FF0FF34EFE79B
:101C2000F8B5064600F0ACF80C22C46B0027651E20
:101C300002FB0404002D00DAF8BDD4E90D23E16BAA
:101C4000C4E90E7713B1012A03D19847013D0C3C3A
:101C5000F0E7022A02D130469847F7E7032AF5D188
:101C600008469847F2E7002A44D010F0010F0346D7
:101C70003AD0013A03F8011B012A39D9F0B541EAFB
:101C800001259E07ADB22CD0023A23F8025B032A4D
:101C900019D95C0705EB054616BF141F144643F817
:101CA000046BB446224604EB030E072A13D8E2085D
:101CB0006FF0070707FB02423C40032A234484BF1E
:101CC000043A43F8046B012A02D9023A23F8025B72
:101CD00002B11970F0BDAEEB0207083AC7E900C6C1
:101CE000E3E7032AD5D8F0E7012AC7D11970704776
:101CF000002AFBD17047421E11F8013B02F8013F58
:101D0000002BF9D17047FFEC064B07B51B78034158
:101D1000DB0703D5019201AA00F0D1FD03B05DF805
:101D200004FB00BF640400240EB403B503AA52F8F8
:101D3000041B0192FFF7E8FF02B05DF804EB03B06B
:101D40007047FFEC30B50C4B0025D3E900428A42C6
:101D500008D0A14206D0013508331F2DF5D10C461D
:101D60004FF480528368C46123F4805323F00F033F
:101D700013438360002030BD84781708C069704722
:101D800008B500F002F8006808BD1FB5002001A9E1
:101D900001F0BEF90028ACBF0298002005B05DF844
:101DA00004FBFFEC08B5FFF7F0FF08B1143008BDE5
:101DB0000048FCE7744B0024044608B500F003F823
:101DC000204601F0C7F82DE9F041FFF7D9FF05469D
:101DD0000024FFF7DAFF4FF001082F7B061D08FAF9
:101DE00004F31F4208D056F8240028B105F110036F
:101DF00053F8243003B198470134042CEFD1BDE8E7
:101E0000F08170B504460D46E36D2046DB6A9847C5
:101E10000028F9D0E36D294620465B6ABDE8704092
:101E200018472DE9F74F858F0446B0F940308846B2
:101E30002DB24FF0800901920135AB42D8BF002589
:101E4000E28F12B2AA420AD0A38F2DB2626C002098
:101E50001BB202F80380A58703B0BDE8F08F019B99
:101E6000002B30D0EFF3118AEFF3108772B689F3AD
:101E7000118887F31088E28F12B2AA421ED1E2784D
:101E800002F0FF0BE2B90121E26D20466170926A17
:101E9000904704F11C0001F079F9E26D06465946BD
:101EA000926A204690475FFA8AFA8AF31188E278AC
:101EB00062B9002EC4DA6FF00300CDE70026F2E726
:101EC0006FF07F06EFE76FF00A00C5E76FF07F0065
:101ED000C2E72DE9F74F836881460E4601925C699F
:101EE00004F14807384601F051F9051E2FDB0025A3
:101EF0004FF0800B019B9D4204D2E3785BB30DB998
:101F00006FF07F05E36D012120469B699847B4F887
:101F10005020B4F8523012B21BB29A42B4F9542095
:101F2000C0F29E80B4F85010B4F8523009B21BB21F
:101F3000C91A0A2392FBF3F2914205D8E36D1B6A9A
:101F400013B1002220469847384601F06FF9284621
:101F500003B0BDE8F08FB4F85230B4F8502019B295
:101F600012B28A421FD0A26D0133525C1BB2B4F987
:101F700054109942D8BF0023A4F85230A36813F438
:101F8000E07F05D00A2A07D113F0400F18BF0D22B9
:101F9000013506F8012BADE70D2AF9D113F4807F46
:101FA00018BF0A22F4E7002DACDCD9F80830002B6A
:101FB00050D0D9F8001011F040014ED1EFF3118A42
:101FC000EFF3108872B68BF3118888F31088E26DF6
:101FD00020465FFA8AFA92699047B4F85010B4F834
:101FE000522009B212B291422CD1E26D0121204659
:101FF00092699047B4F85010B4F8522009B212B266
:10200000914202D08AF3118874E7E278BAB90122CA
:1020100004F12400A27001F0B9F88AF311880028B5
:1020200003DBE378002B3FF465AF002D7FF46AAF4C
:10203000E378002B7FF464AF6FF0030562E76FF085
:102040007F00EAE78AF31188E36D012120469B694E
:1020500098474FE76FF0500554E76FF00A0551E7D6
:10206000B4F85230B4F850101BB2D31A03FA81F10D
:102070005FE72DE9F04183685E6906F114052846A3
:1020800001F084F8041E23DBF378002B36D133787B
:10209000013313F0FF0734D0012F2DD1EFF3118856
:1020A00000238022EFF3108372B682F3118883F34A
:1020B000108833795FFA88F86BB9F36D30461B6886
:1020C0009847041E07DA88F31188284601F0AEF815
:1020D0002046BDE8F081F36D30469B689847041EAA
:1020E000F36D03DA5B6830469847ECE79B690121A2
:1020F0003046984788F311883770E6E76FF07F0421
:10210000E3E76FF01704E0E7F7B50E4600F160076C
:1021100000F1700557F8044F8CB16368A26843F072
:10212000180333401343A3604BB101A920690AF09F
:10213000D3FA019B002B02DC206901F077F8AF4253
:10214000E8D103B0F0BD2DE9F84383680E4615468B
:102150005C6904F12C08404601F018F8071E4ADBC0
:10216000002D52D004F16002002352F8045F002DCC
:1021700037D104EB8302193304F1340904EB8303F0
:1021800056664846736101F03BF8A38FB4F94020CE
:102190001BB201339A42D8BF0023E28F12B29A4297
:1021A0002CD1484604F1480901F040F8484601F0B6
:1021B00027F8B4F85020B4F85230484612B21BB297
:1021C0009A421EBF736803F001031D4301F02EF80D
:1021D000E378BBB145F0180529462046FFF794FF88
:1021E00006E00133042BC0D100236FF00F077361A9
:1021F000404601F01BF83846BDE8F883756805F0E5
:102200000405CEE7002DF3D0E6E77369002BEFD08D
:102210001D607561ECE7FFEC2DE9F04783688046AF
:102220000F4616465D69464B1B6823B1EB78ABB190
:102230006FF07F0425E000F05FFF0028F6D105F184
:10224000340A504600F0A2FF041E1ADBEB7803F0BC
:10225000FF018BB3504600F0E9FFE9E7EFF311848B
:1022600000238022EFF3108372B682F3118883F388
:10227000108807EB0608B84506D1E4B284F311884C
:1022800034462046BDE8F087EB6817F8011BD807F5
:1022900003D50D2905D11A0705D42846FFF7B1FD4E
:1022A000E9E70A29F9D113F0240F03D00D212846BC
:1022B000FFF7A7FD0A21F0E7D8F80030B14628461D
:1022C00083F04008EB6DC8F380189B6A9847B9F11A
:1022D000000F01D1344623E0EB6817F8011BD80743
:1022E00003D50D290AD11A070AD442462846FFF71A
:1022F00098FD041E10DB09F1FF39E8E70A29F4D143
:1023000013F0240F01D10A21EFE742460D212846A0
:10231000FFF787FD041EF6DAB14501D2A6EB0904EA
:10232000AA8FEB8F12B21BB29A4204D0EB6D01213F
:1023300028469B6A9847504600F078FFA1E700BF07
:10234000704B00242DE9F04700F1340804460E4696
:10235000404600F01BFF051E1DDBEFF31187002335
:102360008022EFF3108372B682F3118883F3108812
:10237000E37803F0FF0553B3A38F6FF07F05E38786
:10238000FFB287F311881E4F002DD7F800902CDA8A
:10239000404600F04BFF2846BDE8F087E36D012181
:1023A000204684F801A09B6A9847484600F0EEFE5C
:1023B000E36D054600219B6A20469847002DDFDB30
:1023C000A28FE38F12B21BB29A42E7D1D8E74FF047
:1023D000010A04F11C09F3E74FF47A7001F09CFB49
:1023E0003B68A3EB0903B34206D2E36D20461B6BA7
:1023F00098470028F0D0CBE76FF07305CBE700BF1C
:10240000844B00242DE9F0410B7905460C462BB195
:102410000B6943F001030B610523CB60012200210E
:1024200004F1340004F11C070AF03BF901220021F9
:1024300004F148000AF035F90122002104F11400EA
:102440000AF02FF90022384604F1240611460AF05A
:1024500028F90022304611460AF023F90122002112
:1024600004F12C000AF01DF90021384601F0E3F8D0
:102470000021304601F0DFF8234628464FF4DB7296
:102480000249BDE8F04100F06EBA00BF7C79170840
:1024900010B504460121FFF737FEA3783BB10023B6
:1024A00004F12400A370BDE8104000F0BFBE10BDD1
:1024B00010B504460421FFF727FE63783BB10023E3
:1024C00004F11C006370BDE8104000F0AFBE10BD09
:1024D00070B583680E4615465C69E36D1B695BBB8E
:1024E00040F207339E422ED0B6F5427F1CDAB6F595
:1024F0008A7F00F08E8040F215139E4200F0AD807E
:102500006FF0180040F201139E4200F0B280B6F561
:10251000817F37D1002D00F0B4802B68A3606B68F9
:10252000E360EB6823612CE037D040F209339E4230
:102530004FD06FF0180025E0984710F1190FCFD059
:102540000028DFD01EE0EFF3118100238022EFF39B
:10255000108372B682F3118883F31088B4F8522086
:10256000B4F8503012B21BB29A420CDCB4F85030BE
:10257000B4F852201BB212B29B1ACAB282F311886D
:102580002B60002070BDB4F85220B4F8500012B295
:10259000B4F9543000B2121AEEE7EFF311810023C0
:1025A0008022EFF3108372B682F3118883F31088D0
:1025B000E28FA38F12B21BB29A4203DCA38FE28F89
:1025C0001BB2D8E7E28FA08F12B2B4F9403000B24C
:1025D000E1E7EFF3118100238022EFF3108372B65D
:1025E00082F3118883F31088A28FE38F12B21BB29B
:1025F0009A4206DAE38FA28F1BB212B29B1A013BFA
:10260000BBE7A28FE08F12B2B4F9403000B2121AC9
:10261000F4E7EFF3118600238022EFF3108372B604
:1026200082F3118883F3108835F0020209D1B4F8DF
:102630005030A4F85230E36D1B6A13B111462046A6
:102640009847013D012D04D8A38F2046E387FFF76B
:102650002FFFF6B286F3118893E742F210712046FD
:10266000FFF770FE00288CD010F1190F3FF461AF16
:1026700088E735B1A3682B60E3686B602369EB6082
:102680007FE76FF015007DE770B504460D46EFF368
:10269000118600238022EFF3108372B682F3118833
:1026A00083F3108881F00103C37089B91821FFF703
:1026B0002BFD637823B104F11C00657000F0B6FDBA
:1026C000A3782BB1002304F12400A37000F0AEFD29
:1026D000F6B286F3118870BD10B5044600211C3097
:1026E00000F0FFFD002104F1240000F0FAFD0121BB
:1026F00004F1340000F0F5FD012104F1480000F080
:10270000F0FD04F12C000121BDE8104000F0E9BD0E
:1027100070B5836805465C6904F11406304600F024
:102720006FFD2378012B06D9013B2370304600F062
:102730007DFD002070BD0021E36D204621709B6966
:1027400098472B685B0604D44FF47A612046FFF764
:10275000F9FDEFF3118500238022EFF3108372B6A9
:1027600082F3118883F31088E36D2046DB68984775
:1027700023791BB9E36D20465B689847EDB285F37A
:1027800011882046FFF784FE2046FFF7A5FFCDE71E
:1027900070B5002504462E46A28FE38F12B21BB2FD
:1027A0009A4211D1A28FE38F12B21BB29A4204D186
:1027B000E36D002120469B6A9847ADB2EDB12046FB
:1027C000BDE87040FFF774BEE36D2046DB6A9847B2
:1027D0000028E7D0E38F2046616C1BB2E26DC95C34
:1027E000526A9047E38FB4F9402001331BB29A42FA
:1027F000E38700DCE6870135CEE770BD2DE9F341C4
:10280000B0F850505A23B0F9546004462DB2002756
:102810000135AE42D8BF002516FB03F6642396FBB4
:10282000F3F6E36D2046DB69984700283FD0B4F803
:102830005280B4F85020B4F852300FFA88F812B22F
:102840001BB29A4220DBB4F85010B4F8523009B2EF
:102850001BB2C91AB142E36D21D2E36D01A9204632
:102860005B6998474545DCD0B4F850300137A26D1C
:102870001BB2D0542BB20135A4F85030B4F9543007
:10288000AB42D8BF0025CCE7B4F85220B4F954309D
:1028900012B2B4F850109B1A03FA81F1DAE71B6AFE
:1028A000002BDAD00122204698470028D5D0BFB2AD
:1028B00017B12046FFF7ECFD02B0BDE8F08130B55E
:1028C00085B00C461546684600F018F82A6821467F
:1028D000684609F0F7FF05B030BD0D2938B504464C
:1028E0000D4607D0284600F015F8031E03DBE36809
:1028F0000133E36038BD0433F4D0FBE7034B0360DE
:10290000034B83600023C360704700BFDB280208CD
:10291000E5DC020838B50C4B04460C4D1B681BB1B6
:10292000286858B9204638BD00F0E6FB0028F7D1EA
:1029300028680028F6D003681B6801E003685B681C
:1029400021469847EEE700BF704B0024680400243E
:1029500010B514460846114607F09AFD204610BDF2
:102960000846FEF76DBA2DE9F34107460E4690463C
:102970001D4600F01BF8041E12DB01AA4146384632
:1029800000F07AF8041E09DB019B0024DA8922F0AA
:102990000F0242F00102C3E90465DA8100F028F871
:1029A000204602B0BDE8F08100F05AB838B50F4CAF
:1029B00001F028FB0546A368984204D1A3890020B2
:1029C0000133A38138BD204600F022FC002807DA3D
:1029D000FFF7E8F900680428F5D08C28F3D04042CE
:1029E0000028EFD10123A560A381EBE77004002448
:1029F00008B501F007FB0A488389012B0CD100239D
:102A000083814FF0FF33836000F05EFC002805DA1D
:102A1000BDE80840FFF7C6B9013B838108BD00BF90
:102A20007004002410B503460446184613F8012B21
:102A30002AB9001B1C3009F0CBF918B910BD2F2A98
:102A4000F3D1F6E700F11803013C14F8012F12B995
:102A500000221A70F2E72F2AFAD003F8012BF4E7CC
:102A600008B50348FFF7DEFF024B186008BD00BF42
:102A700081DF1608784B002400232DE9F04116462B
:102A80001360027888B0002A45D08DF81C30CDE95B
:102A9000010301A8CDE90333CDE9053300F04AF87D
:102AA000002835DA019FDDE90354384600F036F896
:102AB000037880463846D3B1FFF7B4FF48B96FF0CA
:102AC0000B04069808B109F06BF9204608B0BDE880
:102AD000F0813DB16B68C0E9004368604746044639
:102AE0000025E2E7A368C0E90043A060F6E7FFF72E
:102AF00099FF0028E3D035B16B68C0E900436860F6
:102B000000243060DDE7A368C0E90043A060F7E778
:102B10006FF01004D5E76FF01504D6E7027803468E
:102B200001300AB12F2AF9D11846013302782F2A31
:102B3000FAD07047F8B5036804461B782F2B11D0E4
:102B400005462E4800F0CAF82D4A55F8143B0028D7
:102B500018BF02462B49284609F06AFE6369002B1C
:102B600046D02360284B196823681A782F2A42D14F
:102B700000252E4641B90A466FF001002261C4E9E2
:102B80000031C4E90265F8BD53B301F117005F1EBF
:102B900010F801CF17F8012FBCF1000F06D182B158
:102BA0002F2A0ED04A680E461146E3E722B12F2A9B
:102BB00002D09445F6D3EBD900216FF001000A460C
:102BC000DCE71846FFF7AAFF0346007858B1CA8928
:102BD00002F00F02032A08D08A680D460021E2E7BE
:102BE0001A461946C8E71A46C8E71A460020C5E73C
:102BF0006FF00B00C7E76FF01500C4E7D64B16085F
:102C000032D41608DB341608784B002430B58DB06A
:102C100000230546694601A8009307F04BF9041EFE
:102C200005DB01A80BF0DAFA009B28606B602046F8
:102C30000DB030BD73B50346124CC0B122460068DA
:102C4000596803C26846104E00F032F82368009AB3
:102C5000002061689B1A019A891A23600A46002A9B
:102C600003F1FF3507DB50B9616002B070BD20464B
:102C7000FFF7CCFFE6E732442B460120EFE7C4E93B
:102C80000032F2E77C4B002400CA9A3B08B506F0FC
:102C9000AFFF07F017F80020BDE80840FFF7CABFF4
:102CA000024A136801331360704700BF844B00244D
:102CB00038B50025074B04464FF47A721868294648
:102CC000002314F0F5FD044B206028465343636055
:102CD00038BD00BF844B002440420F0038B5044685
:102CE00018B300F0CBF9124B1B689D688DB12146DB
:102CF000284601F0AFFA041E0CDB2B6C3D2153F883
:102D000024000BF011F968B1441C00F0C7F920460B
:102D100038BD2C4600F0C2F96442FFF743F8046066
:102D20000024F4E76FF01504F4E76FF01504F3E7FF
:102D3000744C00243F4C01233F4DA82204F18C0623
:102D40002B7083B500212046FEF78DFF0323182248
:102D50003A49237730463A4B3A4FC4E905330623C4
:102D6000A3860BF0F6F8384920463E6009F029FCAE
:102D7000364B374E1C6002232B7000F0D9FA01A9A4
:102D8000684606F00BFFDDE9000108F0F3FF0423BD
:102D900033603368012B49DD3068800009F018F892
:102DA0002C4B186033680460224894F8341001F00A
:102DB000FDFAA3681F489B6A9F6007F0B7FC1D4897
:102DC00001F03CF91B4801F01FFBA36805221A72B1
:102DD0000022214B1A6003232B7000F04FF90CF0F6
:102DE00055FE1E4B0BB101F06FFB1D4B0BB1FFF7F6
:102DF0004DFF1C4B0BB101F055FD02F01FFB07F01E
:102E00002DFB0BF07BFE04230A482B702FF174FD81
:102E1000084801F029FB05232B7000F025F8062354
:102E20002B7000F03BF907F07FFCFCE733685B0098
:102E3000AEE700BF904B0024384C0024B07917084F
:102E4000352D0208884B0024744C0024704C00245B
:102E50003C4C0024404C0024444C0024C94402084B
:102E60008D2C0208A548020813B500240122094947
:102E7000094801F007FA01F08DF901F097F9074BC5
:102E800040F67A4264210094054800F086FE204610
:102E900002B010BD32D41608D64B1608A55402084D
:102EA000E1341608A52870B505460C461AD8EFF38C
:102EB000118600238021EFF3108372B681F311880D
:102EC00083F310881CB9FEF7ADFB2246074C084B74
:102ED000F6B243F8354003EBC5035A6086F3118818
:102EE000002070BD6FF01500FBE700BF312F020816
:102EF000004F0024A52808B50CD8094A52F83030F4
:102F00005BB102EBC00252689847064B1A68064B49
:102F10001A6008BD0022054BF6E71A46FBE700BF22
:102F2000004F0024744C0024704C0024312F020800
:102F300008B5EFF3118300238022EFF3108372B6FC
:102F400082F3118883F3108836210148FEF728FEAA
:102F5000EA3416080E4B37B504461D684FF0FF33B0
:102F6000002201A90320019300F08CFB01F030F84E
:102F7000214600F033F8044610B10120FEF71AFE96
:102F800002460146284600F0E5FF204607F046FAD3
:102F9000744C002438B50C468D680023016A39B1A1
:102FA0008A6895420A6810D1A3B98AB9C0E9083382
:102FB00004F1140000F0CEF804F10C0000F0CAF89F
:102FC0002046BDE8384008F0EBBE0B461146E6E768
:102FD0000262EDE702B943621A60E9E7F7B5044619
:102FE0000F4600F0EEFF00F118060546304600F0EF
:102FF00007F92146284600F038F8044630B9304633
:1030000001F081FA4FF0FF3003B0F0BDC76101233A
:1030100000F10C0701A98371384609F05DFB0146F8
:1030200030B16379E3B121462846FFF7B3FF17E0DB
:10303000019A002AF5DA14340132204609F031FBF6
:10304000384601F060FA18B901A9384609F044FB86
:10305000019B002B01DA0028F2D0204600F0D0F8C6
:10306000304601F050FA0020CEE7006A10B18368C4
:103070008B4200D170470068F8E7FFEC054B1B68F6
:103080002BB1054A126812B9DA8E0132DA860020B5
:10309000704700BF744C0024704B0024134B10B5D4
:1030A0001A68C2B1124B1B68ABB9EFF311848021CF
:1030B000EFF3108372B681F3118883F31088B2F9AD
:1030C0003630002B09DC0023D3860A4B1B6853B92A
:1030D000E4B284F31188002010BD013B1BB2D386FB
:1030E000002BF5D1EFE707F0DFF9F1E7744C00248E
:1030F000704B0024684C0024044B1B6823B11868F3
:10310000B0FA80F04009704701207047744C0024E9
:1031100038B50F4B0C461D6870B101F03FFAA0B1F5
:10312000AB8E03F00303022B07D0AA6883689A4290
:1031300003D06FF00C0007E02846C36C2360036DDA
:103140006360436D0020A36038BD6FF00100FBE7B2
:10315000744C002408B540B103881B0401D401233A
:10316000038000F0C9F9002008BD6FF01500FBE7EF
:1031700010B5FFF7EFFF041E05DA6442FEF712FEFA
:1031800004604FF0FF34204610BDFFEC1B4B70B5C0
:1031900004461D68EFF3118600238022EFF31083AD
:1031A00072B682F3118883F3108820B303881BB2B0
:1031B000002B038803F1FF331BB2038008DD0024DA
:1031C00000F0D8F9AC65F6B286F31188204670BDE0
:1031D000A865FFF753FF204600F0D4F9002305212E
:1031E00028462B8707F0BCF8B5F9384004B1644293
:1031F000FFF754FFE7E76FF01504E4E7744C002491
:1032000010B504462046FFF7C1FF031DFAD010BDDC
:1032100010B5FFF7BBFF041E06DA6442FEF7C2FDDD
:1032200004604FF0FF3010BD0020FCE770B505468C
:10323000002844D0EFF3118600238022EFF310839F
:1032400072B682F3118883F31088038847F6FF7201
:103250001BB2934205D1F6B286F311886FF08A0053
:1032600070BD00F099F92B8801331BB22B80FFF75A
:1032700005FF2B881BB2002B1FDC124B1C687CB196
:10328000A36DAB4217D12946204600F04BF904F15B
:103290003C0000F0E1FE00232046A36507F0A2F900
:1032A0002946204600F09CF9F6B2FFF7F7FE86F3B8
:1032B00011880020D4E72468E1E70024F0E76FF0EC
:1032C0001500CDE7604C002410B5FFF7AFFF041EDA
:1032D00005DA6442FEF766FD04604FF0FF342046D5
:1032E00010BD70B505460C46FFF7C8FEEFF311861A
:1032F00000238022EFF3108372B682F3118883F3E8
:1033000010882B881A0409D42B881B040ED5F6B21A
:1033100086F31188FFF7C2FE002070BD002CF3DD9C
:10332000013C2846FFF782FF24B2EAE72C80EEE753
:1033300000F0CEB8CB6803F130021B6B1BB18B429F
:1033400012D14B6813600023021DC1E90133CB6029
:103350000B8243681BB18B4209D10B681360054B8C
:103360001A6819600A6070471A1D5B68E6E71A461A
:103370001B68EFE77C4C002408B503460846B3F908
:103380001020002A04DC1946FFF7D4FF012008BDF5
:103390000020FCE708B50B4601461846FFF7CAFFB8
:1033A000002008BD10B5C068117C90F82E309942FD
:1033B0000ED9047CA1420DD9A34206D2437F0F2B24
:1033C0009FBFC11801338C774377117C01F03AF924
:1033D000002010BD437F0F2B9FBFC2180133917790
:1033E0004377F5E70346084670B51546B3F9102054
:1033F000DC68002A02DC1946FFF79CFF227C94F867
:103400002E108A4204D0637F23B9204601F062F96E
:10341000002070BD297C8A4218D804F11E060020C5
:10342000012225189342A97F09DC013B20461EBFDB
:10343000E218927FAA77637701F004F9E8E716F8BB
:10344000015F8D4288BF10460132EAE704F11D009A
:10345000002210F8015F8D4207D1013B1FBFE11828
:103460001219897F91776377D2E701329342F0DCBA
:10347000CEE7FFEC054B10B51B68C4689C4203D136
:10348000FFF7B0FF012010BD0020FCE7744C0024C2
:10349000064B10B41B68C4689C4203D05DF8044B13
:1034A000FFF7A0BF00205DF8044B7047744C002468
:1034B000F8B504460D4616464068002300B103B136
:1034C000F8BD076832462146A84703463846F5E767
:1034D000074A0021074B1A6002F11403013143F837
:1034E000143C14331F29F9D10023C2F86C32704701
:1034F000804C00247C4C002410B5EFF31184002391
:103500008022EFF3108372B682F3118883F3108860
:1035100000220349E4B2FFF7CBFF84F3118810BD0A
:1035200095330208036830B5DBB18B78DB0718D41C
:103530004A681346B3B90E4C236893B11D681A60EC
:1035400000224B601A822560C3E90210026B5A60A8
:103550000363B3F9102047F6FF718A421CBF0132A2
:103560001A8230BDDC68A042F3D01B68E2E700BFDE
:103570007C4C0024024B01461868FFF7D3BF00BF04
:10358000744C0024024B03491A68FFF791BF00BF37
:10359000744C0024A53302080C4B002210B51146D0
:1035A0001C68436833B9012A02BF0B8A03F1FF3359
:1035B0000B8205E0D968A14203D11A8A013A1A8226
:1035C00010BD194601321B68ECE700BF744C0024A3
:1035D000024608460149FFF76BBF00BFE53302080A
:1035E00038B504460D4690B10A4B1B681BB1BDE8C7
:1035F0003840FFF7EDBF024607492846FFF758FF5E
:10360000224606492846BDE83840FFF751BF02462A
:103610000349F7E7704B002491340208753402081F
:103620007933020810B50446216B01B910BD8868D2
:10363000FFF780FEF8E7012908B50AD002290DD06E
:1036400079B9827842F001028270FFF755FF0020BD
:1036500008BD827822F001028270F8E76FF08500E1
:10366000F6E76FF01500F3E710B5FFF7E4FF041E6F
:1036700005DA6442FEF796FB04604FF0FF34204603
:1036800010BDFFECF8B51746194B06460C461D68F1
:10369000FFF7F4FC0FB1EB6D3B60D4B1EFF3118396
:1036A00000228021EFF3108272B681F3118882F339
:1036B0001088022E11D0032E14D0012E14D1EA6DE1
:1036C00021680A430024EA65DBB283F3118800F025
:1036D00011F8FFF7E3FC2046F8BD2168EA6D22EA05
:1036E0000102EFE72268EDE76FF01504ECE700BF99
:1036F000744C0024174B37B51D68FFF7BFFCEC6D09
:10370000284601F02DF9E4430440019424B9FFF761
:10371000C5FC204603B030BD01A800F06FF8431C83
:10372000044610D0014601A808F0F9FF21462846BA
:1037300000F012F8044630B1011D284600F06EF882
:10374000204600F02DF8019B002BE5D1FFF7A6FCE9
:103750000120DFE7744C002438B58368EFF311854E
:1037600000228020EFF3108272B680F3118882F37A
:10377000108800205C6B3CB122798A4209D103F1A8
:10378000340148B108F002FFEDB285F311882046FC
:1037900038BD20462468EEE7084608F0EDFEF3E762
:1037A00010B5037B83B9EFF311848022EFF310830C
:1037B00072B682F3118883F310880E4908F0A8FED0
:1037C000E4B284F3118810BD022B0CD1EFF3118405
:1037D00000238022EFF3108372B682F3118883F303
:1037E00010880549EAE7012BEDD1BDE8104008F04B
:1037F000D7BA00BF385400243054002438B50546E9
:1038000001242146284608F09AFF20B90134202CD3
:10381000F7D14FF0FF34204638BDFFEC2DE9F041E1
:103820000D460978044629B35C3008F088FF01286A
:1038300007467ED1EFF3118600238022EFF3108339
:1038400072B682F3118883F31088237FF6B2062BB9
:1038500012D1297804F1600008F071FF60B12B6883
:10386000204663676B68A3670023236606F0BAFEF1
:1038700086F311880026C0E086F31188A4682978B1
:10388000EFF3118200238020EFF3108372B680F3F0
:10389000118883F31088636B13B11879884208D1BB
:1038A000D2B282F3118833B12A685A606A689A608A
:1038B000E0E71B68F0E7564B1B68FBB1554808F082
:1038C0005BFE20B9544808F057FE0028D2D02B6880
:1038D00043606B688360EFF3118500238022EFF370
:1038E000108372B682F3118883F3108804F13401D7
:1038F000EDB208F00DFE85F31188BBE7EFF31186FA
:1039000000238022EFF3108372B682F3118883F3D1
:1039100010884048F6B208F02FFE86F31188002880
:10392000D5D1102008F044FA0028A3D00123037356
:10393000CDE7FFF7A3FB2978A06801F02DF8064634
:1039400058B343684BB301F039F8002858D0736876
:103950004360B2688260F3689B0604D4297801232F
:103960008B40134383602B68C3606B680361EFF384
:10397000118600238022EFF3108372B682F3118840
:1039800083F3108804F16401F6B208F0C1FD234905
:10399000204606F011FF86F311880026FFF77EFB14
:1039A000EFF3118800238022EFF3108372B682F3C5
:1039B000118883F31088237F062B08D12B682046BB
:1039C00063676B68A3670023236606F00BFE5FFA4C
:1039D00088F888F31188002F15D1237F052B03D198
:1039E0000421204600F03BFF237F072B05D12B78D5
:1039F000082B02D1204600F077FE3046BDE8F0816A
:103A00006FF00B06CAE7F8DA6FF01506F5E700BFAE
:103A1000704B002438540024305400243B3A0208F0
:103A200010B50C4600F0BAFD20B12146BDE81040AB
:103A3000FFF7F4BE6FF0020010BD2DE9F04F87B024
:103A40000446FEF7AFF903684FF0800A04F16C09F1
:103A50000193B4F93830029304F164030593EFF352
:103A60001183EFF3108772B68AF3118887F31088F9
:103A7000B4F8348018F400725FFA83F804920AD024
:103A800088F31188FEF78EF9019B0360029B238760
:103A900007B0BDE8F08F059808F06EFD06460028D7
:103AA000EED0A28E494642F40072A28608F030FDA4
:103AB000D4F85CB0B5684BEA0505E56588F3118874
:103AC000736806F10C01049A307B9847EFF3118874
:103AD000039BEFF3108372B68AF3118883F3108887
:103AE00003934946A38E30465FFA88F823F40073A7
:103AF000A386E36D5D4083EA0B031D4085EA0B0559
:103B0000E56508F023FD88F31188FFF7F3FD3046E3
:103B100000F080FFA3E7FFEC07B568B1084A002179
:103B2000B0FBF2F302FB130000934FF47A73584397
:103B30000190684600F0CAFF03B05DF804FB00BFC7
:103B400040420F002DE9FF410546A8208846164651
:103B50001F4608F03DF90446E0B10023A0F8348088
:103B60002946324603930C9B02930B9B01930A9BBD
:103B700000933B4600F044F8051E06DA204608F0A4
:103B80000FF9284604B0BDE8F0812046E56800F052
:103B90009BF9F6E76FF00B05F3E71FB5069C009263
:103BA0000A46CDE9013400231946FFF7CBFF04B0E4
:103BB00010BD13B5049C0094FFF7EFFF041E05DA57
:103BC0006442FEF7EFF804604FF0FF34204602B085
:103BD00010BD1FB5079C0294069CCDE90034134626
:103BE0000A460221FFF7AEFF04B010BD13B5049CD6
:103BF000CDE9003413460022FFF7EBFF02B010BD01
:103C00002DE9F34790F834608846054691463146E1
:103C10001F46DDF828A000F0C9FB041E40DB0D990B
:103C200006F00306A86800F0CDFA041E11DB284652
:103C300000F036FC041E0CDB87B15246394628469C
:103C400006F0FAFC041E05DB284600F0F7F9041E16
:103C500013DA57B1284600F0DDFB21E03246514629
:103C6000284606F0B5FB041EEEDA2B6D002BF1D0D2
:103C70003146284606F03EFCECE70B9B49460A4AD3
:103C80002846009600F0A4F8041EE2DB0C9A414698
:103C9000284600F0ADF8041EDBDB284600F0B4FB3C
:103CA000204602B0BDE8F087013F02082DE9F74F3A
:103CB00004460E4601929946EFF3118700238022B5
:103CC000EFF3108372B682F3118883F31088DFF864
:103CD000F8A0DFF8F880DAF800500020D8F80030BB
:103CE0000135374A116888420DDB1068C00008F0C2
:103CF0006FF8334A0546002844D1FFB287F3118894
:103D00006FF00B0038E0012D1168B8BF01250139B3
:103D1000294053F821B0BBF1000F30D143F82140C6
:103D2000FFB2E560CAF8005087F31188019BF6B234
:103D30009DF83020594603202674667484F82E605E
:103D4000C4E90539A38E62F3010304F15C0223F098
:103D50006003A386FFF796FC204684F81CB006F0AB
:103D6000E5FCFFF78BF91749204608F02AFC0423ED
:103D70002377FFF793F9584603B0BDE8F08F01357C
:103D80000130AFE711684FF0000C0D4B4900116096
:103D90001A68D8F8000002EBD272BCEB620F04DBA9
:103DA00007F0FEFFC8F8005095E750F82C000CF122
:103DB000010C1A68C168013A0A4045F82200E7E799
:103DC0003C4C0024484C0024444C0024404C00242B
:103DD00010B49DF8044001945DF8044BFFF766BFF2
:103DE00013B501240094FFF761FF02B010BDFFEC92
:103DF000344B2DE9F74F002914BF884698460746F3
:103E000000241546414618228C300AF0BEF8404680
:103E100087F8A4400AF0B1F8461C4DBB2C4602348A
:103E2000384606EB840106F0B9FB06464FEA8409E2
:103E3000002844D000EB090AA9F10809B346043D63
:103E4000C0F800A040460AF098F80446B144414644
:103E500001345046FDF74FFF5444CB451BD10020A1
:103E60004AF8040CBB689B6A9E6003B0BDE8F08F03
:103E700040F2011955F824000028D0D001360AF08C
:103E80007CF8FB6C06449E4216D201344C45F1D1BD
:103E90006FF00600E9E74BF8044F55F8041F084699
:103EA00001910AF06AF880460199204608F101085C
:103EB000FDF721FF4444D0E76FF05A00D5E76FF0DB
:103EC0000B00D2E7FC79170838B50446EFF31185EB
:103ED00000238022EFF3108372B682F3118883F3FC
:103EE0001088037F042B01D02EF128FD2046EDB26F
:103EF0002EF102FD204606F075FB85F3118838BDD2
:103F000038B5134B1C68A38E03F00303022B02D0B9
:103F1000204600F0E9FEA368012040F201119B6AEF
:103F20009A6852F820304BB9A38EA56903F00303B9
:103F3000022B08D11146A847FDF73CFE013088420C
:103F4000EFD10120F8E70146284608F09FFBF8E78B
:103F5000744C002470B5838E0E460446190517D4A0
:103F60003AB9806828B1437A012B02D1543009F064
:103F700007FC204600F03AF8A56855B9204600F045
:103F800049FA204600F074FDA38E43F40063A38633
:103F900070BDA38E03F00303012B03D06B690BB13B
:103FA00036021E606B7A012BE8D1002305F10C0666
:103FB0006B61EB72AB891B04E0D53046FFF736F935
:103FC000F8E708B500F0EAFA00B1806808BDFFEC38
:103FD000054B186830B1037F032B01D1C0687047CF
:103FE0006FF00200704700BF744C002410B5044607
:103FF00000F0ADFA204600F063F82046BDE810401E
:1040000000F00CBC054B186830B1037F032B01D1C5
:10401000C06870476FF00200704700BF744C002406
:104020000446002208B5E4B2034B21461868FFF7A6
:1040300091FF204606F0F2F9744C002410B51821C7
:10404000044606F0ABFA20B1A3689B6A0360002027
:1040500010BD6FF00B00FBE738B50446EFF3118598
:1040600000238022EFF3108372B682F3118883F36A
:104070001088F0B14368E3B1104B00201B68DBB13E
:10408000A3420FD123681BB19A68A1680A449A60C1
:1040900058B10A4908F07AFA00206060EDB285F361
:1040A000118838BD18461B68E9E7044808F064FA2F
:1040B000F2E76FF01500F1E71B68FFDE58540024AB
:1040C0003C30FFF7C9BF2DE9F84300220B461146EB
:1040D000586809F034FD0546EFF311848026E4B2F8
:1040E0000023EFF3108372B686F3118883F31088F0
:1040F000002700F108084046FFF782F8284608F03C
:104100003BFA03460028F6D00269002AF3D0406942
:104110001F6184F311889047EFF31184E4B24B469A
:10412000EFF3108372B686F3118883F310889946F3
:10413000E1E7FFEC2DE9F0418CB004460E4617464E
:104140000DF11008114A20211D46404608F07DFB64
:10415000CDF808804FF00008CDF80C80FEF78EFFF8
:1041600002AB20463A4631460093094BFFF73EFD2D
:10417000041E07DB2C614446FEF790FF20460CB07E
:10418000BDE8F081FEF78AFFF8E700BF02351608A8
:10419000C7400208034B4FF4A062F9210248FFF721
:1041A000C9BF00BF9404002407351608034B4FF421
:1041B000CC6232210248FFF7BDBF00BF800400245B
:1041C0000E3516082DE9F041214B0C4606461D68B8
:1041D000FEF754FF7CBBAB681C6C64BBFEF75EFF54
:1041E0002046BDE8F081013554F82570002FFAD142
:1041F0005DB34FEA850808F1040007F0D9FD0746D2
:10420000B0B10023444440F82530013D54F8040D7A
:1042100009F0B3FE013007F0CBFD47F8250078B96F
:1042200007EB850555F8040F38B9384607F0B8FD97
:104230006FF00B040AE00025D6E707F0B1FDF1E7C7
:104240002168FDF758FD013DE0D200243764C5E741
:10425000744C002470B5046C84B1002054F82030F4
:1042600063B14A1E013B12F8016F13F8015FAE42C1
:10427000F9D00EB93D2D03D00130EFE76FF001000A
:1042800070BDFFEC2DE9F8430F46144605460028A3
:1042900060D009B10B782BB9B4B12846BDE8F8431A
:1042A00000F05EB8FEF7EAFE2B4B1B68D3F80880DF
:1042B000D8F8403073B129464046FFF7CBFF011EC6
:1042C00008DB24B9FEF7EAFE0020BDE8F88340468B
:1042D00000F066FE284609F050FE0446384609F014
:1042E0004CFE2044023007F063FD064638B3D8F890
:1042F0004090B9F1000F2BD1082007F059FDD8B13B
:104300004C4640F82460002300EB84042A461349FD
:1043100063603B46C8F84000304608F072FAD1E7C7
:10432000013459F82430002BFAD1A11C48468900E9
:1043300007F046FD0028E4D1304607F031FD0C249B
:10434000FEF7ACFEFDF72EFD04604FF0FF30BCE73A
:104350000024E6E71624F5E7744C0024153516080A
:1043600038B5114B04461B689D6828B103781BB112
:104370003D2109F0D9FD30B1FDF714FD162303608E
:104380004FF0FF3038BDFEF779FE45B12146284693
:10439000FFF760FF011E02DB284600F001FEFEF77A
:1043A0007DFE0020EEE700BF744C002470B5064689
:1043B0004FF47D7007F00CFD044610B300F0BCFC18
:1043C000051E04DA204607F0EBFC284670BD04F118
:1043D0004400B4600BF08BFB204609F0DBFA0122AD
:1043E000002104F1180008F05CF90C3400220025CB
:1043F0002046114608F055F900212046FFF71BF929
:10440000E3E76FF00B05E0E7D0E902321A60012222
:104410005A72704738B58468054634B1637A012B07
:1044200004D9013B63720023AB6038BD204600F025
:1044300094FC204600F035FB204600F070F804F1B3
:1044400044000BF058FB204609F0C3FA204600F068
:1044500093FDA37A23B1237A43F008032372E2E7A2
:10446000204607F09DFCDEE738B5032105460B48E2
:104470000BF01DFF041E0BD101210BF031FC204677
:1044800002210BF02DFC2846BDE8384000F0A6BD07
:1044900001DD0BF074FC6FF0160038BD44321608D5
:1044A000084B10B51B680446816898684431443055
:1044B0000BF0BBFB002804DB2046BDE8104000F0F9
:1044C0008DBD10BD744C00240023044A044942F8F9
:1044D00033100133A62BFAD1FDF7CCB8004F0024DE
:1044E000312F020808B53AB119B9FEF74FFE404224
:1044F00008BD00F00BF9FAE711B9FEF781FEF6E707
:1045000000F008F9F3E708B528B1FEF78FFE0028A0
:1045100003DA404208BD1620FCE70020FAE738B570
:104520000446256A2DB904F11800BDE83840FEF7AD
:1045300011BE284650F8143B2362FEF70BFE05F12E
:104540000C00FEF707FE284607F02AFCE9E7F8B55D
:10455000802600270446FEF791FDE36F1BB9BDE8F6
:10456000F840FEF79BBDEFF311832A46EFF310826C
:1045700072B686F3118882F31088E06F1546DBB2BD
:104580000268E267076083F31188037C043043F01C
:1045900002030373FFF7B7FFDFE7FFEC0346EFF318
:1045A000118100228020EFF3108272B680F311880F
:1045B00082F310880A4A106860B1002B0EDB094AAA
:1045C0001268013A1A4050F8220018B1C2689A42A3
:1045D00018BF0020CBB283F3118870470020F9E7A1
:1045E000404C00243C4C002438B5044618B3C06845
:1045F000B0B1EFF3118200238025EFF3108372B680
:1046000085F3118883F310880C4B00251B68013B50
:1046100003400B48006840F82350D3B283F311885D
:10462000236D13B1204605F065FF2046FFF7F2FE2B
:10463000204607F0B5FB002038BD00BF3C4C0024ED
:10464000404C0024F8B54B1E0446FE2B3BD8EFF33C
:10465000118600238022EFF3108372B682F3118853
:1046600083F31088027FCDB2022A0DD0032A17D11E
:1046700003681B7C994224DC294605F04DFFF6B205
:1046800086F311880020F8BD104B1B681B7C9942F3
:10469000F2DC00F0DDFC2046257400F0B5FCEEE70E
:1046A0000B4B53F8327003EBC2031B79DB0708D5C1
:1046B000394607F091FF39462046257400F0DCFCAE
:1046C000DDE72574DBE76FF01500DCE7744C0024B0
:1046D000BC79170838B504460D46FFF7B3FF10B98B
:1046E00084F82E50607738BD10B5EFF311840023A5
:1046F0008022EFF3108372B682F3118883F310885F
:1047000005F070FFE4B284F3118810BD0A46002161
:1047100000F008B80A46002100F04EB80A46002111
:1047200000F056B8214B2DE9F743074689469046DD
:104730001D68EFF3118600238022EFF3108372B619
:1047400082F3118883F3108800F0D8FC044688B106
:10475000D8F80420164B9A4224D801AA414648466C
:1047600000F0DCFB28B9019C002C0ADC6FF073041C
:1047700000E04442F6B286F31188204603B0BDE85B
:10478000F0833C35FFF724FC21460346094A2846BE
:1047900000F0EEFA3846FEF7F9FC04462846FFF72B
:1047A0005BFCE7E76FF01504E4E700BF744C0024FE
:1047B000FFC99A3BEB47020870B504460D46164602
:1047C000324629462046FFF7ADFF031DF8D070BDE5
:1047D00010B5FFF7A7FF041E05DA6442FDF7E2FA01
:1047E00004604FF0FF34204610BD10B5EFF3118484
:1047F00000238022EFF3108372B682F3118883F3D3
:104800001088FFF7CBFE28B1037F052B02D174215E
:1048100000F025F8E4B284F3118810BD70B50446A9
:10482000EFF3118500238022EFF3108372B682F339
:10483000118883F31088037F052B09D1866D3146DB
:10484000FEF7C6FE338801331BB233800023A36515
:104850002046EDB2FEF7E6FE85F3118870BDF8B58F
:1048600004460E46EFF3118500238022EFF31083F8
:1048700072B682F3118883F31088037F052B0DD164
:10488000876D3946FEF7A4FE3B88204601331BB2F4
:104890003B8000232687A36505F0A4FEEDB285F3D7
:1048A0001188F8BDF8B50024284B294E6020C3E9D3
:1048B0000044284BC3E90044274BC3E90044274B7D
:1048C000C6E90044C3E9004407F072FA054648B15E
:1048D00000F160072C7528461835314607F018FEA0
:1048E000AF42F7D1602007F063FA044658B100F1F7
:1048F00060050227174E277520461834314607F009
:1049000007FEAC42F7D1402007F052FA044658B1F6
:1049100000F140050027104E277320461034314621
:1049200007F0F6FDA542F7D1402007F041FA044612
:1049300058B100F140050227084E27732046103475
:10494000314607F0E5FDAC42F7D1F8BD50540024E4
:104950004854002440540024385400243054002487
:10496000002337B582680193EFF311858021EFF3BF
:10497000108372B681F3118883F31088546B2CB9BD
:10498000EDB285F31188019803B030BD217901A8FB
:1049900007F0B9FE2468F2E738B50D46044640B189
:1049A000FEF76CFBE46A14B1237CAB4203D1FEF743
:1049B00075FB204638BD2468F5E7FFEC124B10B5B7
:1049C0001B6843B1114807F0D7FDE0B91048BDE8B6
:1049D000104007F0D1BDEFF3118400238022EFF3E4
:1049E000108372B682F3118883F310880748E4B20B
:1049F00007F0C2FD84F3118828B9182007F0D8F910
:104A000008B10123037510BD704B002448540024E5
:104A10004054002410B5037D83B9EFF31184802244
:104A2000EFF3108372B682F3118883F310880E4976
:104A300007F06EFDE4B284F3118810BD022B0CD197
:104A4000EFF3118400238022EFF3108372B682F318
:104A5000118883F310880549EAE7012BEDD1BDE801
:104A6000104007F09DB900BF485400244054002472
:104A700038B5044600F16405284607F07DFD50B9BD
:104A800004F16C05284607F077FD38B94FF0FF3286
:104A9000C4E9172038BDFFF7BDFFEDE7FFF7BAFF08
:104AA000F0E738B5044600F12C05284607F064FD10
:104AB00028B93434204607F05FFD18B938BD00F03E
:104AC00045FBF2E7FEF76CFEF4E7FFEC2DE9F74358
:104AD0000F46054600283BD042681F4B9A4237D804
:104AE000EFF3118600238022EFF3108372B682F376
:104AF000118883F31088DFF864906846F6B2D9F81D
:104B0000008007F018FE2A460021684600F0F6FBF8
:104B100010F10B0F044606D186F3118800242046BD
:104B200003B0BDE8F08387B101A9284607F074FD02
:104B3000D9F8003001983946A3EB080290428ABFA9
:104B4000C01A0020404407F059FD86F31188E6E7BB
:104B50006FF01504E3E700BFFFC99A3B844B0024C4
:104B60007FB51D46CB0714462AD5EFF311860023E7
:104B70008022EFF3108372B682F3118883F31088DA
:104B800002A9F6B200F06EF9002806DA86F3118861
:104B90004FF0FF34204604B070BD6A4602A920469B
:104BA00007F056FD29466846FFF790FF044686F356
:104BB0001188002CEEDA6442FDF7F4F80460E7E7B0
:104BC00029461046FFF782FF0446F2E77047FFECE4
:104BD0000F4B70B51D68AC68FEF750FAE37A5A07C0
:104BE00006D4284600F068FABDE87040FEF756BAD1
:104BF000626900230AB11360636104F10C06E37279
:104C0000A3891B04EDD53046FEF710FBF8E700BF83
:104C1000744C002408B5064B1B689B8E03F00303FD
:104C2000012B02D10020FDF7C7F80120FCF7C2FFDD
:104C3000744C002408B580683C3007F080FD0028E3
:104C4000D4BF0020012008BD0023094A10B512F886
:104C5000334002EBC301844204D14878C04300F0E2
:104C6000010010BD01330B2BF1D10120F9E700BF8A
:104C7000087A170838B580684AB10023194A12F833
:104C8000335002EBC304A94214D16468B4B9EFF302
:104C9000118400238022EFF3108372B682F311880F
:104CA00083F310883C30E4B207F039FD84F31188B7
:104CB000002414E001330B2BE1D1E8E7EFF3118579
:104CC00000238022EFF3108372B682F3118883F3FE
:104CD00010883C30EDB207F016FD85F311882046B0
:104CE00038BD00BF087A17082DE9F0438668002414
:104CF000104D4FF002093C36A04685B0304607F013
:104D00001AFD6B6873B12F7801A90022CDF80C90C1
:104D10003846CDE90138012300F02EFA39463046F5
:104D200007F0F1FC013408350B2CEAD1002005B066
:104D3000BDE8F083087A170838B505464C2007F01F
:104D400047F8044630B10122002107F0AAFC0020F8
:104D5000AC6238BD6FF00B00FBE710B5846A2046EB
:104D6000FEF7F8F92046BDE8104007F019B8FFEC4F
:104D70002DE9F0410C4616469846054600284ED0CF
:104D8000002A4CD000294ADBEFF311870023802250
:104D9000EFF3108372B682F3118883F310884368AF
:104DA0000BB1FFF759F91F4901346E600E68C5F861
:104DB0000C801EB9284607F0ABFB24E03046324693
:104DC000002391685B1801D5116831B9A3420CDC4E
:104DD000116829B9E41A1349ECE710460A46F0E7CE
:104DE0008868034410460A46F0E791689642A3EBB0
:104DF0000103A4EB0304A1EB040191600AD109496A
:104E0000284607F08FFBAC60FFB287F311880020C3
:104E1000BDE8F081034A294607F08AFBF3E76FF00B
:104E20001500F5E75854002438B50D4C236843B1FC
:104E30009A680025013A9A60236813B19B68002B99
:104E400000DD38BD204607F097FB23681BB19A6848
:104E500081680A449A6043684560C0689847EBE7F8
:104E600058540024431E012B37B50D460CD8084674
:104E7000FDF71EFF0446002C36DA6442FCF792FF71
:104E800004604FF0FF342FE0002830D16846FDF772
:104E90000FFF04460028EED1EFF31183002280219A
:104EA000EFF3108272B681F3118882F310881149F2
:104EB000DBB2009A0868496802440092019A0A44E9
:104EC000019283F311880C4A019B934208DD0B4841
:104ED000009A93FBF0F10A4400FB11330092019316
:104EE000009B2B60019B6B60204603B030BD6FF0D0
:104EF0001504C2E77C4B0024FFC99A3B00CA9A3BC9
:104F000002680B689A4204D306D840684B68C01AFE
:104F100070474FF0FF307047012070477FB50E4655
:104F200069461546FFF79EFF044608BB69463046B2
:104F3000FFF7E6FF002805DA4FF0FF332B6020462D
:104F400004B070BD019B7468009AE41A3368002CA9
:104F5000A3EB02030394029304DA064A013B2244C2
:104F600002930392294602A807F056FB0446E6E79F
:104F70001624E4E700CA9A3B38B5036C04466BB9C3
:104F80000023236438BD06F00BFF236C5859043509
:104F90000028F8D1184606F003FFF1E70025F4E7F2
:104FA00070B5036C05460C4653F8210006F0F8FE78
:104FB000A1002A6C0B1DD05842F824000134286C43
:104FC000C658002EF4D1012C03D106F0E9FE2E6460
:104FD00070BD083106F0F4FE0646F8E700230246ED
:104FE000012110B5044618460BF0C2FD00232246ED
:104FF000062101200BF0BCFD0023224606210220E1
:105000000BF0B6FD002010BD0F4B10B51B68044619
:10501000B3F93620002A0ADD1A7C037C9A4206D2B4
:105020000A4900F029F80123002023770AE0064905
:10503000204600F021F802230028F5D00322227731
:105040002268137710BD00BF744C0024684C002404
:1050500038B5436804465BB90368032201251A7713
:105060002046044907F0B8FA00232846237738BDC4
:105070000025F5E7744C002410B50B68027C5BB189
:105080001C7C944206D25A68C0E900328AB9586042
:10509000086007E01B68F2E74A68036022B94360D2
:1050A000C1E90000012010BD42601060486000208E
:1050B000F9E710605860FAE738B50446EFF3118558
:1050C00000238022EFF3108372B682F3118883F3FA
:1050D0001088037F043B032B0BD800F0A1F90423B5
:1050E00007212046238700F087F9EDB285F3118868
:1050F00038BD072105F034F9F7E7FFEC38B5124B5E
:105100001D68E8B1EFF3118400228021EFF31082D3
:1051100072B681F3118882F31088028812B2002AD5
:105120000BDD0288013A12B20280FEF723FA00205A
:10513000A865E4B284F3118838BD6FF00A00F8E77F
:105140006FF01500F8E700BF744C002410B5EFF3C2
:10515000118400238022EFF3108372B682F311884A
:1051600083F310880349E4B207F0D2F984F311887D
:1051700010BD00BF505400242DE9F04F1746554A8A
:105180001F2885B0D2F800A005460C46DAF8089032
:1051900004D96FF0150005B0BDE8F08FD9B92946E4
:1051A0004846FFF7F9FB0646FFB994B12768012F7F
:1051B00032D13A4629465046FFF75CFD07468FBB81
:1051C0003EB1304609F12C0107F0C0F93046FFF737
:1051D000BDFF0020DFE7002BE1D10B68012BDED003
:1051E000FFF732FD0028DAD1D3E729465046FFF712
:1051F00021FD30B100230122C7E900230223BB6057
:10520000D3E72EB173683B60B3687B60F368F6E761
:10521000C7E90066BE60C8E7002229465046FFF78E
:1052200029FDCCE7E6B9EFF3118B4FF0800A00239C
:10523000EFF3108372B68AF3118883F3108826483F
:105240005FFA8BFB07F098F906468BF31188DFF8BD
:1052500088B05EB109F12C013046357407F058F979
:1052600077606368B360A368F360B2E7502006F02C
:105270009FFD0646C0B1EFF31183EFF3108872B6BD
:105280008AF3118888F3108800F15002304659469D
:105290001436CDE9022307F03BF9029A039B9642AC
:1052A000F4D1DBB283F31188EFF31183019A0293F7
:1052B000EFF3108272B68AF3118882F31088584691
:1052C000019207F059F9029B0646DBB283F311887D
:1052D000BFE700BF744C002450540024027F062A0C
:1052E0000AD140F2FF22A0F87420742280F87620C0
:1052F0000022826705F076B97047FFEC394B2DE943
:10530000F74306460D4691461C68EFF311880023CB
:105310008022EFF3108372B682F3118883F3108832
:1053200007682046FFF71CFB38405FFA88F70190BA
:10533000A0B101A8FEF762FA01462046FEF70CFA7A
:105340001DB143682B6083686B600679FEF728FA0D
:1053500087F31188304603B0BDE8F08333682366D5
:10536000B9F1000F32D0D9F8040004F13C081E4A0C
:105370000023C117D9F800E08018DFF878C01B4A75
:1053800041F10001EEFB0C0112F092FA23460146B6
:10539000174A4046FFF7ECFC2046062104F0E0FFE8
:1053A0004046FEF759FE94F8741000231F29236627
:1053B00011D8304607F0C3F980B194F87460002D1D
:1053C000C6D0636F2B60A36F6B60C1E706212046D8
:1053D00004F0C6FFE7E76FF00A06F0E76FF0030698
:1053E000EDE700BF744C00243F420F0040420F0025
:1053F000DD52020800CA9A3B38B50C46074B0546F9
:1054000053F8311003EBC4031B79DB0703D5FFF717
:1054100033FE2C7738BD07F0C9F8FAE7BC791708D6
:10542000054B027F10B553F83210044607F0D4F84C
:105430000023237710BD00BFBC79170800F01AB80D
:1054400038B50D4604462F21284608F022FD00B14C
:10545000451C284606F051FF031E08DB06F060FFDE
:10546000C368236083682362436823770023184658
:1054700038BDFFEC014800F003B800BFA8040024C9
:1054800010B5044648B1FDF7F9FD054B1A682260D6
:105490001C60FDF703FE002010BD6FF01500FBE758
:1054A0006054002437B504460D46002001A911F0D0
:1054B00099F8019B642B05D0642301A90020019376
:1054C00011F05EF800F012F82946204600F02CF8A2
:1054D000044611F02DF80449224600F51A7008F030
:1054E0002AFA012003B030BD1B35160808B500F0BC
:1054F00007F800214FF60170BDE8084009F0B7BA7F
:10550000002307B5054A00930123054905480BF020
:10551000C1FCC01703B05DF804FB00BF423516089C
:10552000493516084E35160870B5054601200E4659
:1055300000F0EEF8044670B100F0BCF9204600F02F
:10554000C1F9334601212A46204600F085FC636AF2
:105550000146204698476FF00B0070BD00F529709A
:10556000704770B504460E461546B2B1D0F8943275
:105570003BB1D0F8980208F0EDF8D4F8940208F0A6
:10558000E9F8D4F890322B60D4F88C326B60D4F800
:105590009832AB60D4F89432EB600023C4F88C628C
:1055A000C4F8943270BD38B50446D0F8945210F067
:1055B000BFFF00F59C70854209D110F0B9FF00F5DE
:1055C0009C7008F0C7F80123C4F88C3238BDD4F8B9
:1055D000940268B108F0BEF8D4F8940207F026FFF0
:1055E0004FF0FF33C4E9A3330023C4E9A533EDE74B
:1055F000D4F88C020028F3DB0128F1D00AF0F9FB83
:10560000EEE738B50D460446FFF7CDFF2B68C4F82A
:1056100090326B68C4F88C32AB68C4F89832EB688F
:10562000C4F8943238BDFFEC10B5D0F8943204467B
:105630000BB1002010BD0949D0F88C0207F0BAFE6A
:10564000C4F8940230B1D4F88C32C4F89802C4F88B
:105650009032EEE74FF0FF30ECE700BF663C1608F3
:105660000EB417B50446FFF7DFFF58B906AA05992F
:10567000D4F89802019208F06BF903B0BDE810402D
:1056800003B070474FF0FF30F7E70EB417B504468C
:10569000FFF7CAFF58B906AA0599D4F894020192F7
:1056A00008F056F903B0BDE8104003B070474FF062
:1056B000FF30F7E770B505460C461646FFF7B4FF16
:1056C00068B92046D5F894323246012107F0BFFF71
:1056D0000446D5F8940208F03DF8204670BD4FF01E
:1056E000FF34FAE710B50446FFF75DFFD4F89C02DB
:1056F00008B106F055FB2046BDE8104006F050BB4F
:105700000C4608B5FFF7EEFF2046FCF753FAFFEC16
:1057100038B505464FF4497006F05AFB044638B3D5
:10572000144B154A0360154BC2618360144B154A34
:10573000C360154B02624361144B80F888520361C9
:10574000134B8361134B4362022380F82B32C0F862
:10575000903210F0EDFE012300F51A70C4F88C327F
:10576000C4F8980210F0E4FE00F59C70C4F89402AE
:10577000204638BD9957020863550208E5560208CD
:10578000B5560208035602088B56020861560208F5
:105790005D5502080157020808B590F88802FFF726
:1057A000B7FF08BD2DE9F74F0D461146044600F03E
:1057B000BBF80646F8B1A36920469847074600287B
:1057C00068D036493046D4F8308207F00AFEC4F873
:1057D0003002B0B92769FCF7E5FA006808F014FB5D
:1057E0002F4B2A462F4900902046B847304600F0FC
:1057F000BFF8C4F830824FF0FF35284603B0BDE84B
:10580000F08F4FF0FF35DFF8A890DFF898A010F088
:105810008FFE00F59C7007F09DFFD4F8300207F072
:105820008EFE0023C4F834029842A4F838320CDA11
:10583000D4F810B0FCF7B6FA006808F0E5FA1A4B95
:1058400000904A4651462046D847D4F8302280215D
:10585000384607F09CFE98B194F82B329A0704D48E
:1058600063693A461149204698473946204601F077
:10587000E5FD05460028CAD094F82B32DB07C6D4D4
:10588000D4F8300207F0D2FDC4F83082304600F080
:105890006FF8B2E74FF0FF35F8E700BFAB3A1608F4
:1058A00058351608C17A17085E3516083D83160864
:1058B00064351608014A0249FFF774BF69351608B6
:1058C0007835160838B50446FDF7D8FB084B012299
:1058D0001D781A70FDF7E2FB45B9064A20460649D5
:1058E000FFF760FF022384F82B3238BD0020FCE76D
:1058F000645400248035160858C8160808B50249B3
:1059000043699847002008BD785C170808B504482B
:10591000FDF7E4F9034B002808BF184608BD00BF97
:10592000697A1708607A170870B506460C4609B1FF
:105930000B7823B90C48BDE8704008F057BA2F2BFC
:1059400001D10846F7E7FFF7E1FF08490546204681
:1059500008F0F4FA08B92846EDE722462946304611
:10596000BDE8704000F066BC607A17081B0F17088E
:1059700008B106F015BA704701292DE9F341064632
:1059800017464EDD55682949284608F0D7FA0446DF
:10599000002847D02649284608F0D0FA044650BBD4
:1059A0002448FDF79BF9244B002808BF184608F04F
:1059B0001DFA804608F004FD054670B13F68356960
:1059C000FCF7F0F9006808F01FFA1C4B00903A460B
:1059D0001B493046A8474FF0FF35B8F1000F02D001
:1059E000404606F0DDF914B12046FFF7C1FF284616
:1059F00002B0BDE8F0811349284608F09FFA04463A
:105A000038B9FFF783FF08F0F1F9804606F022FD70
:105A1000D0E729463046FFF787FF4FF000080446DD
:105A2000C8E70024A0460448C4E700BF9035160824
:105A3000873A1608627A1708607A170892351608AE
:105A4000C17A1708683F17082DE9F04F012387B086
:105A5000074690464FF0000A5F4C029101932246A0
:105A60004146029808F066FC431C10D108F06FFC18
:105A7000D0F800904FF05C0B08EB8908029B994529
:105A80001FDB019B002B40F0A18000200DE065286A
:105A90000ED06E280FD0452810D03B693846D8F874
:105AA00000204E4998474FF0FF3007B0BDE8F08F17
:105AB0004FF0010AD3E700230193D0E74FF0000A2B
:105AC000CDE708F044FC03684B4503D07B693846BA
:105AD00043499847BAF1000F63D0D8F800502C46DC
:105AE0002B780BB923705CE05C2B04D02E4604F8B5
:105AF000013B751CF4E76B786E1C0D2B0AD80D2B3F
:105B00000ED8DFE803F04A0D0D0D0D0D0D57590DA0
:105B10005D615B5F5C2B35D0782B08D0302B16D0C5
:105B2000234603F802BB6A7862701C46E1E703353E
:105B30000023049616F8012F05931046039206F0F1
:105B400010FC059BDDE90321A0B90E461AE00435DF
:105B50000021737832460136303BD8B2082803D989
:105B6000164604F8011BC4E7AE4203EBC101F0D1B5
:105B70003246F5E7A2F130011B01092905D80B4493
:105B8000AE42D6D104F8013BB3E71046039306F0CA
:105B9000F6FB039B57380344F2E7002384F800B078
:105BA00063707B69384658F8042B09F101090D49E7
:105BB000984763E70723E5E70823E3E70C23E1E7DA
:105BC0000A23DFE70D23DDE70B23DBE77B6938469C
:105BD0000549984759E700BF98351608877B17088D
:105BE000BA3C16083D831608AC1F170838B50446A2
:105BF0004569FFF78BFE034902462046A84700206F
:105C000038BD00BF785C17082DE9FF474E4B16469C
:105C10000DF10C0801291A8804469B780D46ADF851
:105C20000C2088F802300DD10022484900F0D4FB46
:105C3000054663692046ED1745499847284604B054
:105C4000BDE8F087022901D0042968D17768384679
:105C500008F093F901280FD836682569FCF7A2F8F7
:105C6000006808F0D1F83B4B32463B490090204693
:105C7000A8476FF01505E1E797F80090B9F12D0FEF
:105C80000ED0B9F12B0F0BD036682569FCF78AF8D6
:105C9000006808F0B9F82F4B324630490090E6E72B
:105CA0004FF0010A17F8011F11F0DF0F22D1022374
:105CB000033D012D46D801339D0056F8230000F026
:105CC0009BFA0746043D7059FDF708F848BB715927
:105CD0003A46204600F022FB051EAFDA68422769EB
:105CE000366808F091F81E4B009032461D49204658
:105CF000B847A3E7404608F017F90028C4D0A0EB46
:105D0000080394F82B22B9F12B0F0AFA03F30ABF08
:105D1000134322EA0303DBB284F82B32C2E70123E8
:105D2000C6E7705901223946FEF7ACFA051E85DA3E
:105D300027693668FCF736F8006808F065F80A4B02
:105D40000090D2E7002579E79D141708FD58020856
:105D5000AC1F1708B6111708BB7B1708877B1708FD
:105D60009C351608C17A1708B6351608F7B551687C
:105D70000446154600F00CFB002825DA831C23D0CE
:105D80002F684042266908F03FF8104B3A460090D1
:105D900020460F49B0474FF0FF366868FEF7E0FA3B
:105DA00000280EDA2D682669FBF7FCFF006808F072
:105DB0002BF8084B00902A4605492046B0474FF083
:105DC000FF36304603B0F0BD0026E6E7A7351608DB
:105DD000C17A1708B4351608032973B50546144669
:105DE00017D1916801226068FEF74CFA002819DA91
:105DF0002E692468FBF7D6FF006808F005F8124BFF
:105E00000090224611492846B0474FF0FF3002B0BB
:105E100070BD516800F076FA0D4B002814BF0146A2
:105E20001946DFE76168284600F0B2FA002809DA6F
:105E3000831C07D040422E69246807F0E5FF054B1C
:105E40000090DEE70020E2E7B4351608C17A1708B3
:105E500081DF1608A7351608F7B5044617461D4614
:105E600041B1D0F89412374807F036FDD4F89402C7
:105E700007F070FC012F29DC334F04F52976D4F8A4
:105E80009412384607F028FDD4F8940207F062FC1B
:105E900010F04EFB054610F04BFB802100F59C7383
:105EA00005F10802304600F0B0FA013040D1D4F8D4
:105EB0009842FBF777FF006807F0A6FF234B00909E
:105EC0002046234A234907F036FD0AE06E6822493E
:105ED000304608F033F830B9636920462A681F4914
:105EE0009847002013E01E49304608F027F880B993
:105EF000022F06D0A968204603B0BDE8F04001F0AB
:105F00009DBA23692A68174920469847012003B0A3
:105F1000F0BD337829682D2B03D10A462369124935
:105F2000F2E73246204603B0BDE8F040FFF73ABC46
:105F30003146204601F082FAD4F8940207F00AFCB8
:105F40009DE700BFFF7B1708F97B1708EB351608A4
:105F5000F4351608C17A1708BD351608C03516087D
:105F6000E8351608BB7B1708E27B17082DE9F74FC9
:105F700004460D461046012116460AF0A5F9071EF3
:105F80001DDA05223F49304607F073FF28B927691B
:105F900033462A463C492046B8472669FBF702FFAC
:105FA000006807F031FF394B00904FF0FF392A4667
:105FB00037492046B047484603B0BDE8F08F4FF45C
:105FC000007005F0F5FE064658B9384609F011FF95
:105FD0002669FBF7E7FE006807F016FF2D4B0090DF
:105FE000E3E74FF00009DFF8B4A021E007F00CFF71
:105FF000294B00902A4626492046C0472CE02DD048
:106000004FF00008E368ABEB080206EB08012046FE
:106010009847002832DAFBF7C5FE0068D4F81080F4
:10602000042822D12A4651462046C0474FF0FF3966
:106030004FF40072314638460AF080F9B0F1000B97
:10604000DDDAFBF7AFFE0068D4F810800428CDD16C
:106050002A4612492046C0474FF0FF39384609F01A
:10606000C8FE304605F09CFEA5E707F0CDFE0C4BC0
:1060700000902A4606492046C047D7E78044C345DA
:10608000C0DCD5E70036160806361608593516085E
:10609000C17A1708373616080A571608707A170893
:1060A0008FBB16082DE9F74F05468846104601219B
:1060B0001F460AF009F9061E11DA2C694FF0FF3A63
:1060C000FBF770FE006807F09FFE1D4B00904246F4
:1060D0001C492846A047504603B0BDE8F08F0C9BF2
:1060E0000024B94603F1FF3B3C705A46494630460E
:1060F0000AF024F9B0F1000A16DAFBF753FE036840
:10610000042B19D02C69FBF74DFE006807F07CFECC
:106110000D4B009042460B492846A0474FF0FF3AEE
:10612000304609F066FED6E7FAD054444FF000033B
:10613000D144ABEB0A0B3B550C9B002BD5D1EDE7C3
:1061400059351608C17A17080A5716082DE9F34180
:10615000044610460F461546984606F016F90646C0
:10616000E8B905221749284607F083FE28B92669B1
:106170002B463A4614492046B0472569FBF712FEE4
:10618000006807F041FE009020464FF0FF340F4BAF
:106190003A460F49A847204602B0BDE8F081304694
:1061A00006F021F9024658B1089B29462046C0470F
:1061B0000028F4DA4FF0FF34304606F001F9EAE740
:1061C0000446F9E700361608063616083E36160865
:1061D000C17A170810B5044607F0CFFE0021231836
:1061E0001A1B013A002A03DD13F8012C2F2A00D0D4
:1061F00010BD03F8011DF3E7F8B5044620782546E5
:106200002646013468B92846002707F0B6FE2C1848
:10621000B44204D014F8010C06F099F830B92846BD
:10622000F8BD06F094F80028E8D1ECE704F8017D09
:10623000EEE7FFECF7B50D46044610491646284632
:1062400004F1280707F07AFE78B933460C4A4FF478
:106250000071384606F0F9FA0023384684F82831F0
:1062600003B0BDE8F04007F0C1BD2B46054A4FF42E
:1062700000713846009606F0E8FAEDE732D41608C9
:10628000DD341608DB34160870B5D0E9A7450E4694
:106290002544AC4212D2701E611E10F8012F11F875
:1062A000013F9A42F9D01AB93D2B01D1204670BD69
:1062B000204607F062FE01300444EAE70024F5E7D7
:1062C00070B5D0E9A73605460C468B421E4416D859
:1062D0008E4214D9084607F050FE0130631E044474
:1062E000321B002A06DCD5F8A0321B1A0020C5F8A4
:1062F000A03270BD14F8012B03F8012FF0E74FF026
:10630000FF30F6E708B5FFF7BFFF034618B13D21A0
:1063100007F00AFE431C184608BDFFECF8B5D0F89C
:106320009C3205460E46174633B1FFF7ADFF0146D6
:1063300010B12846FFF7C4FF304607F01EFE0446A2
:10634000384607F01AFE0444D5F89C020234B0B176
:10635000D5F8A0321C44214605F032FD024610B9A2
:106360006FF00B00F8BDD5F8A03218443B46074942
:10637000C5E9A724324606F044FA0020F2E7204699
:1063800005F016FD0028EBD00246EFE7153516089C
:1063900010B5044698B1FFF777FF014678B1204663
:1063A000FFF78EFFD4E9A70100290CDC20B105F02E
:1063B000F7FC0023C4F89C320023C4F8A032FCF799
:1063C0006DFE002010BD05F0FBFC10B1C4F89C026E
:1063D000F5E76FF00B00F5E72DE9F041D0E9A746AE
:1063E00005460F4690462644B44202D30020BDE83D
:1063F000F081224641462846B8470028F7D120467A
:1064000007F0BBFD01300444EEE75B68526800F022
:106410002FB800690AF07CBA13B504468DF807104E
:1064200001220DF1070120690AF072FA002802DB4F
:10643000F6D002B010BDFBF7B5FC0368042BF7E7FC
:1064400013B5044601220DF10701E06809F076FF5B
:10645000002809D003DB9DF8070002B010BDFBF750
:10646000A1FC0368042BEDD04FF0FF30F5E7FFEC03
:1064700010B586B0074C0492074A01940292074A6D
:10648000059303920A46014601A800F009F806B0F8
:1064900010BD00BF416402081964020813640208B9
:1064A000012A2DE9F04706460F46914604DC0024F8
:1064B0000C702046BDE8F0870025836803222C4934
:1064C00098474FF00008336830469847431C04460D
:1064D0000BD1002DEDDD00232C467B55E9E74FF075
:1064E0000108F0E74546D046EDE7B8F1000F09D0C6
:1064F0005B28E6D1B8F1020818BF4FF001084FEA57
:106500004808E0E71B28EAD012DC0A2812D00D2840
:1065100010D0082817D1002DD5DD7368304608212A
:10652000013D9847B3680322114930469847CAE7AE
:106530007F28EFE76C1C0A210023304679553B5534
:1065400073689847B5E7E0B205F0F8FE8246002888
:10655000B9D17C5505F101080235736821463046F2
:1065600098474D45BEDB444607F808A0A1E700BFA9
:106570006D7A170890F83B220346043200EBC20202
:1065800092F82802800901280CD1002081F0010135
:1065900083F82A0292F8283261F3000382F8283245
:1065A00000207047022803D1002083F82A02F1E777
:1065B00093F83C221A4492F83D02800901280CD13C
:1065C000002083F82A0292F83D32C3F38000414054
:1065D00061F3000382F83D32E2E7484283F82A1271
:1065E0007047024610B50023104612F8014B5C2C90
:1065F00000D143B18C4202D1002BF4D110BD002C4C
:10660000F1D12046FAE70123EEE70023027802B930
:1066100070475C2A00F101010AD14BB903465A7850
:1066200003F8012B002AFAD1014601230846EDE7C1
:106630000023FBE790F83B32024600EBC30393F8DC
:1066400048329909032902D113F001000CD092F8C5
:106650003C321A4492F83D0283070CD48309022B82
:1066600005D0032B04D0012000F001007047C04387
:1066700000F00100F8E70020F6E770B50568044671
:1066800095F8293213B1406809F0B3FBAB6828468E
:1066900004F1080600259847A368AB4204DC2046B5
:1066A000BDE8704005F07CBB56F8040F013505F0DD
:1066B00077FBF1E72DE9F041804617460C46B9B16A
:1066C000084607F05AFC0646384607F056FC411CBF
:1066D0002046314405F074FB054658B92546D8F8E4
:1066E0001030074A4046074998472846BDE8F081E0
:1066F0000E46E9E700233946835507F059FBF4E7D6
:1067000046361608A97A170838B500F10C028168D8
:106710000446006801F09AF805462046FFF7ADFFF1
:10672000284638BD2DE9F04F89B089460446154604
:10673000129F1E460097116802F042FA002808DBFB
:1067400014BF01210021204609B0BDE8F04FFFF73A
:1067500011BF94F82932B3B139464FF4DB72304699
:1067600009F0B2FD071E10DA2D682669FBF71AFB47
:10677000006807F049FB554B00902A4654492046D3
:10678000B0470121DFE74FF0FF3794F82832002BA4
:1067900000F08380236820469847804640B15C2003
:1067A00005F016FB064658B9D8F808304046984719
:1067B00094F82932002BE4D0384609F01AFBE0E7C0
:1067C00083464FF0000AC0E900874BF8089FD14587
:1067D0001EDC94F829322BB1D8F81C30002239463F
:1067E0004046984702A900200FF0FCFEC8B1276977
:1067F0002D68FBF7D7FA006807F006FB354B0090D1
:106800002A4633492046B8473046FFF736FFB8E7F7
:1068100055F82A000AF1010A07F0E8FA4BF8040FCC
:10682000D5E7D4F82C32002B0BD0029F4FF001009B
:10683000A7EB03071EDA05F0DDFE8742A8BF074677
:10684000029704A805F032FE012104A805F03CFEE1
:1068500002A904A805F040FE33461F4A04A903A874
:1068600005F048FE60B127692D6807F0CDFA1B4B93
:106870000090C5E705F0C0FE8742B8BF0746DFE7D6
:1068800003980FF0FDFD029B154920460093039BE2
:1068900066692A68B047002155E794F8293223B188
:1068A000E36904AA3946204698472A4649462046C5
:1068B00000F0CCFF94F8293205461BB1236A04A9E5
:1068C00020469847002DE6DA5BE700BF59351608E9
:1068D000C17A17084836160809670208563616089E
:1068E00065361608F8B50025044606462F46236887
:1068F0009D4201DB2760F8BD56F8040F013505F015
:106900004FFA3760F3E7FFEC2DE9F04F0446BDB0D6
:106910000E46D1F80090A44F0592039399F8008099
:106920004D4609F10109B8F1000F17D0414638462C
:1069300007F0FAFA0028F1D1B8F13E0F0AD16B78CE
:106940003E2B0DBF0235994DC6F80090356008BF4B
:10695000974D04E0B8F1230F05D135600025284696
:106960003DB0BDE8F08FB8F1220F039B8E4F8246F9
:1069700004BF00234D460393A9468E4B08BF1F4614
:106980000346C84619F8011B69BBC6F80080AA4631
:1069900000268949504607F01BFA83460AEB0B078D
:1069A00007F1010897F80090BBF1000F4DD0B9F145
:1069B000000F33D1002E67D0314652462046FFF7F4
:1069C00079FE0546FFF721FE2E46002EC7D0059B17
:1069D0001B681D2BC3DC059A02EB83020133566052
:1069E000059A1360BBE718B102785C2A00D193B115
:1069F0005C2903D0602903D18AF0010A00230BE04F
:106A0000BAF1000FFAD13846FFF7EBFD0028F5D0B8
:106A100008F801ABB9E701234046B2E70BF1FF33B9
:106A200000225344A3EB0B0013F801195C2903D196
:106A3000834282F00102F7D152B10BF1010B5E49A2
:106A4000781C07F0C5F98344A8E7B9F1000FB1D06D
:106A5000B9F1600F40F059814FF0000331465246C2
:106A6000204607F8013BFFF725FE49460646384613
:106A7000FFF7B7FD049058B9504B25691A465049A5
:106A80002046A8474F4DA0E72846FFF7BEFD66E722
:106A9000049B4FF000021A7000230793FDF798FA49
:106AA000494A0346494907A805F0C2FE002804DB0D
:106AB000DDF81C90B9F1000F18D123692046444A33
:106AC000444998474FF000083E4F31463A46204629
:106AD000FFF7F0FD0646B8F1000F02D0404605F082
:106AE0005FF9049B03F10108C24652E750220021DE
:106AF00009A8FBF7B8F87C2200211DA8FBF7B3F822
:106B00004FF48073B4F828B21DAAA4F8283208A95B
:106B1000002320460897FFF7F7FE074668B3204694
:106B2000FFF788FD40B30DF1240A4FF001080997E3
:106B300000231DAA08A92046FFF7E6FE4AF8040F25
:106B400020B108F10108B8F1130FF1D13CAB0022DC
:106B5000B8F10F0F03EB880343F8CC2C04DD236955
:106B60003A461D4920469847262309AA4146204611
:106B700000934B46FFF7D6FD07461DA8A4F828B2A0
:106B8000FFF7B0FE77B32769FBF70CF9006807F051
:106B90003BF9124B009020460D4A1149B84707981F
:106BA00005F0FEF88EE700BF327C1708287C170836
:106BB000257C17084D3A16082A7C170884361608D3
:106BC000A27B17081E7C1708713616087636160841
:106BD00083361608A97A1708187B17088636160810
:106BE000C17A1708DDF81C801DA9404609F0DCFDBC
:106BF000834620B32769FBF7D5F8006807F004F94E
:106C00006F4B009020466F4A6F49B8474FF000081D
:106C10006E4F079809F046FE00280CDAD4F8109061
:106C2000FBF7C0F8006807F0EFF8694B00902046CA
:106C3000644A6549C847079805F0B2F845E7DDF8AA
:106C40008C9009F1010005F0B3F8074628B92369D3
:106C500020465C4A5F499847D8E74046012109F041
:106C600033FBB0F1000833DAD4F81080FBF79AF860
:106C7000006807F0C9F8584B00902046514A524925
:106C8000C047384605F08CF8C0E74FF40072404624
:106C900009F054FB00281ADAFBF784F80368D4F8EB
:106CA0001090042B07D1474A20464C49C84740461C
:106CB00009F09FF8E5E7FBF775F8006807F0A4F81E
:106CC000474B009020463F4A3F49C847EFE783447F
:106CD000D94507EB0B01D8D88A46DFF82091BA4591
:106CE00007D01AF8011C48460AF1FF3B07F01CF9CF
:106CF00048B90023AAEB070A4046B84607F80A300D
:106D000009F077F885E7DA46E9E7B9F1240F7FF46F
:106D1000EBAE4FF00003B9463146524609F8013B4D
:106D20002046FFF7C7FC7B7806467B2B32D107F164
:106D300002097D214846FFF754FC18B92569294B03
:106D4000294A9CE680464FF0000308F8013B039B6C
:106D500013B10123039A13602449484607F0EEF863
:106D6000F0B994F82A12224A224F00290CBF924609
:106D7000BA4694F82B329B0705D453464A461E491F
:106D800020466769B847314652462046FFF792FCD5
:106D90000646A9E6484607F0F0F809EB0008D6E7F2
:106DA00049462046FFF7AEFA82460028E1D1484620
:106DB000FBF794FF054B002814BF82469A46D8E79C
:106DC0008B36160883361608C17A17081E7C1708FA
:106DD00090361608A97A170859351608707A1708D8
:106DE0000A571608AAC0160897361608237C1708F3
:106DF000217C17081F7C17089A361608327C170862
:106E00002DE9F04FB9B004460D465022002105A8E7
:106E1000FAF729FF7C22002119A8FAF724FF0023A2
:106E200019AA03A92046A4F828320395FFF76CFDA0
:106E30000546002800F03082A64907F07FF8814619
:106E4000A549284607F07AF8B9F1000F02D00028CA
:106E500040F08C80002319AA03A92046FFF754FDB7
:106E6000074608B103781BB923692A469B4925E0E8
:106E700094F83C8204EB080393F83D329B09012B04
:106E800014D094F83B6204EBC60393F84832C3F382
:106E90008113033303F00303012B07D9D4F83032F5
:106EA00023B1D4F834A2BAF1000F02DA23692A46DA
:106EB00078E0062E1BD923692A468949204698473F
:106EC00094F84832002203F03E03A4F83A2243F03B
:106ED0000103C4F84C2284F8483219A8FFF702FDD8
:106EE0000121204639B0BDE8F04FFFF743BB013622
:106EF000B9F1000F2046F6B214BF02250125FFF7B5
:106F000099FB321D002384F83B6204EBC60604EBB8
:106F1000C20284F83A3240EA8513B4F8381292F883
:106F200028023D4623F03E03514400F03E00034357
:106F300082F8283286F84982C6F84C1269492846F8
:106F400006F0FCFF0746002840F03181034619AAED
:106F500003A92046FFF7D8FC054618B10378002B9B
:106F600040F08B8023695F4A5C49AAE05E4928466D
:106F700006F0E4FF034608BB19AA03A92046FFF761
:106F8000C3FC94F83B320546043304EBC30393F887
:106F90002812C1F38112033202F00302012A03D93D
:106FA0002369514A514989E741F0C00183F8281209
:106FB0000028C3D10023C4F82C3259E14C4928469B
:106FC00006F0BCFF0346002848D119AA03A92046B1
:106FD000FFF79AFC024610B12369454A46E794F848
:106FE0003B02031D04EBC30393F828128D09032D04
:106FF00002D023693E4AD5E718B923693C4A3D4986
:107000005CE7C80725D5D3F82C12D4F8300206F077
:1070100076FA00280BDA2569FAF7C4FE006806F054
:10702000F3FE354B00902046314A3449A8470123EE
:1070300084F83A3294F83B321A1D013B04EBC20249
:1070400092F8281221F0C00182F8281284F83B320D
:10705000B0E741F0010183F82812EBE794F83B32E6
:1070600004EBC30393F84832C3F38113033303F0F3
:107070000303012B3FF662AF18E7214906F05EFFDC
:10708000034668B919AA03A92046FFF73DFC054647
:1070900000283FF467AF0378002B3FF463AF01276C
:1070A00094F83C62A31993F83D329B09012B03D15C
:1070B00023690C4A0D4904E0062E23D92369094AA5
:1070C000074920469847B4F83C3203F46053A4F8CB
:1070D0003C3202E7A3361608A9361608877B170844
:1070E000FD7A1708BD361608AF361608D97A170884
:1070F000B2361608907A1708B7361608C17A1708FC
:10710000D348170820460136FFF794FA80F00103B0
:10711000F6B25B0084F83C62264443F0400396F8E4
:107120003D2243EA870302F0380223F03803134379
:1071300086F83D320023C4F82C32B349284606F0C5
:10714000FDFE0346002840F0B2800A2203A9204633
:10715000C4F82C2219AAFFF7D7FB0546002800F037
:107160008780AA4906F0EAFE0646002840F09F8084
:10717000034619AA03A92046FFF7C6FB07460028C5
:1071800000F09580324604A906F09FFCC4F82C025A
:107190001430272805D8049B9F4202D01B78002B6F
:1071A0007DD023692046984A9949984795E69949A0
:1071B000284606F0C3FE0346D8B919AA03A92046FB
:1071C000FFF7A2FB94F83C220546224492F83D3298
:1071D0009909012902D023698E4A6BE7022161F3E4
:1071E000871382F83D320023C4F82C32002DA4D13D
:1071F0003EE08949284606F0A1FE0346A8B919AA2F
:1072000003A92046FFF780FB94F83C32054623444F
:1072100093F83D229109022902D023697E4A49E769
:1072200042F0C00283F83D22DDE77C49284606F0A3
:1072300085FE034620BB19AA03A92046FFF764FB7D
:1072400010B12369754A8FE694F83C32E21892F83F
:107250003D227F2A02D82369704A2BE71BB9236994
:107260006F4A70492DE7013BC4F82C0284F83C3288
:10727000002519A8FFF736FB284639B0BDE8F08F86
:1072800094F83C32234493F83D329B09012B7FF460
:1072900051AF23692A460DE7C4F82C02E8E719AA82
:1072A00003A92046FFF730FB05460028E0D0204622
:1072B000FFF7C0F90028DBD001264FF00008DFF807
:1072C0007891059504AB19AA03A92046CDF8108042
:1072D000FFF71AFB38AB07464FEA860A03EB860333
:1072E00043F8CC0C00286ED0049BE3B105AB9A4464
:1072F0005AF804BB5F461BF8011BA1B1484606F0D3
:1073000013FE0028F6D0013607F8018BBB4617F8AC
:10731000011B21B1484606F007FE0028F6D1132EC6
:10732000CAF800B0E4D10136122ECBDD771E38AB9F
:107330003D4903EB870353F8CC0C06F0FFFD18B969
:1073400001233E4684F82832022E58DDA6F10209B8
:1073500038AB364903EB890353F8CC7C384606F04A
:10736000EDFDA8BB012394F82982204684F8293238
:1073700038AB03EB860656F8D01C4E46FEF7D4FA1F
:107380004FF02609074638AB00220F2E03EB860389
:1073900043F8CC2C04DD23692A462549204698472A
:1073A0003B4605AA31462046CDF80090FFF7BAF9D2
:1073B000054627B13846FEF7DBFA84F8298219A87A
:1073C000FFF790FA58E7012EB0DC80468146DAE7F5
:1073D0001849384606F0B2FD88B9012394F829828D
:1073E000204684F8293238AB03EB860656F8D01CC9
:1073F0004E46FEF799FA4FF016090746C3E74FF0DD
:107400000008C1464746BEE7CD361608D2361608F4
:10741000877B1708C0361608C5361608CA36160800
:10742000BD361608907A1708D5361608287C170836
:10743000187B1708257C1708327C17082DE9F047C0
:10744000002305460E460C4688461F4F80F83A3208
:1074500095F83AA2BAF1000F01D000202EE0A31B4C
:1074600039462046A5F8383206F0B2FC235C2218D3
:107470001BB10A2B01D0232B05D141462846BDE87C
:10748000F047FFF7BDBC3B2B02F1010909D1414692
:10749000284682F800A0FFF7B3FC78B94C46C846EE
:1074A000D6E722214846FFF79CF848B9074B284603
:1074B0002C691A460649A0474FF0FF30BDE8F08717
:1074C000441CC146EBE700BF2D7C17084D3A160857
:1074D000A27B170890F83B32043300EBC30393F808
:1074E00028229209032A09D193F8292280F83C2204
:1074F00093F8282222F0010283F828220020704706
:1075000008B503490369126898474FF0FF3008BD7A
:107510004E7B1708002070474FF0FF30704708B5CA
:107520000021436A9847FFEC10B4CB680A684469AD
:1075300023B1A44604495DF8044B60472346034940
:107540005DF8044B184700BFD7361608705C170863
:1075500070B504460D460D4E306830B923692A4691
:1075600020460B49BDE870401847294606F0E6FC66
:1075700050B963692A460749204698473146204654
:10758000BDE87040FFF7D0BF1036E5E7387C17083C
:107590004E7B1708E036160801292DE9F74F0446FF
:1075A0000F46164640F3F1809349506806F0C6FC3A
:1075B000054600285FD1022F06D00222012356F88B
:1075C0002250002B00F0DE80636920468B499847EB
:1075D00063698B492046984763698A4920469847E2
:1075E00063698949204698476369884920469847D6
:1075F00063698749204698476369864920469847CA
:1076000063698349204698476369834920469847C0
:1076100063697C49204698476369804920469847BA
:1076200063697F49204698476369794920469847AE
:1076300063697C49204698476369724920469847A8
:107640006369794920469847636975492046984798
:1076500063696F4920469847636972492046984795
:10766000002D00F0C38029462046FFF771FF00205F
:1076700003B0BDE8F08F01220023A0E729461035B2
:107680002046FFF751FF2B68002BF7D100273E461D
:107690003D46384604F044FE002854D1002DE6D083
:1076A0000236013D4FF000086369502E5F492046C5
:1076B00096BF50270127B7FBF6F73D449847B5FB27
:1076C000F7F54545D3D0C1464FF0000A636920461F
:1076D00057499847484604F023FE834640B1DBF8FB
:1076E0000C30002B3AD10AF1010AA9445745F1D1D7
:1076F000636920464F4908F101089847E1E7B94618
:107700004FF0000B4FEA09134B4920465AF803206B
:10771000636901929847019A104606F02EFC0346D1
:107720009D42626908D80BF1010BC1445E4557D0F8
:10773000B9F1240FE6D953E0404920460193904720
:10774000019B0133ECE7C36833B10068013506F0F3
:1077500014FC864238BF064601379AE7DBF8002062
:107760002046636934499847DBF8000006F005FCC1
:1077700083465E45B7D96369204630490BF1010B5A
:107780009847F6E7002D7FF46EAF00262C4920467F
:10779000DFF8B4A03546FFF7DBFE636920462549D4
:1077A00098475AF82600043606F0E7FB854238BFB2
:1077B0000546942EF5D102350027502D96BF502650
:1077C0000126B6FBF5F606F12408B8FBF6F8B84535
:1077D0003FF45CAF6369204615499847242F8ED942
:1077E00063692046134901379847F0E763692046EB
:1077F0001449154D984746E7EA361608ED3616083F
:10780000013716083C371608403716084C3716085B
:10781000543716086D371608753716087C37160862
:107820008B371608913716089A371608AE371608A0
:10783000B93C1608AC1F17083D831608BA3C160859
:10784000A9371608BE371608387C17082DE9F0410D
:1078500004460E461746D2F80080124D286808B933
:10786000114B17E0414606F069FBC8B92B7AB342C9
:1078700008DD236942460D49204698474FF0FF3006
:10788000BDE8F0816B7AB34203DA236942460849C6
:10789000F2E76B683A4631462046BDE8F0411847AA
:1078A0001035DBE7387C170801750208BB7B170829
:1078B000187B170810B50749044606F03FFB38B19E
:1078C0000549204606F03AFBB0FA80F0400910BDA9
:1078D0000120FCE71B0F1708683F17082DE9F0434C
:1078E0009D0795B00446884616461F4670D0E2B103
:1078F0000132FEF79FFC814605A908F055FF0546B9
:10790000484604F04DFAB5B12569FAF74BFA00681C
:1079100006F07AFA434B00902046434A4349A84771
:107920004FF0FF3015B0BDE8F08305A9404608F0E0
:107930003BFF0546E7E7B90743D53D4B02AD186865
:1079400059681A899B7A03C5AB702A80079D05F494
:107950007043B3F5C04F4FD162238DF80830EA056C
:1079600044BF72238DF809302B0644BF77238DF86E
:107970000A30680644BF78238DF80B30A90644BF4F
:1079800072238DF80C30EA0644BF77238DF80D3052
:107990002B0744BF78238DF80E306807204644BF7C
:1079A00072238DF80F30A907224944BF77238DF841
:1079B0001030EA0702AA44BF78238DF811306369BA
:1079C0009847FB0704D5636920460B9A1A499847E4
:1079D000636916B3771C174920463A4698473378AF
:1079E0006569042B17D13846FFF764FF98B913492E
